:020000040800F2
:1040000000500020BD7B0008917A0008957A0008D6
:10401000997A00089D7A0008A17A00080000000043
:10402000000000000000000000000000A97A000865
:10403000A57A000800000000AD7A000889A60008F3
:10404000B17A0008B57A0008B97A0008BD7A00088C
:10405000C17A0008C57A0008C97A0008CD7A00083C
:1040600000000000D17A0008D57A000800000000A6
:104070000000000000000000000000000000000040
:104080000000000000000000F57A0008F97A00083E
:10409000097B0008197B0008357B00080D450008E6
:1040A000457B0008694B0008D1480008000000006B
:1040B00065460008B545000839460008497B0008F8
:1040C0008DBD0008517B000809BE0008597B00081F
:1040D0005D7B0008617B0008F9440008E5440008A6
:1040E0006D7B0008717B0008757B000800000000F4
:1040F00000000000000000000000000000000000C0
:0C41000000000000000000005FF800005C
:10410C0030BF704720BF704740BF7047BFF36F8F01
:10411C007047BFF34F8F7047BFF35F8F704701DF5E
:10412C007047EFF31480704780F31488BFF36F8FE0
:10413C007047EFF30980704780F309887047EFF3FD
:10414C000880704780F30888704772B6704762B673
:10415C00704771B6704761B6704780F3118870472D
:10416C00EFF31280704740BA704700BA70470000F6
:10417C00054A0649064B1160064A1360064A13604D
:10418C00064A1360704700BFAC0400208D920008F3
:10419C00459100088804002058030020800400206A
:1041AC00044B054A1360054A1360054A1360054A1F
:1041BC0013607047459100085803002088040020C4
:1041CC00AC04002080040020704700BF704700BF83
:1041DC0030B597B003F034FA03F052FA0AF078FCD9
:1041EC00594B00244FF480301C700AF091FC0AF0FB
:1041FC00F5FD012832D10F300BF028FB02200BF01B
:10420C000DFB20460AF0D4FC20460AF0E5FC4FF4E6
:10421C0080600AF0D7FC4D4B4D4A1B68934202D18B
:10422C004FF4403004E04B4A934205D14FF48030B8
:10423C004FF4E0110AF098FC01200AF0A1FC39209F
:10424C000AF0B6FD0028FAD002200AF09FFC0AF012
:10425C00A7FC0828FBD13C4B01221A700120014617
:10426C000AF05CFD3C4C4FF480414FF000600AF0CA
:10427C00B7FE4FF440700AF015FEFFF791FFFFF701
:10428C0077FF05F083FA05F0BBFA07F0CBFC03F0DF
:10429C0047FE06F0D5F92046304905F05DFD05F0E6
:1042AC0089FA2F4B1B78012B05D1207804F0F8FCF0
:1042BC00E07804F005FC2B4B1B78012B25D12A4C04
:1042CC000DF1100C25460FCDACE80F00AE46BEE844
:1042DC000F00ACE80F009EE80F0030340DF1400EDB
:1042EC008CE80F000FCCAEE80F0094E8030002241A
:1042FC008EE80300009404AC0194202010AC1B4900
:10430C0004220023029405F07FF800F011FB01F069
:10431C00A5F903F081F940F2167006F001FE40F2A7
:10432C00127006F05BFE03F0A9FA03F071FA01209B
:10433C0002F018FF00F0D4FF03F070F906F026FE2F
:10434C0000F0F0FEF1E700BF9804002050000020C0
:10435C000024F40000127A00B0040020C4030020F2
:10436C0042000020450000206006010800140140B6
:10437C00014B1868704700BF94010020014B58682E
:10438C00704700BF94010020014B1868704700BFB4
:10439C000C090020014B9868704700BF9401002065
:1043AC0008B5024B18680CF02FF908BD480900201D
:1043BC00014BD868704700BF94010020014B18686E
:1043CC00704700BF64090020014B1868704700BF9C
:1043DC0018090020014B1868704700BF2009002005
:1043EC00034B93F8422022EA000283F842207047E4
:1043FC00C4030020034B93F8423018420CBF00203A
:10440C0001207047C4030020034B93F8512040EA6D
:10441C00020283F851207047C4030020034B93F829
:10442C00512022EA000283F851207047C403002077
:10443C00034B93F8513018420CBF002001207047F9
:10444C00C4030020014B1868704700BF34090020DA
:10445C00014B1868704700BFF8080020014B5868E2
:10446C00704700BFF8080020014B1868704700BF68
:10447C004C090020014B5868704700BF4C090020C4
:10448C0008B50120FFF7D4FF48B1054B00220420EA
:10449C00DA60FFF7CDFF10B10120FFF7BFFF08BDB9
:1044AC009401002008B506F08BFF08BD08B506F096
:1044BC00EBFD08BD08B54FF4803005F03BF908BDA5
:1044CC0008B5044B93F860301BB94FF4003005F07D
:1044DC0031F908BDC403002008B5034B1B78012B30
:1044EC0001D104F025FB08BD4300002008B5034BA7
:1044FC001B78012B01D104F077FB08BD1C020020B6
:10450C0008B54FF480700BF013FA70B14FF4807053
:10451C000BF01CFA054B1B78012B03D0044B1B78BA
:10452C00012B02D1034B01221A7408BD400000205C
:10453C001B0200209401002008B50220FFF75AFF4F
:10454C0038B1044BB3F8400006F06CFF0220FFF7C3
:10455C0047FF08BDC403002010B50120FFF74AFF38
:10456C00D8B106F06DFF0D4991F82530CA6B5B0888
:10457C00B2FBF3F3B0FBF3F202FB1303084AA1F80E
:10458C004030147834B9074B40311868022240305F
:10459C0005F0C0FA0120FFF723FF10BDC403002073
:1045AC00220200200400002008B5044B19780129D0
:1045BC0003D1034B186809F02FFF08BD4000002001
:1045CC003C00002038B5164C0221206809F01EFF73
:1045DC00012819D10221206809F01EFF002003F0E8
:1045EC0085F9104C05460146607C06F015FD0E4B16
:1045FC00657493F8213082B2062B00D023B9094B95
:10460C0012B2D9685218DA60054C0121206809F001
:10461C00FDFE0128014602D1206809F0FDFE38BDDF
:10462C003400002094010020C403002008B5074B7F
:10463C001978012903D1064B186809F0EDFE054BDA
:10464C001B78012B01D1FFF7BDFF08BD1B02002019
:10465C003C0000201902002008B5074B19780129ED
:10466C0003D1064B186809F0D7FE054B1B78012BBC
:10467C0001D1FFF7A7FF08BD1A0200203C00002063
:10468C0038000020B0F5007F10B5044610D003DCD4
:10469C00B0F5807F37D121E0B0F5806F03D0B0F555
:1046AC00006F30D10DE005F03DF84FF4807019E04B
:1046BC0005F038F84FF4807005F03CF84FF480604A
:1046CC0014E005F02FF84FF4807005F033F84FF438
:1046DC00806005F02FF84FF400700BE005F022F825
:1046EC004FF4806005F026F84FF4007005F022F8C6
:1046FC004FF4006005F01EF84FF4804005F01AF8F6
:10470C00024BA3F86240024B1C6010BDC403002096
:10471C001C09002010B504464FF4803005F012F847
:10472C00012808D0044B4FF400601C60FFF7AAFF6F
:10473C00024B00221A6010BD2409002048090020F9
:10474C0038B505464FF4803004F0FCFF01281CD02E
:10475C000E4B4FF480601C680D4B9D60FFF792FF71
:10476C004FF4804004F0E6FFB4F5007F04D1094B10
:10477C001A68094B1A6008E0B4F5006F05D1074BB5
:10478C0018680BF027FD044B186038BD1C0900207D
:10479C009401002048090020E0080020180900209E
:1047AC0008B5034BDB68C018FFF7CAFF08BD00BF94
:1047BC009401002008B54FF48070FFF763FF08BD2B
:1047CC0038B52C4B93F82130082B52D8DFE803F086
:1047DC00055151515151052F4B00274A0128D368DF
:1047EC00254D08BF536101286A69244C6B6102D1C5
:1047FC00AB6923603DE01F499B1A886991F825C07D
:10480C001F494FF0140E0EFB00FE59434FEA5C0C8F
:10481C00062303FB0CFC91FBFEF1206891FBFCF1E1
:10482C00282207F0EBFD20602368AB6121E0012812
:10483C00114B124C02D1DB69236010E011490D4A77
:10484C000D680F48916905FB00FC14204843D16B9F
:10485C009CFBF0F292FBF1F222602268DA61094BC8
:10486C0000221A6005E0084B18680BF0CDFE034BD4
:10487C00186038BDC40300209401002018090020E2
:10488C00804F1200600900204809002010B5044632
:10489C004FF4804004F04EFF034B0120DC609C6021
:1048AC00FFF78EFF10BD00BF9401002008B5034830
:1048BC0004F0EAF8024804F0E7F808BDF808002014
:1048CC003409002008B50248202109F0B5FD08BDC7
:1048DC00002C014038B505464FF4803004F032FF0F
:1048EC0001281AD00D4B4FF400701C680C4B1D6046
:1048FC00FFF7C8FEB4F5006F05D10A4B18680BF032
:10490C0069FC094B1860094B9B6813F4005F04D1D8
:10491C0004F032FF08B902F01DFF38BD1C0900205D
:10492C0064090020180900204809002000100140EB
:10493C0010B502F0FFFE012003F0A2F9444804F088
:10494C00A3F8444C444804F09FF8444804F09CF805
:10495C0094F8210006F04EF994F82130062B0ED174
:10496C004FF4004004F0DEFE802004F0E3FE012052
:10497C0006F002FC94F82500400806F0C3FB354C09
:10498C0094F82130072B23D14FF4004004F0D2FED1
:10499C00802004F0CFFE94F82A30012B02D10020A5
:1049AC0006F0EAFB2B4CE06B94F82C1006F0BEFDE5
:1049BC0094F82510E06B490806F0CCFC06F0DAFC04
:1049CC00274B00221A7403F021FC012006F0D8FCBE
:1049DC00204C94F82130082B11D14FF4004004F0F6
:1049EC00A9FE002006F0C8FBE06B94F82C1006F032
:1049FC009DFD94F82510E06B490806F0ABFC154CB6
:104A0C0094F8213073B94FF4004004F08BFE8020F1
:104A1C0004F090FE012006F0AFFB94F8250040084E
:104A2C0006F070FB0B4B4FF4004293F850000D4B0B
:104A3C005A6100B1012003F029F90A4B4FF480525E
:104A4C001A6102F5E0425A6102F084FE10BD00BF0B
:104A5C00F8080020C40300204C090020E4080020C2
:104A6C00940100200010014038B5094C094D94F810
:104A7C00202095F821309A4208D0FFF759FF0120E9
:104A8C00FFF79EFE95F8213084F8203038BD00BF2A
:104A9C0094010020C40300200A4938B5CC680023D7
:104AAC008C600949094D0B60094900220A602A6093
:104ABC00084A094D01202B601360FFF781FEFFF7B8
:104ACC0037FF38BD940100206409002048090020FC
:104ADC00E00800200C0900202409002038B51A4BEE
:104AEC001B78012B02D106F071FC03E0174B186800
:104AFC0009F084FC164B0422D96B91FBF2F2904224
:104B0C000ADA4FF0030C0CFB02FC124B5B6A634598
:104B1C0002DDCB1A1B180DE003235343984206DD2C
:104B2C000C4B5B6A934202DAC31A5B1A02E0094B24
:104B3C005B6AC31A074A0849D4680D68E41AEB1A71
:104B4C000B605062D46038BD220200203C00002073
:104B5C00C403002094010020600900202DE9F045D9
:104B6C009F4B93B01B889F4C13F0100F40F0A28208
:104B7C00A36A18460133A36204F0D4FC216B9A4B50
:104B8C00E26A013193F821302163984901324FF4E4
:104B9C008040072B0861E26208D1954B1B78012BF2
:104BAC0001D106F029FC0120FFF798FF8E4B93F8FA
:104BBC002130082B05D18E4B1B78012B01D106F02F
:104BCC001BFC894D1422AB69864C5343226B9A42D1
:104BDC00C0F09B80002318462363FFF7F1FD636B45
:104BEC004FF480600133636304F0ACFD00282DD0DA
:104BFC00A168804BE268284603F0ECFE7E4B1860FF
:104C0C0004F0D4FC58B104F04DFD022807D1A26881
:104C1C00E3680E920F930EAB0FCB04F0E9FC714AD4
:104C2C00714B9068D168DA68411A0029B8BF4942C3
:104C3C0091420BDC714A9B681268002AB8BF524241
:104C4C009A4203DC4FF4804004F06CFD664C94F8FF
:104C5C002030012B25D14FF4806004F073FD68B136
:104C6C00604A6749D3689568634A20461268009584
:104C7C0003F032FA0BF0AEFA624B18604FF400708E
:104C8C0004F060FDC0B15F4C20680BF0BDFC5A4BCA
:104C9C0001461A68544803F0E9F90BF09BFA2060BE
:104CAC000AE0554B216818680A46494207F086FB12
:104CBC000BF090FA534B18604FF4007004F042FD67
:104CCC0020B900F5806004F03DFDF0B14D4D4B4C2A
:104CDC0028680BF099FC266801464B4B324642483B
:104CEC0003F028FE494B186004F060FC68B104F036
:104CFC00D9FC012809D128680BF086FC23680E909A
:104D0C000F930EAB0FCB04F073FC364E364BF16A9F
:104D1C00DA699142C0F0A281B76B1A8D0137B76383
:104D2C000027F7623E260AAC0096394D06F5D2767E
:104D3C00C8216423204601964FF40266029603F0C4
:104D4C003BF894E8070085E807004FF4806004F016
:104D5C00F9FC01280CD04FF4007004F0F3FC01288E
:104D6C0006D04FF4006004F0EDFC012840F0F48014
:104D7C001D4F97F82140002C54D0204B244AD3F8D7
:104D8C0000801D4B6D4607CAD3F800C085E80700AC
:104D9C0038461B4F134C1D4E05971A4F04F13C0E11
:104DAC00194B1C491C4ACDF810E0CDF81CC00697D5
:104DBC00CDF82080039603F06FFAB4F93C30B4F9C7
:104DCC003E10DFF85CA03468C918144BDAF8000008
:104DDC0010221C6007F012FBCAF80000ACE000BF08
:104DEC00002C014094010020C4030020001001405D
:104DFC002202002034090020640900201809002038
:104E0C00E008002048090020F808002024090020B0
:104E1C00280900204C090020E40800200C0900207F
:104E2C0020090020012192480AF0E8FE05F016FD49
:104E3C00012806D003D3022805D020460CE08D4D66
:104E4C0002E08D4D00E08D4D286802F0E9FE04462D
:104E5C00286802F0D5FE201A894B4FF4F174198D95
:104E6C0064223E2300944FF40264019402F0E0FEAD
:104E7C00844B854E93F840300446012B08BF4442C6
:104E8C0021461022306807F0B9FA804D07462A688F
:104E9C0023467F497A48376003F0BCFD7D4A794B45
:104EAC001268002858642A6002DD002283F8402032
:104EBC00744B5A6C002A02DA012283F8402001203C
:104ECC0002F014FD6E4B054693F8243013B980F0B4
:104EDC000705EDB26B4F70487E6C002EB8BF764262
:104EEC00B6B2314609F032FA6B48314609F030FA65
:104EFC003146694809F02EFA294697F840200120DE
:104F0C0005F050FE6448202108F0DCFF04F04EFB55
:104F1C0090B104F0C7FB03280ED105F09FFC64236D
:104F2C0043436FF0630278330E930F9411921092F7
:104F3C000EAB0FCB04F05CFB04F038FB60B104F05B
:104F4C00B1FB48B9514B1A684F4B0E921B680F932B
:104F5C000EAB0FCB04F04CFB4B4B1A68484B002AA2
:104F6C005B68B8BF52429A4205DD012004F0DAFBBF
:104F7C0002F02EFC04E0012004F0DCFB02F02EFC1D
:104F8C00414B3F49186805F06DFF4FF4003004F0B9
:104F9C00D9FB012808D1414803F076FD404803F0C5
:104FAC0073FD0020FFF7B6FB02F0DEFE3D4BDB7914
:104FBC000BB102F061FC324B93F8222012F0010F7E
:104FCC0022D0394A1268002A1EDD93F8233013F0E0
:104FDC00010F03D0002002F02DFC40B9284B93F8B0
:104FEC00230010F001000FD102F024FC60B9022064
:104FFC00FFF71EFA10B1234B0022DA600020FFF7F6
:10500C0069FC2A4B00221A601D4B93F8222012F0E7
:10501C00020F23D0244A1268002A1FDA93F8233097
:10502C0013F0020F03D0012002F004FC48B9144B1A
:10503C0093F8233013F0020F10D1012002F0FAFB89
:10504C0060B90220FFF7F4F910B10E4B0022DA60C0
:10505C000020FFF73FFC154B00221A60084B93F819
:10506C002130002B34D1124B4FF480425A612FE087
:10507C00002401401402002014000020180000201D
:10508C00C403002094010020200900200C090020FA
:10509C004C09002024090020002C0140F8080020B5
:1050AC0034090020B0040020180900204809002011
:1050BC0000100140A36C18460133A36404F038FAC5
:1050CC00074B4FF48042074801215A610AF096FDC4
:1050DC000548012109F0A0F913B0BDE8F08500BF27
:1050EC000010014000240140002C014008B502F0E2
:1050FC0041FBA0B904F040FB88B900F5005004F066
:10510C0021FB60B900F5807004F01CFB38B9044B2E
:10511C004FF461729A861A879A8702F01BFB08BDBE
:10512C00002C014010B505F085FA204CE36CC31A35
:10513C00002BB8BF5B42B3F57A7F36DD1C4B9B6806
:10514C0013F4806F2AD102F015FB60B1012004F03A
:10515C00E9FA402004F0E6FA94F850300A2B02D811
:10516C00013384F850304FF4807004F0EBFA20B91E
:10517C00FFF7B0FB0F4B00221A6002F0FBFA80B174
:10518C000A4B93F850300A2B0BD8094B4FF40062A2
:10519C001A6140205A6104F0CDFA02E0002384F831
:1051AC00503005F047FA014BD86410BD9401002033
:1051BC00001001404809002010B505F03BFA1A4CCC
:1051CC00636DC31A002BB8BF5B42642B2ADD174BEF
:1051DC00186802F015FD164B206093F82B30012B4C
:1051EC000AD103F55E63984206DD02F0BBFA042097
:1051FC0004F098FAFFF7DEFA0B4B1A6840F21633FC
:10520C009A4202DC022004F08DFA074B1A6840F235
:10521C0016339A4202DD022004F08CFA05F00AFAE9
:10522C00014B586510BD00BF9401002020000020E8
:10523C00C403002010B505F0FDF9264CA36DC31A6C
:10524C00002BB8BF5B42B3F57A7F42DD224B186866
:10525C0002F0D6FC6060082004F074FAB8B96368F8
:10526C0040F6B322934209DD083004F05BFA02F0F9
:10527C0095FA02F077FAFFF79DFA26E0B3F5156F71
:10528C000ADC082004F056FA02F08EFA09E0626893
:10529C0040F60B239A4218DC082004F04BFA02F07B
:1052AC0089FA0E4B9B6813F4005F0ED104F064FA7C
:1052BC0058B900F5005004F045FA30B900F580708B
:1052CC0004F040FA08B902F045FA05F0B3F9014BC5
:1052DC00986510BD940100202400002000100140AE
:1052EC0070B505F0A7F94F4C0646E36DC31A002BB9
:1052FC00B8BF5B42B3F57A7F0DDB206E04F0FAF891
:10530C000025A06B256604F0FBF8606BA56304F028
:10531C00FDF8E6656563444A424B1168434A186ED2
:10532C0012690029B8BF49420130002AB8BF524265
:10533C009142186603DC102004F0F4F902E010200E
:10534C0004F0F8F9374CFFF78FFBFFF735FFFFF749
:10535C0071FF237C63B1354B93F82130072B07D1B8
:10536C00FFF7FAF8FFF7E8F8FFF78AF80023237441
:10537C0005F0B2FD2D4D6B6D984225D905F05AF90B
:10538C00284C636EC31A002BB8BF5B42B3F57A7F0F
:10539C001ADB05F05FFD4FF4003004F0C3F995F80B
:1053AC0060305BB9224B29461868012201F8602F46
:1053BC00603004F0AFFB05F03DF9A06605F09EFDF2
:1053CC0005F038F9174B586605F034F9154B1749A9
:1053DC009A6E8B6D821A002AB8BF52429A420BD336
:1053EC0091F86020012A07D1114B1868002301F8AD
:1053FC00603F603004F08EFB0C4B93F86030012B57
:10540C0003D14FF4003004F08DF904F0D5F838B125
:10541C00084B1868044B1968024BDA6804F054F90D
:10542C0070BD00BF9401002018090020C4030020A7
:10543C00040000202009002008B5054A034602207C
:10544C0093FBF0F080B282F8253005F077FF08BDB1
:10545C00C403002010B5124B5B781BB1012B114B10
:10546C001AD111E0104A01209178104A1468104AA0
:10547C001070104A11700133E21812F8011C0D4A19
:10548C00082B9954F7D109E00921022219715231E4
:10549C0099715A71DA7101E003221A7010BD00BFC4
:1054AC004C030020A0040020B004002028000020A1
:1054BC00B4030020B8030020044B5A6840F2D243D6
:1054CC009A4202D1024B01221A7070474C03002001
:1054DC006809002010B51C4A1C4B116801EA030333
:1054EC001B498B422ED152681A4B9A422AD102F098
:1054FC0039F9194B1B78012B10D103F035FF05F04E
:10550C0099F8044601E002F083F905F093F8001BCA
:10551C000028B8BF4042B0F57A7FF4DB04F038F9CC
:10552C0009F08EFC002009F013F900210B480AF059
:10553C00B3FA0A480AF010FA09480AF09FFC002056
:10554C0004F030F910BD00BF4C03002000FFFF0039
:10555C0000819200D6C5B4A345000020080002408B
:10556C000024014010B5164B9A78012A08D003D3B9
:10557C00022A144C0FD109E0587802F05BF902E0D2
:10558C00587802F091F90F4B586006E0587802F009
:10559C0063F9606001E0042323700B4B1B786BB143
:1055AC00084B0A495A680A4B0A601AB91A6842F041
:1055BC00080202E01A6822F008021A6010BD00BF4F
:1055CC004C030020A004002084040020B003002021
:1055DC005403002008B5104B9A78012A02D0022AF5
:1055EC0016D10CE05A7842B9586810B904F0D2F8C8
:1055FC0011E0104604F0D2F80DE0032209E05A68DD
:10560C00587812B902F006F905E002F00BF902E045
:10561C000422024B1A7008BD4C030020A004002089
:10562C0008B50B4B9A78022A0ED15B78372B09D828
:10563C009B00084903F5E260C9180A30023204F0F5
:10564C00E7F804E0032200E00422034B1A7008BDC3
:10565C004C030020DC040020A0040020144A00238A
:10566C001360144A10B51360134A1360134A136085
:10567C00134A1370134A002199500433B3F5806F09
:10568C00F8D1114B1B7E63B940F21A740F492046B6
:10569C000919042204F0BCF8043440F2FA739C4259
:1056AC00F4D1094A0A4B527D02B101221A7010BD85
:1056BC004C040020B0030020D80400205403002028
:1056CC0048030020DC040020B0040020C2FDFF1FB2
:1056DC008C04002008B5124B9A7812B1022A1AD108
:1056EC000AE05B784E2B14D10E4B18680E4B07302A
:1056FC00D97904F0B1FA11E05B78372B09D89B000B
:10570C000A4903F5E260C9180A30042204F002FACF
:10571C0004E0032200E00422054B1A7008BD00BF10
:10572C004C03002090010020B0040020DC04002079
:10573C00A004002008B5604B9A781AB1022A40F0F8
:10574C00A68099E05B78502B69D01FD8462B51D09E
:10575C000ED8422B43D005D8402B37D0412B40F0EC
:10576C0089803AE0442B40D0544B554A40D83AE01B
:10577C004B2B48D004D8472B3FD0492B7AD13FE054
:10578C004D2B46D042D34E2B74D145E0812B5AD0B1
:10579C000ED8532B4CD004D8512B43D0522B69D15B
:1057AC0043E05A2B4AD0802B4BD0552B62D142E090
:1057BC00842B53D004D8822B4CD0832B5AD14BE062
:1057CC00FE2B4ED050D8F02B54D14AE03D4B1868EC
:1057DC0004F06CF8394B58605CE0394B42E0384BC4
:1057EC005A78364B4FE012794DE0354BDA69F8E7D1
:1057FC00527948E0324BDA68F3E7314B9A68F0E7BC
:10580C002F4BDA7D32E02E4BDA78EAE72C4B9A7884
:10581C00E7E72B4B5A7DE4E7294BDA79E1E7284B94
:10582C009A7DDEE7264B1A7DDBE7254B1A6AD8E713
:10583C00234B1A69D5E7224B1A7ED2E7204B5A6AC2
:10584C00CFE7214B0EE0204B1A78042A14BF00221C
:10585C000122C6E71D4B02E01D4B00E01D4B1A68F0
:10586C00BFE71D4B1A78BCE71C4B1A78003A18BFDF
:10587C000122B6E703220BE05A78104B372A04D8E2
:10588C00174951F822205A6004E0032201E0042257
:10589C000A4B1A70134B1B786BB1084B12495A68A0
:1058AC00124B0A601AB91A6842F0080202E01A6830
:1058BC0022F008021A6008BD4C030020A00400204E
:1058CC00B00400200C0000208C0400204C040020AC
:1058DC00700900206C090020980400207C04002032
:1058EC00DC04002084040020B003002054030020BA
:1058FC0010B58A4B9A781AB1022A40F0238104E140
:10590C005A784C2A00F09E801ED8442A60D00CD8BD
:10591C00412A44D003D8402A40F012813BE0422A6D
:10592C0046D0432A40F00C814AE0472A68D005D87B
:10593C00452A55D0462A40F0038159E0492A67D0C0
:10594C004B2A40F0FD8070E0532A00F0B38010D851
:10595C00502A00F08B8005D84D2A7BD04E2A40F07F
:10596C00EF807FE0512A00F08980522A40F0E880D5
:10597C0098E0832A00F0BD8006D8552A00F0A2805A
:10598C005A2A40F0DD80A9E0842A00F0B680FF2A74
:10599C0040F0D680B6E01979614B186805E0614A91
:1059AC001B791068604A1946137004F055F9CCE065
:1059BC005C4A1B7910685C4A013019465370F4E755
:1059CC00584A1B791068584A043019461371ECE791
:1059DC00544A5B68106854491C3041F81C3F84E001
:1059EC00504A1B791068504A053019465371DCE750
:1059FC004C4A5B6810684C490C3041F80C3F74E021
:105A0C00484A5B6810684849083041F8083F6CE028
:105A1C001A79454B12B1454901224A60DA75414B5E
:105A2C001868414B1730D97DBFE73E4A1B79106887
:105A3C003D4C03301946E37004F00EF9E07803F0A6
:105A4C003FF882E0374A1B791068374A0230194612
:105A5C009370AAE7334A1B791068334A15301946FC
:105A6C005375A2E71A79304BDA716EE02D4A1B7927
:105A7C0010682D4A16301946937596E72A4A127DFE
:105A8C0012F0010F05D01B7913F0010F01D103F0B7
:105A9C009FFF244A214B10681B79234A1430194666
:105AAC00137582E71F4A5B6810681F49203041F864
:105ABC00203F1AE01B4A5B6810681B49103041F804
:105ACC00103F12E05A68012A3CD8164A1B7910681C
:105ADC001549183001F8183F012207E0114A5B689C
:105AEC0010681149243041F8243F042204F012F8C4
:105AFC002BE00E4B5A680E4B02E00C4B5A680D4BC8
:105B0C001A6022E01A790C4B1EE05A78372A17D803
:105B1C0059680A4B43F8221017E000BF4C030020D1
:105B2C000C00002090010020B0040020A0040020F4
:105B3C00700900206C0900207C040020DC0400208B
:105B4C00032200E00422014B1A7010BDA0040020B7
:105B5C0008B5034B987808B9FEF7BCFE08BD00BF2A
:105B6C004C03002008B5034B9A7812B95868FEF71D
:105B7C00B1FE08BD4C03002008B5044B9A781AB945
:105B8C0058684042FEF7A6FE08BD00BF4C0300203B
:105B9C0008B5A94B9A78002A41F0D5805A78AD2ADD
:105BAC0000F022856FD81E2A00F0B78230D8092A5F
:105BBC0000F0A78113D8032A00F0138105D8012A1D
:105BCC0000F0E48000F2F080D2E0062A00F0408180
:105BDC00072A00F06A81042A41F0B38007E1192AF0
:105BEC0000F0188208D80B2A00F0E281C0F0B481D2
:105BFC000D2A41F0A68007E21B2A00F05282C0F069
:105C0C002C821C2A00F053821D2A41F09A807DE2DE
:105C1C009C2A00F04D831CD8922A00F0EE8209D801
:105C2C00852A00F09482862A00F0BC821F2A41F05B
:105C3C00888085E2972A00F0158303D8962A41F0D4
:105C4C00808009E3982A00F013839B2A41F0798025
:105C5C0014E3A32A00F0E08308D8A12A00F06083A3
:105C6C0000F293839F2A41F06C8027E3A52A00F071
:105C7C003584C0F00584A62A00F06284AC2A41F079
:105C8C00608000F089BCD42A00F0E48531D8C32AA6
:105C9C0000F07E8515D8BF2A00F042850AD8B22ABA
:105CAC0000F00785BE2A00F02D85B12A41F049800D
:105CBC0000F0C1BCC12A00F04F8500F25B8500F0FA
:105CCC003DBDC72A00F09C8506D8C52A00F07C850E
:105CDC0000F2888500F06ABDC92A00F0A685C0F0E4
:105CEC009D85D22A00F0A885D32A41F02A8000F0A5
:105CFC00AABDF42A00F0A3861FD8E52A00F0E3859C
:105D0C000AD8E22A00F0D185E42A00F0D585E12AF0
:105D1C0041F0178000F0A6BDEA2A00F0148604D8E2
:105D2C00E62A41F00E8000F0D5BDEB2A00F0338658
:105D3C00F12A41F0068000F056BEFB2A00F03D87A8
:105D4C0009D8F92A00F0CA8600F2F286F52A40F04A
:105D5C00F88700F09DBEFD2A00F08487C0F05887BC
:105D6C00FE2A00F0A887FF2A40F0EB8700F0C8BF9E
:105D7C00052805D1304B5868FEF7E2FC00F0FABF5D
:105D8C00062840F0F787FEF705FB26E0052805D12D
:105D9C00294B5868FEF77AFD00F0ECBF062840F05E
:105DAC00E987FEF705FB18E0052811D1224B234AA1
:105DBC00586800F5423303F5A863934203D8FEF705
:105DCC0089FD00F0D7BF1E4B04221A7000F0D2BF21
:105DDC00062840F0CF87FEF7F1FA194B586000F017
:105DEC00B7BF062840F0C687FEF7EEFAF5E70528A0
:105DFC000AD1114B13495B688B4295BF124A104B69
:105E0C0013601A7000F0B6BF062802D10E4B1A6848
:105E1C006BE2072806D10D4B0B49186803F07AFE8C
:105E2C0000F0A8BF082840F0A587084B0649186861
:105E3C0003F0EEFC00F09EBF4C030020801A06001D
:105E4C00A0040020400D0300C40300200400002027
:105E5C0005280ED19A4B44F670125B68934203D816
:105E6C00984A536000F086BF974B04221A7000F0DA
:105E7C0081BF062802D1934B5A6836E2072808D115
:105E8C00924B042218689249801803F043FE00F0EC
:105E9C0071BF082840F06E878C4B042218688C491F
:105EAC00801803F0B5FC00F065BF05280DD1844BBC
:105EBC00884A5B68934203D8824A936000F05ABFC9
:105ECC00814B04221A7000F055BF062802D17D4B7D
:105EDC009A680AE2072808D17C4B7F49186804228B
:105EEC00083003F017FE00F045BF082840F0428749
:105EFC00764B794918680422083003F089FC00F0CD
:105F0C0039BF05280CD15B68724A934203D86D4A9D
:105F1C00136100F02FBF6C4B04221A7000F02ABFE3
:105F2C00062802D1674B1A69DFE1072808D1674BB5
:105F3C006A4918680422103003F0ECFD00F01ABF17
:105F4C00082840F01787614B644918680422103008
:105F5C0003F05EFC00F00EBF05280DD1584B604AD3
:105F6C005B68934203D8574AD36000F003BF564B8B
:105F7C0004221A7000F0FEBE062802D1514BDA68DA
:105F8C00B3E1072808D1514B5649186804220C304C
:105F9C0003F0C0FD00F0EEBE082840F0EB864B4B42
:105FAC005049186804220C3003F032FC00F0E2BEB9
:105FBC0005280DD1424B4A4A5B68934203D8414AAB
:105FCC00536100F0D7BE404B04221A7000F0D2BED1
:105FDC00062802D13B4B5A6987E1072808D13B4B75
:105FEC00414918680422143003F094FD00F0C2BE3D
:105FFC00082840F0BF86354B3B4918680422143002
:10600C0003F006FC00F0B6BE062840F0B386FEF79F
:10601C00C7F9E2E6052804D15A682A4B9A6500F0C4
:10602C00A9BE062802D1274B9A6D5EE1072808D13C
:10603C00264B2E4918680422583003F06BFD00F0F3
:10604C0099BE082840F09686204B284918680422EF
:10605C00583003F0DDFB00F08DBE052805D1184B40
:10606C005A68184B5A6500F085BE062802D1154BAC
:10607C005A6D3AE1072808D1144B1D4918680422BF
:10608C00543003F047FD00F075BE082840F07286CE
:10609C000E4B174918680422543003F0B9FB00F07A
:1060AC0069BE062840F0668604F016FF95E60528C2
:1060BC0020D1034B586804F01BFF00F05BBE00BFFF
:1060CC004C030020C4030020A00400200400002086
:1060DC00C8030020400D0300CC030020D403002093
:1060EC00A0860100D0030020D80300201C0400204F
:1060FC0018040020062802D104F0F4FE6DE60728EF
:10610C0040F0388604F0FAFE00F034BE052840F06A
:10611C001D86FEF7D5F900F02DBE052804D1586870
:10612C0004F016FF00F026BE062802D104F00AFF88
:10613C0053E6072840F01E8604F010FF00F01ABE4C
:10614C00052840F00386FEF7A7FC00F013BE0528D7
:10615C000CD1A24B5B680A2B03D8A14A936100F0C7
:10616C0009BEA04B04221A7000F004BE062802D10E
:10617C009B4B9A69B9E0072808D19B4B9B4918683F
:10618C000422183003F0C6FC00F0F4BD082840F0DF
:10619C00F185954B954918680422183003F038FBAB
:1061AC0000F0E8BD05280CD18C4B5B680A2B03D89A
:1061BC008B4AD36100F0DEBD8A4B04221A7000F0CA
:1061CC00D9BD062802D1864BDA698EE0072808D1A2
:1061DC00854B8749186804221C3003F09BFC00F0A7
:1061EC00C9BD082840F0C6857F4B81491868042238
:1061FC001C3003F00DFB00F0BDBD05280ED15B6813
:10620C00012B06D8754B1A79754B83F8202000F0BA
:10621C00B1BD744B04221A7000F0ACBD062804D139
:10622C006F4B93F8202000F0D9BC072808D16E4B97
:10623C00704918680122203003F06CFC00F09ABD04
:10624C00082840F09785684B6A491868012220306D
:10625C0003F0DEFA00F08EBD062840F08B85FEF7C9
:10626C00B9F8BAE5062840F08585FEF781F8B4E563
:10627C00062840F07F85FEF781F8AEE5052811D1A0
:10628C00564B49F2E022586800F592437033934222
:10629C0003D8FEF73FFA00F06DBD524B04221A7082
:1062AC0000F068BD062840F06585FEF76DF894E5B2
:1062BC00062840F05F8503F055FA8EE505280FD1CE
:1062CC00464B5B689A1F022A00D923B9444A82F8CC
:1062DC00213000F04FBD434B04221A7000F04ABD30
:1062EC00062806D13E4B93F821203E4B5A6000F015
:1062FC002FBD072808D13C4B3F491868012221309B
:10630C0003F008FC00F036BD082840F03385364B0E
:10631C00394918680122213003F07AFA00F02ABDBD
:10632C00052813D12D4A2E4B52683AB193F85120BF
:10633C0042F0010283F8512000F01CBD93F851206B
:10634C0022F0010283F8512000F014BD062805D17B
:10635C00234B93F8512002F00102C6E7072808D11D
:10636C00214B264918680122513003F0D3FB00F071
:10637C0001BD082840F0FE841B4B204918680122FF
:10638C00513003F045FA00F0F5BC052813D1134A3F
:10639C00134B52683AB193F8512042F0020283F841
:1063AC00512000F0E7BC93F8512022F0020283F850
:1063BC00512000F0DFBC062805D1094B93F8512081
:1063CC00C2F3400291E707281AD1074B0B49186812
:1063DC000122513003F09EFB00F0CCBC4C0300209A
:1063EC00C4030020A004002004000020DC030020D3
:1063FC00E0030020E4030020E50300201504002046
:10640C00082840F0B784964B964918680122513001
:10641C0003F0FEF900F0AEBC052812D15A68924B7D
:10642C003AB193F8512042F0040283F8512000F065
:10643C00A1BC93F8512022F0040283F8512000F003
:10644C0099BC062805D1884B93F85120C2F38002E1
:10645C004BE7072808D1824B82491868012251303A
:10646C0003F058FB00F086BC082840F083847C4B7A
:10647C007C4918680122513003F0CAF900F07ABC4B
:10648C0005280ED1794B5A68032A05D81A79764B10
:10649C0083F8222000F06EBC754B04221A7000F0B9
:1064AC0069BC062803D1704B93F822201DE70728FE
:1064BC0008D16B4B6F4918680122223003F02AFB7C
:1064CC0000F058BC082840F05584654B69491868A1
:1064DC000122223003F09CF900F04CBC052812D1AB
:1064EC00624B5B68B3F5803F08D25F4A9BB218469B
:1064FC00A2F8403004F07AFF00F03CBC5C4B042264
:10650C001A7000F037BC062803D1574BB3F8402063
:10651C00EBE6072808D1524B574918680222403045
:10652C0003F0F8FA00F026BC082840F023844C4B0A
:10653C00514918680222403003F06AF900F01ABC85
:10654C0005280ED1494B5A68032A05D81A79464BAF
:10655C0083F8232000F00EBC454B04221A7000F087
:10656C0009BC062803D1404B93F82320BDE607282D
:10657C0007D13B4B414918680122233003F0CAFA7A
:10658C00F8E3082840F0F683354B3C4918680122A3
:10659C00233003F03DF9EDE305280BD1334B5B6859
:1065AC00B3F5803F02D2304A1363E3E3304B04224D
:1065BC001A70DFE3062802D12B4B1A6B95E60728DD
:1065CC0007D1274B2E4918680422303003F0A2FA69
:1065DC00D0E3082840F0CE83214B294918680422C7
:1065EC00303003F015F9C5E305280AD15B68B3F523
:1065FC00803F02D21C4A5363BCE31D4B04221A7029
:10660C00B8E3062802D1184B5A6B6EE6072807D15F
:10661C00134B1C4918680422343003F07BFAA9E3AD
:10662C00082840F0A7830E4B164918680422343012
:10663C0003F0EEF89EE305280CD10C4B44F67012D7
:10664C005B68934202D8084A936393E3084B042295
:10665C001A708FE3062817D1034B9A6B45E600BFDF
:10666C000400002015040020C40300204C0300206B
:10667C00A0040020E603002004040020E70300200F
:10668C00F4030020F8030020072807D1A04BA149F0
:10669C0018680422383003F03DFA6BE3082840F008
:1066AC0069839B4B9B4918680422383003F0B0F87F
:1066BC0060E305280BD1984B5B68012B03D8974AF4
:1066CC0082F8613056E3964B04221A7052E3062886
:1066DC0003D1924B93F8612007E6072807D18C4B26
:1066EC00904918680122613003F014FA42E308283B
:1066FC0040F04083864B8B4918680122613003F0CF
:10670C0087F837E3052804D1854B586802F0F2FE70
:10671C0030E3062840F02E8302F0B0FEFFF75DBB9D
:10672C00052804D17E4B586802F0EAFE22E30628C5
:10673C0040F0208302F0A8FEFFF74FBB052804D1E0
:10674C00774B586802F0E2FE14E3062840F01283FF
:10675C0002F0A0FEFFF741BB052804D1704B58682E
:10676C0002F0DAFE06E3062840F0048302F098FEFD
:10677C00FFF733BB052804D1694B586802F0D2FEF1
:10678C00F8E2062840F0F68202F090FEFFF725BBF7
:10679C00052804D1624B586802F0CAFEEAE20628CA
:1067AC0040F0E88202F088FEFFF717BB052804D101
:1067BC005B4B586802F0C2FEDCE2062840F0DA823D
:1067CC0002F080FEFFF709BB052804D1544B586832
:1067DC0002F0BAFECEE2062840F0CC8202F078FE3F
:1067EC00FFF7FBBA052804D14D4B586802F0B2FEF6
:1067FC00C0E2062840F0BE8202F070FEFFF7EDBA50
:10680C00052804D1464B586802F0AAFEB2E20628CD
:10681C0040F0B08202F068FEFFF7DFBA062840F0C5
:10682C00A982FDF721FEFFF7D8BA062840F0A28214
:10683C00FDF720FEFFF7D1BA062840F09B82FDF74A
:10684C0035FEFFF7CABA062840F09482FDF72AFEFF
:10685C00FFF7C3BA062840F08D8201F0DFFC00B2CE
:10686C00FFF7BBBA052805D12B4B5A682B4B83F885
:10687C0050207FE2062803D1284B93F8502034E5B2
:10688C00072807D1224B284918680122503003F001
:10689C0041F96FE2082840F06D821D4B22491868BF
:1068AC000122503002F0B4FF64E2062840F062820C
:1068BC00FDF7C8FDFFF791BA062840F05B82FDF7A3
:1068CC00C7FDFFF78ABA062840F05482FDF7C6FDD3
:1068DC00FFF783BA05280BD10F4B5B68B3F5803FEC
:1068EC0002D20E4A536445E20D4B04221A7041E267
:1068FC00062802D1094B5A6CF7E4072818D1044B2F
:10690C000A4918680422443003F004F932E200BF4B
:10691C0004000020FC0300204C030020C4030020D2
:10692C00A0040020250400201404002008040020EA
:10693C00082840F01F828E4B8E4918680422443080
:10694C0002F066FF16E205280BD18B4B5B68B3F5A2
:10695C00803F02D2894A93640CE2894B04221A705C
:10696C0008E2062802D1854B9A6CBEE4072807D1B1
:10697C007F4B844918680422483003F0CBF8F9E1C6
:10698C00082840F0F7817A4B7E4918680422483079
:10699C0002F03EFFEEE105280BD1774B5B68B3F5B7
:1069AC00803F02D2754AD364E4E1754B04221A701D
:1069BC00E0E1062802D1714BDA6C96E4072807D186
:1069CC006B4B7149186804224C3003F0A3F8D1E1E9
:1069DC00082840F0CF81664B6B49186804224C3074
:1069EC0002F016FFC6E105280FD1634B67495A68C0
:1069FC0002F5423303F5A8638B4202D85F4BDA658C
:106A0C00B8E15F4B04221A70B4E1062802D15B4B4B
:106A1C00DA6D6AE4072807D1554B5D4918680422E2
:106A2C005C3003F077F8A5E1082840F0A381504BC7
:106A3C005749186804225C3002F0EAFE9AE10528F6
:106A4C000BD15B6842F21072934202D84B4AD3844A
:106A5C0090E14B4B04221A708CE1062803D1474B72
:106A6C00B3F9262041E4072807D1414B494918685E
:106A7C000222263003F04EF87CE1082840F07A819F
:106A8C003B4B444918680222263002F0C1FE71E1EA
:106A9C00052808D1384B5A68384B003A18BF0122E8
:106AAC0083F82B2066E1062803D1344B93F82B2076
:106ABC0094E0072807D12E4B3749186801222B3058
:106ACC0003F028F856E1082840F05481284B32494D
:106ADC00186801222B3002F09BFE4BE105280BD1EC
:106AEC00254B5B68022B03D8244A82F82A3041E1FB
:106AFC00234B04221A703DE1062804D11F4B93F856
:106B0C002A20FFF7F2BB072807D1194B2349186835
:106B1C0001222A3002F0FEFF2CE1082840F02A81E5
:106B2C00134B1E49186801222A3002F071FE21E134
:106B3C0005280DD1104B5B68B3F5803F04D20F4A8A
:106B4C00D363FDF7A9FF15E10D4B04221A7011E177
:106B5C00062803D1094BDA6BFFF7C7BB072821D1F5
:106B6C00034B0F49186804223C3002F0D3FF01E1BB
:106B7C0004000020080400204C030020C403002063
:106B8C00A00400200C04002010040020801A060031
:106B9C0020040020EA030020EF030020EE03002075
:106BAC0000040020082840F0E580734B73491868F6
:106BBC0004223C3002F02CFEDCE0052809D15A6896
:106BCC006F4B003A18BF012283F82C20FDF764FFAD
:106BDC00D0E0062807D16A4B93F82C20003A18BF56
:106BEC000122FFF782BB072807D1634B6549186860
:106BFC0001222C3002F08EFFBCE0082840F0BA8055
:106C0C005D4B6049186801222C3002F001FEB1E0A6
:106C1C0005280BD15C4B5B68012B03D8584A82F8D2
:106C2C002D30A7E0594B04221A70A3E0062804D19A
:106C3C00534B93F82D20FFF758BB072807D14E4B29
:106C4C005349186801222D3002F064FF92E00828A5
:106C5C0040F09080484B4E49186801222D3002F0CC
:106C6C00D7FD87E005280BD1474B5868831EFC2BBA
:106C7C0002D8FEF7E1FB7DE0444B04221A7079E068
:106C8C00062804D13E4B93F82520FFF72EBB07288E
:106C9C0007D1394B3F4918680122253002F03AFFE1
:106CAC0068E0082866D1344B3A491868012225302F
:106CBC0002F0AEFD5EE0052808D1334B5A68304B2C
:106CCC00003A18BF012283F8242053E0062803D190
:106CDC002B4B93F8242081E7072807D1264B2E490C
:106CEC0018680122243002F015FF43E0082841D136
:106CFC00214B294918680122243002F089FD39E022
:106D0C00052804D1204A1E4B92881A8532E00628A9
:106D1C0003D11B4B1A8DFFF7E8BA072807D1164B86
:106D2C001E4918680222283002F0F4FE22E00828DE
:106D3C0020D1114B194918680222283002F068FD45
:106D4C0018E0032200E00422104B1A70062811D11F
:106D5C00134B1B7873B10D4B12495A68124B0A60D6
:106D6C0022B91A6842F008021A6003E01A6822F08D
:106D7C0008021A6008BD00BF0400002000040020B7
:106D8C00C4030020F00300204C030020A0040020CA
:106D9C00F1030020E9030020E8030020EC030020AD
:106DAC0084040020B00300205403002010B5274BAE
:106DBC00997821B15B78032B01D0042B41D1234B63
:106DCC005B780A2B3BD8DFE803F006090C0F141A8A
:106DDC001D282D30350002F03DFC2DE002F036FC74
:106DEC002AE002F03BFC27E0184B586802F038FC14
:106DFC0022E0164B0846596802F0B8FB24E002F07A
:106E0C00CDFB21E002F0D2FB044602F0D5FB104B87
:106E1C0040EA0404E4B25C6016E00C4B586802F0E3
:106E2C002FFC11E002F03EFC06E0084B586802F023
:106E3C003FFC09E002F042FC054B586004E00322E1
:106E4C0000E00422024B1A7010BD00BF4C0300205E
:106E5C00A004002008B50B4B9A7872B95A7812B17D
:106E6C00012A08D103E05868FDF76AFC08E058686D
:106E7C00FDF796FC04E0032200E00422024B1A709A
:106E8C0008BD00BF4C030020A004002010B5A94A87
:106E9C00A94B107851686422232859601A705870D5
:106EAC0000F0F68053D8132800F0CB8028D808289F
:106EBC0011D8052880F0B080022800F0A48003D8F7
:106ECC00012840F049819BE0032800F09F800428B2
:106EDC0040F042819DE00B2800F0A78006D80928DD
:106EEC0000F09D800A2840F037819BE00E2800F0CE
:106EFC00A2800F2800F0A2800C2840F02D8197E092
:106F0C001B2800F0B08011D8162800F0A38006D8FA
:106F1C00142800F09980152840F01E8197E017285E
:106F2C0000F09B80182840F0178199E01F2800F092
:106F3C00A38006D81C2800F099801E2840F00C81F4
:106F4C0097E0212800F09E8000F29F8097E0822835
:106F5C0000F0C58029D8432800F0AC8011D8402817
:106F6C0000F09F8006D8242800F09580272840F058
:106F7C00F38093E0412800F09780422840F0EC80A9
:106F8C0095E0462800F09F8006D8442800F09580B4
:106F9C00452840F0E18093E0802800F09A8000F2D0
:106FAC009B80472840F0D88090E0882800F0B6807D
:106FBC0011D8852800F0A48006D8832800F0928090
:106FCC00842840F0C98090E0862800F0A1808728B2
:106FDC0040F0C280A5E08D2800F0B28006D8892848
:106FEC0000F0A2808C2840F0B780A0E0F22800F0DE
:106FFC00AD80FF2800F0AD808E2840F0AD80A2E07F
:10700C00FEF7B0FDABE0FEF7B7FDA8E0FEF7A0FD84
:10701C00A5E0FFF71FFFA2E0FEF7BAFD9FE0FEF729
:10702C0067FC9CE0FEF786FB99E0FEF753FB96E0CD
:10703C00FEF7F6FA93E0FEF7CDFA90E0FEF792FA3F
:10704C008DE002F06DFF8AE003F048F887E003F072
:10705C00D3F884E003F0C6F881E003F027F97EE072
:10706C0003F03CF97BE003F0B3F978E003F048F966
:10707C0075E003F04BF972E003F060F96FE003F098
:10708C008DF96CE002F0A0FF69E003F0C5FA66E050
:10709C0003F0B6FA63E002F0F5FF60E002F09AFE4E
:1070AC005DE000F0BDFA5AE000F0BCFA57E000F0E9
:1070BC00BBFA54E000F0BAFA51E000F0B9FA4EE035
:1070CC0000F0B8FA4BE000F0B7FA48E000F0B6FA7E
:1070DC0045E002F0CFFE42E002F096FE3FE002F007
:1070EC00A5FE3CE002F0A8FE39E000F03BFB134BA0
:1070FC001C7D02F037FB0146204603F01BF82EE006
:10710C0003F034F800F026FB0020FDF703FB26E02B
:10711C000A4B197D987803F011FA20E0FEF79AF9E2
:10712C001DE003F029F81AE003F04EFA17E003F023
:10713C00D9F914E04C030020A0040020B004002076
:10714C0002F09EFE0BE0FFF731FE08E0FEF7C2F9FD
:10715C0005E0FEF7B1F902E0014B02221A7010BDF6
:10716C00A0040020F0B5944B87B01B78044663B1A3
:10717C00924B1B78062B08D00A2B06D00F2B04D071
:10718C001F2B02D08E4B00221A708E4B1B78012BBA
:10719C004CD18B4A1278032A20D18B4B1B7893B994
:1071AC008A4E8B4DB07877782A786B78C719BF18D0
:1071BC00EA79FF18AB79BF186A79FF182B79BF18D9
:1071CC00FF18FFB218E0012B30D10025814BE85C91
:1071DC00013501F085FC092DF8D127E0042A25D1D1
:1071EC007A4E7B4DB27877781046D719013700224A
:1071FC002B706A60FFB26A7001F072FC707801F05B
:10720C006FFC287801F06CFC687801F069FCE87977
:10721C0001F066FCA87901F063FC687901F060FC70
:10722C00287901F05DFC384601F05AFC6A4B1B785A
:10723C00012B5FD1624A1278072A35D1624B1B7839
:10724C002BBB624A624B5578967893F800E093F822
:10725C0001C0AF19D8797744997967445A79C7191D
:10726C001B79CF19D719DF198DF808708DF80060CC
:10727C008DF801508DF802E08DF803C08DF80400F4
:10728C008DF805108DF806208DF8073009E0012BDC
:10729C0007D1013B4F4A995C0DF803100133092BC0
:1072AC00F8D16846092123E0082A23D14749484AE6
:1072BC0091F801C091F802E000250EEB0C060136A6
:1072CC006846092155608DF802308DF803502F4621
:1072DC008DF804508DF805508DF806508DF8075038
:1072EC008DF80860557013708DF800E08DF801C0B2
:1072FC0001F024FF394B34491A7800230B703049C4
:10730C000B7012B1012002F04DFA2E4B1B78012BA1
:10731C0075D10DF1170001F0BDFB00286FD001F005
:10732C00D5FB10B1264B00225A70254A9DF8170048
:10733C0051784B1CDBB28918092B0871537060D142
:10734C00224B1079597800238842537059D11A4630
:10735C001B4D291DC95C01335218082BD2B2F7D131
:10736C002B7B934248D1154B697AAA7AEE7A6F79C6
:10737C0095F806E095F807C0287A1E7199715A7134
:10738C001F7083F801E083F802C0D87103F052F942
:10739C00134B144E1B783060591E13480022C9B28F
:1073AC006A700270033201292A7021D9052B1FD073
:1073BC000E4B01251D7025E07C0400204C030020A1
:1073CC000402002042000020B4030020B00400207E
:1073DC00A0040020B803002045000020680900200C
:1073EC008C0400209C040020A804002084040020AD
:1073FC00594B00221A7004E004232B7001E0002585
:10740C0000E00125554B1B78012B43D103A801F05B
:10741C007DFE00283ED000231A4603A9C95C013327
:10742C005218082BD2B2F8D19DF814104C4C914242
:10743C002ED14C4B9DF811109DF812209DF80D602B
:10744C009DF80EE09DF80FC09DF810009DF81350AC
:10745C0099715A711E701D7183F801E083F802C096
:10746C00D87103F0E7F8404B40491B7808605A1E6E
:10747C003F490020D2B208700721012A217003D99C
:10748C00052B01D0012200E00022334B1A701CE0C6
:10749C0023701AE0CDB934490B78013BDBB2012BD8
:1074AC0013D8012C11D1334B1A68B2F5006F0BD8DD
:1074BC00104601321A602B4902F0D6FA284B0922E9
:1074CC001A70254B1C7000E00D70274B1B78042B99
:1074DC0004D1244B93F90030002B2EDA204B1B786F
:1074EC003BB1042B05D0082B03D0062B01D0FFF7A2
:1074FC00CDFC1B4B1B78092B05D11B4A117802299B
:10750C0001D1033111701C4A12681AB3092B21D115
:10751C00154B1B78012B1DD11649013B096809E05D
:10752C00164850F823000133814203D10E4B05223B
:10753C001A700FE09342F3D30CE0FDF73BF9084BC4
:10754C001B783BB1042B05D0082B03D0062B01D0A4
:10755C0002F09EFF07B0F0BD84040020450000201F
:10756C00040200204C0300208C0400209C0400200A
:10757C00A80400204C04002090040020500400209B
:10758C0073B5204B024640781F4D1870907800263A
:10759C005870D078EC46987010790C46D8715079A8
:1075AC00987192F806E095E8030083F805E0D2792B
:1075BC008CE803001A71154B1E70FFF767FC144B17
:1075CC001B7873B9637023702B78A3706B78E3709E
:1075DC00EB792371AB7963716B79A3712B79E371BF
:1075EC0008E0012B06D10B4B9B195B78A355013698
:1075FC00082EF8D1044B6A4692E8030083E8030096
:10760C007CBD00BF4C030020A0040020840400209B
:10761C00B4030020B8030020704700BF704700BFC0
:10762C00704700BF704700BF704700BF704700BF76
:10763C00704700BF704700BF704700BF704700BF66
:10764C000E4B10B50022012002214FF4FA744FF0BA
:10765C00080C5C6283F805C09860D9601A621A70D5
:10766C0058709970DA701A719A711A611A755A7584
:10767C009A75DA751A76DA6110BD00BFB004002075
:10768C002A4B4FF4FA6CC3F814C04FF0020CC3F839
:10769C001CC00CF1040CF0B583F821C00CF1020CE9
:1076AC0083F825C00CF1C00CC3F85CC040F2DC5C64
:1076BC00C3F838C0DFF878C04FF47A650022012097
:1076CC004FF4FA7405274FF49676DD63C3F854C073
:1076DC001D605D6043F2903C4FF47A751F615E63F0
:1076EC00A3F84020DC6483F85000C3F858C09C60B9
:1076FC00DF60986183F8200083F8222083F8232030
:10770C0083F82420DD841A8583F82A0083F82B0063
:10771C0083F82C201E6383F842205C649C6483F8FD
:10772C00512083F8602083F82D20F0BDC403002085
:10773C0000390300024B4FF400721A61704700BF0E
:10774C0000100140024B4FF400725A61704700BFA9
:10775C0000100140024B4FF400521A61704700BFF9
:10776C0000100140024B4FF400525A61704700BFA9
:10777C0000100140024B986800F40050704700BFA5
:10778C0000100140014B10225A6170470008014063
:10779C00014B10221A61704700080140014B042272
:1077AC001A617047000C0140014B04225A6170476A
:1077BC00000C0140054B9A6812F0040F02D0042211
:1077CC005A6101E004221A61704700BF000C0140AD
:1077DC00014B20221A617047000C0140014B202202
:1077EC005A617047000C0140704700BF704700BFE2
:1077FC00704700BF704700BF704700BF704700BFA5
:10780C00704700BF704700BF704700BF704700BF94
:10781C00704700BF18B9024B4FF480525A61704741
:10782C00000C014018B9024B4FF480521A6170479A
:10783C00000C014018B1012806D0002008E0054BCF
:10784C009868C0F3400003E0024B986800F0010018
:10785C00704700BF000C014008B1002003E0024B50
:10786C009868C0F300307047000C0140704700BFAF
:10787C00704700BF00207047704700BF38B5084BF9
:10788C0040F2FF74074D1868214600F0C1F92868D2
:10789C00214600F0BDF96868214600F0B9F938BD01
:1078AC00140200201400002008B5052804D8DFE8D5
:1078BC0000F005080A0D1013002011E0094B986820
:1078CC000CE0094B00E0074B186807E0054B5868C3
:1078DC0004E0044BD86801E0024B186900F090F901
:1078EC0008BD00BF1400002014020020094B10B585
:1078FC009C6814F0070401D0072C05D1012803D192
:10790C001F3001F00FFF02E0202001F013FF204692
:10791C0010BD00BF000801402DE9F3414E4F01ADF1
:10792C000420012107F0FAF9032410264FF0180364
:10793C0038462946ADF804308DF806408DF80760BE
:10794C0007F038FE082001213E6107F0E7F941F20B
:10795C003C43424829464FF00408ADF804308DF8FA
:10796C0006408DF8076007F025FE4FF400733B4886
:10797C002946ADF804308DF806408DF8078007F0E5
:10798C0019FE4823294635488DF8073040F6030385
:10799C0007F50067ADF804308DF8064007F00AFED5
:1079AC003046012107F0BAF938464FF60023294634
:1079BC00ADF804308DF806408DF8076007F0FAFD3D
:1079CC004FF4A04338463B6129464FF48063ADF831
:1079DC0004308DF806408DF8078007F0EBFD4FF072
:1079EC003F03384629460027ADF804308DF8064091
:1079FC008DF8077007F0DEFD2020012107F08EF9CD
:107A0C0029461748ADF804808DF806408DF80760BC
:107A1C0007F0D0FD3B463A4610484FF48064446171
:107A2C0001468068013210F4006F4FF480600861E9
:107A3C00896808BF013311F4006F18BF01370A2A97
:107A4C00EAD10A2B01D0002003E00A2F14BF00203A
:107A5C000120BDE8FC8100BF00080140000C014082
:107A6C000014014007B500238DF8073004484FF08F
:107A7C003F0301A9ADF8043007F09CFD0EBD00BF1B
:107A8C0000100140704700BFFEE700BFFEE700BFDB
:107A9C00FEE700BFFEE700BF704700BF704700BFA6
:107AAC00704700BF704700BF704700BF704700BFF2
:107ABC00704700BF704700BF704700BF704700BFE2
:107ACC00704700BF704700BF704700BF704700BFD2
:107ADC00704700BF704700BF704700BF704700BFC2
:107AEC00704700BF704700BF704700BF08B5024B1E
:107AFC001B68984708BD00BF5803002008B5024B0F
:107B0C001B68984708BD00BFAC040020684620F0F5
:107B1C000701044B8D4601B51B689847BDE8014031
:107B2C00854670478004002008B5024B1B689847B7
:107B3C0008BD00BF88040020704700BF704700BF1D
:107B4C00704700BF704700BF704700BF704700BF51
:107B5C00704700BF704700BF704700BF704700BF41
:107B6C00704700BF704700BF704700BF704700BF31
:107B7C00704700BF704700BF704700BF704700BF21
:107B8C00704700BF704700BF704700BF704700BF11
:107B9C00704700BF704700BF704700BF704700BF01
:107BAC00704700BF704700BF704700BF704700BFF1
:107BBC00684620F007018D4601B5002303E00B4910
:107BCC005958995004330A4A0A4998188842F6D3EE
:107BDC00094B02E0002243F8042B084A9342F9D3E4
:107BEC00FCF7F6FABDE8014085467047D00A01085B
:107BFC00000000209001002090010020942B002018
:107C0C00024B33F8100080B2704700BF24020020F2
:107C1C00024B03EB40031982704700BF2402002083
:107C2C00024B03EB4003188A704700BF240200206C
:107C3C0010B50A4C24781CB9002914BF0A461A4600
:107C4C0050214843064B424302991878039B002865
:107C5C0008BF0B4692FBF3F010BD00BF7409002067
:107C6C0076090020A5234343044AA3F5A5231068F5
:107C7C004FF48052584390FBF2F070474C000020B8
:107C8C00014B1870704700BF76090020014B18702B
:107C9C00704700BF74090020074B10B51B68074CD8
:107CAC0034F8130080B2FFF7DDFF20220146206A72
:107CBC0004F0A4FB206210BD180000202402002058
:107CCC00F8B5114B114E1B68044636F8130080B200
:107CDC00FFF7C8FF0E4B05461B6836F8130080B241
:107CEC00FFF7C0FF064605FB05F006FB06007719FB
:107CFC007F4207FB070004F0E7FAA680A0606780CC
:107D0C0025802046F8BD00BF14020020240200206C
:107D1C0018000020F8B5114B114E1B68044636F8BC
:107D2C00130080B2FFF79EFF0E4B05461B6836F81A
:107D3C00130080B2FFF796FF064605FB05F006FB25
:107D4C00060077197F4207FB070004F0BDFAA780F5
:107D5C00A060668025802046F8BD00BF140200207C
:107D6C00240200201400002038B5104C257885B171
:107D7C00012D1AD10E4B5B6A002BB8BF5B42B3F5D9
:107D8C00E16F12DDFFF7DEFC00232370094B1D7041
:107D9C000BE0074B5B6AC733B3F5C77F05D8FFF71A
:107DAC00C9FC044A01231370237038BD76090020E6
:107DBC0024020020750900202DE9F74F534C0025B3
:107DCC00074665625248884692469946DDF834B0BB
:107DDC0006F004FBC8F5E168404501D307241EE01A
:107DEC004C4B626A1B68002A34F8130004EB430105
:107DFC000B8A80B2B8BF5242C01A80EAE073A3EB80
:107E0C00E07393420E9BC8BF606251460193CDF85C
:107E1C0000B04A460C9BFFF70BFF062405463C4876
:107E2C0006F0E0FA404501D3002621E03A4A374BF0
:107E3C001268596A33F8120003EB4206328A80B298
:107E4C00801A81EAE172A2EBE17280EAE071A1EBA7
:107E5C00E0719142C8BF58620E9BCDF800B00193FF
:107E6C0051464A460C9BFFF7E3FE24F002040646FB
:107E7C00274806F0BBFA404502D34FF0000822E039
:107E8C00264A224B1268596A33F8120003EB420C53
:107E9C00BCF8102080B2801A81EAE172A2EBE17288
:107EAC0080EAE071A1EBE0719142C8BF58620E9B71
:107EBC00CDF800B0019351464A460C9BFFF7B8FE33
:107ECC0024F004048046022C07D0042C09D0012C89
:107EDC000BD108EB06056D4207E008EB0506764270
:107EEC0003E006EB0508C8F1000805FB05F006FBEE
:107EFC00060008FB080004F0E7F9A7F80480B86056
:107F0C007E803D803846BDE8FE8F00BF24020020F5
:107F1C00002C014014020020140000201800002046
:107F2C0070B590B0FFF79EFD0120014606F0E8FE0B
:107F3C0001214FF4007006F0F1FE414807F00CFDF2
:107F4C00404B00240093404B07260193802305935C
:107F5C00DB18069303F540730793A3F57873384841
:107F6C006946089303F5FF5309930294039604940E
:107F7C000A9407F061FD0121314807F08DFD0125C0
:107F8C004FF4602331480BA90D930B948DF83050AE
:107F9C008DF831400E948DF83C6007F0CDFD2C4BE4
:107FAC002A4819782A46032307F048FE294B022257
:107FBC0019782648032307F041FE274B0322197832
:107FCC002248134607F03AFE244B042219781F4826
:107FDC00032307F033FE224B052219781B48032399
:107FEC0007F02CFE1F4B062219781848032307F0C4
:107FFC0025FE1D4B324619781448032307F01EFE4C
:10800C00224612484FF4FC6107F0DAFD0F4829466E
:10801C0007F0CCFD0D48294607F0BEFD0B4807F0D4
:10802C00D9FD0A4807F0DCFD0028FAD1074807F013
:10803C00DBFD064807F0DEFD0028FAD110B070BD5C
:10804C00080002404C24014024020020002401407E
:10805C002C0000202D0000202E0000202F000020DE
:10806C00300000203100002032000020F0B54469BF
:10807C00856903466543881A4FF47A7C002895FB82
:10808C00FCF6B8BF4042B042B8BF0CFB00F5104E36
:10809C004FF47A7C30682D1895FBFCF00CFB1057D4
:1080AC0037600CB9114611E0914205DA1B68411892
:1080BC009942A8BF194609E008DD064A1B6895FBE2
:1080CC00F2F569185B429942B8BF19460846F0BDF3
:1080DC004C02002018FCFFFF2DE9F047044690F8F5
:1080EC0021000D46062816469846DDF820A0276884
:1080FC0000D0F0B92868014608F0C0F83D4908F0F6
:10810C00BDF8814694F82500400808F063F8014654
:10811C00484608F0B3F8636981467820584308F064
:10812C0059F80146484608F05DF908F06DFA034627
:10813C0011E0072801D000230DE00868014608F083
:10814C009DF82D4908F04EF908F05EFAE36B626970
:10815C00434393FBF2F3C245C8EB0A08B8BF7F4216
:10816C00B8F1000FB8BFC8F100084FF48040984533
:10817C00D8BF002701F0E6FA012803D1304608F0F9
:10818C0029F831E0384608F025F82E68804641463B
:10819C00304608F011FA70B1A069636937B90B2247
:1081AC005043584308F012F8144917E0584308F0AC
:1081BC000DF8134912E04146304608F01BFAA0B105
:1081CC00A069636937B90B225043584307F0FEFF8F
:1081DC000C4903E0584307F0F9FF0B4908F002F98A
:1081EC000146304607F042FF2860286808F00CFA78
:1081FC00BDE8F0870000C0400000F04200401C4683
:10820C0000007A4400401CC600007AC4024B0022D5
:10821C009A601A605A60704750020020014BB3F903
:10822C000C0070475002002070B546680446154695
:10823C000846324671421E4604F0C0F8236B00B269
:10824C00B3607368616B451BE818F1603560706052
:10825C0011B1104B93FBF1F10A46494204F0AEF810
:10826C000346F068B168326858434A434FF4803192
:10827C0090FBF1F0A1F57F4192FBF1F28018306197
:10828C007360A1F5014147F6FF7204F097F800B254
:10829C0070BD00BF0000FF7F2DE9F04F89B0A44DE9
:1082AC00BDF84840BDF84AC02C82A5F812C004465F
:1082BC0028699B46DDF8548089460192169EDDF8AC
:1082CC0060A003F05DFBC0F30F43ADF81A30ADF8BE
:1082DC001800069BB8F800706B6194F82130072BDE
:1082EC0025D0082B00F06282062B40F0DA8202F0D7
:1082FC00F7FE94F82D3085B2012B0AD194F8251095
:10830C001A984908E26902F0C5FE02F07FFE451991
:10831C00ADB294F82430012B03D105F5FE45FF35A1
:10832C00ADB22DB2284602F0A9FE0020FAE103F00E
:10833C002DF8012840F011824FF4806001F002FA10
:10834C00012813D04FF4007001F0FCF9012801D181
:10835C00199B5BB94FF4006001F0F4F9012840F06F
:10836C00F981D8F80030002B00F0F48194F82A0041
:10837C00012800F0788104D302286D4B40F0D7819E
:10838C0073E06B4B42F210715A6801328A425A60A8
:10839C0025D8A56BB4F862305543B3F5007FB5FB17
:1083AC00F1F5ADB202D0B3F5806F02D12BB2C8F8A3
:1083BC000030002002F062FE002002F0FBFF0021E2
:1083CC005C4803F081FA04A9C0F30F43ADF8100028
:1083DC0004223046ADF8123007F07AFD74E2564AAA
:1083EC00002012785860012A12D1A58F03F028F8CA
:1083FC00281A80B2254625F8400F02F0F7FF4F4BA4
:10840C0029461B680222ED18281B01F083FB14E09F
:10841C0002F0C4FF94F82A302BB994F8423043F0A0
:10842C00010384F8423094F82A30022B05D194F8D9
:10843C00423043F0020384F842303D4B4FF00001D0
:10844C0059831983584600F01FFB484600F01CFB6B
:10845C00179A002300201360CAF8003002F090FF36
:10846C004FF4004001F05EF919E21B68032B00F297
:10847C001682DFE813F004004800D000D0002E4A2A
:10848C002B4B1278012A00F0C4805A6842F210710A
:10849C008A422BD8A56B013255435A600020B5FB9C
:1084AC00F1F5009302F0EAFD002002F083FF009B3F
:1084BC00002103F1140003F007FA0422C0F30F4368
:1084CC00ADF8100004A93046ADF8123007F000FDED
:1084DC00B4F86230ADB2B3F5007F03D0B3F5806F62
:1084EC0040F0F2812BB2C8F80030EDE1002000938F
:1084FC0002F054FF94F8422042F0020284F8422029
:10850C00009B012285E00C4A094B1278012A17D1F5
:10851C00B4F84000009302F069FF02F0A3FF00F5ED
:10852C000040009B013000B202221A609860B6E154
:10853C0050020020640200202202002004000020CF
:10854C009D6894F8252085EAE5705208A0EBE5704B
:10855C00C2EB024188425BDAE16DE769C1EBC131E4
:10856C004F435743B4F86220B148B2F5007F97FBF4
:10857C00F0F702D0B2F5806F10D1DAF800A000212C
:10858C00504608F037F808B1ED1B05E050460021C5
:10859C0008F012F870B17D19A64B0AE0B2F5006F25
:1085AC0008D1D8F80020002A01DDED1B01E001D034
:1085BC007D199D609F4F0020258F02F05FFDB868EC
:1085CC0002F0F8FEB7F9081007F1140003F07CF97B
:1085DC000422C0F30F43ADF8100004A93046ADF8E7
:1085EC00123007F075FCB4F86230B3F5007F02D09E
:1085FC00B3F5806F02D12BB2C8F8003094F84270FA
:10860C0017F0020740F060818A4B02221A605CE18D
:10861C0003221A6043E1874D4FF000022A836A83DC
:10862C00584600F031FA484600F02EFA2A6817999D
:10863C000023022A0B60CAF8003005D1002002F09A
:10864C009FFE4FF4004000E080207A4D01F06AF864
:10865C00002002F013FDA86802F0ACFEB5F908107A
:10866C0005F1140020E1FFF741F9724D01468046F7
:10867C00287F02F0D1FC85F81C801FFA80F802F0EC
:10868C002FFD94F8243005B2012B04BF05F5FE45EF
:10869C00FF35284602F0F2FC18F4004F03D005F524
:1086AC00D445AA3511E0B8F1000F00F0358105F57D
:1086BC00144505F5AA7508E000F5FE40FF3080B2C0
:1086CC0000F5FE45FF35ADB227E05B4BE06B1A7849
:1086DC0094F82530012A0BD000B245435B0895FB7A
:1086EC00F3F04FF6FF7390FBF3F080B202F09AFEBA
:1086FC0002F0B8FE4F4B4FF000025A831A83054626
:10870C00584600F0C1F9484600F0BEF9002002F0CE
:10871C0037FE4FF4004001F005F805F50045013532
:10872C002DB2284602F046FE2946444830E003F1BB
:10873C001400002103F0C8F80027C0F30F43ADF874
:10874C00100004A930460422ADF812303D4607F063
:10875C00BFFBBAE000213948A6E002F083FE94F892
:10876C002A3000F500400130012B85B203D102F014
:10877C00B7FC00B200E000200FFA85F802F07EFC96
:10878C00404602F017FE2B4B414603F114009D812D
:10879C0003F09AF804A9C0F30F43ADF810000422BB
:1087AC003046ADF8123007F093FB78E0E26994F8AC
:1087BC0025304FEA0238DAF8000003FB08F807F01E
:1087CC0023FF0028B8BF404200FB08F82B6A40F298
:1087DC00DC5298FBF2F89844642398FBF3F203FB09
:1087EC001283DAF800A02B62002150464FF00005EE
:1087FC0007F000FF08B14FF00105EDB225B10D4BAC
:10880C006FF063019A8907E05046002107F0D4FE0F
:10881C0038B1084B64219A8998FBF1F89044A3F87D
:10882C000C80044BB3F80C8055B108F580480EE071
:10883C00C027090050020020220200206402002000
:10884C005046002107F0B8FE18B1A8F580481FFA71
:10885C0088F80FFA88F1354803F036F80422C0F393
:10886C000F43ADF8100004A93046ADF8123007F0F4
:10887C002FFB02F035FC94F8243080B2012B03D18D
:10888C0000F5FE40FF3080B200B202F0F7FB02F0C0
:10889C00E9FD00F50040013000B202F08BFD00252F
:1088AC0013E005F11400002103F00EF80025C0F3CD
:1088BC000F43ADF8100004A930460422ADF8123075
:1088CC002F4607F005FB00E0002739B24B46B6F9FE
:1088DC0000202046FFF7A8FC154F019B388329B2D6
:1088EC00B6F902202046FFF79FFC788307F11800A9
:1088FC0002F046FF07F1180002F068FFC0F30F43C7
:10890C00ADF80800ADF80A30029B18467B6201F006
:10891C00F3FE09B0BDE8F08F02F0E2FB94F82430CE
:10892C0080B2012B7FF4CCAEC6E600BF64020020FF
:10893C00500200202DE9F041066804461546084611
:10894C00324671421E4603F039FDD4F84880431B71
:10895C00C6F80880E56C1E4933600746F56018467A
:10896C004FF6FF7203F02AFD03467068F168181881
:10897C003360706019B16168090491FBF5F10A4626
:10898C00494203F01BFD3268034605FB00F002FB75
:10899C0008F84FF4803290FBF2F0A2F57F4298FB7E
:1089AC00F2F840443061736094F82130082B08D100
:1089BC00002F01DDA06B09E016BFA06B38464042CA
:1089CC0004E061680A46494203F0F8FCBDE8F08116
:1089DC000100FFFF70B5466C1D4604469E60881A68
:1089EC000023EB6028600A494FF6FF7203F0E6FCA7
:1089FC000346A8684FF48072584390FBF2F028614C
:108A0C002B6021680A46494203F0D8FC70BD00BFB8
:108A1C000100FFFFF8B546680C460546714210464A
:108A2C0032461F4603F0CAFC2E6B6368A660696B66
:108A3C00C71BF8180425E16091FBF5F52760606011
:108A4C0011B10F4991FBF5F10A46494203F0B6FC0E
:108A5C0023680822454396FBF2F65E434FF48033BD
:108A6C0095FBF3F5A3F57C4396FBF3F6AD1960602B
:108A7C0025612846034940F60F6203F09FFCF8BDC0
:108A8C0000000F0EF1F1FFFF002303610360436050
:108A9C00704700BF094B19685A68914201D10020F8
:108AAC000BE01A68D118097A013201701A601A6841
:108ABC00202A01D100221A60012070477802002080
:108ACC00014B9862704700BF78020020034B1A7864
:108ADC00104612B100221A7001207047780900204C
:108AEC0038B50B4B8446DC6A1A6B0134202C08BF5A
:108AFC00002494420BD0DD6A064AED18106885F804
:108B0C0034C040F227710122DC6204F0A1FE38BDB2
:108B1C00780200205400002038B50546002401E0FE
:108B2C00FFF7DEFF2B5D01341846002BF8D138BD62
:108B3C0070B5294C238813F0200F1AD0FEF79AFE3B
:108B4C0008B1A38815E0254B5A6819680132202A10
:108B5C0008BF00228A4205D05968A088C918C0B243
:108B6C0008725A601E4B0A221A601C4B9A6A1D4BE3
:108B7C001A60194E338813F0800F1BD0194B1C68E8
:108B8C00C4B9164DEA6A2B6B9A420DD0FEF76EFEF5
:108B9C002B6B5A1992F834200133B2802B632B6B58
:108BAC00202B07D12C6305E03046224640F227717A
:108BBC0004F04EFE0848038813F0400F0AD040F230
:108BCC00266104F03DFF054B1A6BDB6A9A4201D11A
:108BDC00FEF74EFE70BD00BF00480040780200203A
:108BEC007C0900208009002070B5294C238813F0E3
:108BFC00200F1AD0FEF73EFE08B1A38815E0254BD6
:108C0C005A6819680132202A08BF00228A4205D00E
:108C1C005968A088C918C0B208725A601E4B0A2243
:108C2C001A601C4B9A6A1D4B1A60194E338813F04C
:108C3C00800F1BD0194B1C68C4B9164DEA6A2B6BFC
:108C4C009A420DD0FEF712FE2B6B5A1992F8342073
:108C5C000133B2802B632B6B202B07D12C6305E0E7
:108C6C003046224640F2277104F0F2FD0848038892
:108C7C0013F0400F0AD040F2266104F0E1FE054BE0
:108C8C001A6BDB6A9A4201D1FEF7F2FD70BD00BF90
:108C9C0000440040780200207C090020800900205C
:108CAC0070B57B4B86B01C780546012C2AD17948CF
:108CBC0004F016FF21464FF4003006F03DF8214633
:108CCC00042006F02BF80420002106F043F80820BD
:108CDC00002106F0FFFC06AC4FF0040324F8043D21
:108CEC00032321466C488DF8163015338DF8173058
:108CFC0006F060FC48238DF81730214666484FF08B
:108D0C0008032DE0654B1C78012C2DD1644804F030
:108D1C00E7FE21464FF4802006F00EF8214608208D
:108D2C0005F0FCFF0820002106F014F85D48002136
:108D3C0006F0D0FC06AC4FF4806324F8043D03230A
:108D4C00594821468DF8163015338DF8173006F03A
:108D5C0031FC042354488DF8173021464FF400633E
:108D6C00ADF8143006F026FC684604F03BFD0B2DE4
:108D7C0025D8DFE805F02406090C0F1215181B1E68
:108D8C0020224FF461531CE04FF4964319E04FF44A
:108D9C00E14316E04FF4164313E04FF4614310E047
:108DAC004FF496330DE04FF4E1330AE04FF46133A6
:108DBC0007E03E4B05E03E4B03E03E4B01E04FF439
:108DCC00165300933C4B1A683C4B9A4202D1009BC1
:108DDC005B0800932E4B1B78012B04D1384B2D4A8A
:108DEC001A60262307E02D4B1B78012B05D1344B41
:108DFC002B4A1A6027238DF81030314C69462068B5
:108E0C0004F026FE00250723012604A88DF8113056
:108E1C008DF812508DF8136006F04EF8206840F271
:108E2C00FF3104F0E9FD206828212A4604F010FDEA
:108E3C002068324640F2277104F00AFD2068324661
:108E4C0040F2266104F004FD2068324640F22551C0
:108E5C0004F0FEFC20682A4640F2244104F0F8FCA1
:108E6C0020682A4640F6460104F0F2FC20682A46A7
:108E7C0040F66A1104F0ECFC206860212A4604F0EC
:108E8C00E7FC2068314604F0D5FC06B070BD00BF8D
:108E9C001C02002000440040000801404300002058
:108EAC000048004010001400000C014090D003005A
:108EBC0020A1070040420F00500000200024F400C5
:108ECC0054000020014B03221A607047CC02002092
:108EDC00044A054B927A0AB1052200E001221A607D
:108EEC00704700BF94090020CC020020704700BFDF
:108EFC00014B00225A607047CC02002008B5074B8A
:108F0C001A6892B242F008021A601A6892B242F0E1
:108F1C0004021A60FFF7D6FF08BD00BF405C00409A
:108F2C0010B5064C4FF6FB73226802EA030323606C
:108F3C00FFF7CEFF4FF40643236010BD405C0040AA
:108F4C00072818BF1F4B10B51E4C18BF187023787C
:108F5C00052B33D8DFE803F003060A0E1621FFF7C2
:108F6C00DFFF2BE0FFF7DCFF042328E00223637014
:108F7C00013324E06378013BDBB263706378FBB9A7
:108F8C00042218E0104B1A6892B242F010021A60D8
:108F9C0005232370DB18637012E06378013BDBB2AE
:108FAC006370637863B9084A4FF6EF73116801EA8E
:108FBC00030313600622034B1A7001E0062323708F
:108FCC0010BD00BFF8090020405C0040034B9B7AA9
:108FDC0013B1034B05221A60704700BF940900209F
:108FEC00CC020020014B04221A607047CC020020F6
:108FFC00034B1A7A202A01D100221A72704700BF43
:10900C00CC020020704700BF212808B508D1124BB4
:10901C001B681B7803F07F03212B1AD10F4B0EE03A
:10902C00202816D10C4B0E4A1B681B7810720D4A67
:10903C0003F07F03212B0CBF134600234BB1064AD0
:10904C004FF0000112680020518293619847002074
:10905C0000E0022008BD00BFF4090020A990000820
:10906C00CC020020C5900008074B1B681B7803F04E
:10907C007F03212B05D1022801D0222801D1002009
:10908C0000E00220704700BFF409002019B9012844
:10909C0001D8084600E00220704700BF28B9044BF5
:1090AC004FF008021B681A8200E00248704700BFAC
:1090BC00F40900205800002028B9044B4FF0080296
:1090CC001B681A8200E00248704700BFF4090020B8
:1090DC00580000200B4B10B5DA6882B11B68052BC9
:1090EC0001D000220BE0002303E00749595CC15476
:1090FC0001330449CC68A342F7D30023CB6010465C
:10910C0010BD00BFCC020020000A0020084BDB6819
:10911C00082B01D800200AE00023064A9A5CC254AE
:10912C000133092BF9D1024B0022DA600120704780
:10913C00CC020020000A0020704700BF10B5074C7D
:10914C000B468AB2C021636003F0B6FD0120A188F2
:10915C0003F0DEFB012003F0A9FA10BDCC020020C5
:10916C0008B5064B1B68DB78042B01D9002004E002
:10917C00034901EBC30103F0FFFF08BDF409002014
:10918C006000002008B5024903F0F6FF08BD00BFDF
:10919C008000002008B5024903F0EEFF08BD00BFB7
:1091AC0088000020334B10B51B686FF03F02002481
:1091BC005A72DC729C72204603F0F0F920464FF490
:1091CC00007103F009FA1021204603F01BFA40212C
:1091DC00204603F071FB8021204603F05DFB204606
:1091EC0003F09AFA244B204693F8641003F0B2FB78
:1091FC00204603F069FA0120214603F0EDF9012025
:10920C00C02103F049FB0120202103F0FBF90120D0
:10921C00214603F00FFA02204FF4C06103F0DCF991
:10922C0002204FF4807103F037FB0220214603F03B
:10923C0001FA0220202103F0E5F90320214603F076
:10924C00CBF903204FF4887103F036FB0320402147
:10925C0003F080FB03204FF4405103F0EBF921465F
:10926C00032003F0CFF9204603F094FF034B0122B7
:10927C001A6010BDF409002058000020CC02002018
:10928C0008B5174B174A196889B21180164912880C
:10929C00098801EA020212F4806F05D04FF6FF3202
:1092AC001A60124BDB6B98470E4B1A880E4B1B88BF
:1092BC0003EA020212F4007F08D009490C4A4FF667
:1092CC00FF500860117C0131C9B21174054A128833
:1092DC00134013F4004F01D003F05AFD08BD00BF3A
:1092EC00445C004086090020400A00205800002001
:1092FC00CC02002010B5032003F05CFB064C0346A7
:10930C0002464FF488710548E36003F0EDFC03203E
:10931C0003F0DAF910BD00BFCC020020000A0020D7
:10932C0008B5064A064B20B11068198806F0AAF950
:10933C0003E01068198806F0A3F908BD9009002015
:10934C008C09002038B5064D01232B60054B0024F9
:10935C0020461C60FFF7E4FF03232B60204638BD3A
:10936C00405C0040445C004008B5FFF7EBFF08BDD3
:10937C0008B50120FFF7D4FF064B012119600649FF
:10938C004FF4E0520A8005490020186008601A600A
:10939C0008BD00BF405C0040400A0020445C004017
:1093AC00084B10B51B6800249C72FFF7E1FF064ABE
:1093BC004FF406431460043A1360044A1460044AE0
:1093CC00138010BDF4090020445C0040CC02002046
:1093DC00400A002007B5142200238DF8042001A8B0
:1093EC0001228DF806308DF807208DF8053005F038
:1093FC0063FD0EBD002008B505F006FC4FF400001F
:10940C00012105F099FC08BDF7B5184C184E194F01
:10941C00194D9DF820C031602A803860099930229E
:10942C0004F17E0084F8723084F873C006F050FDAD
:10943C000A99182204F1B20006F04AFDFFF7DAFF90
:10944C00FFF7C8FF03F068FD3868012105F066FCE2
:10945C0003232D888DF8063030680D3301A9ADF843
:10946C0004508DF8073006F0A5F8FEBD580000201A
:10947C0090090020FC0900208C090020014B186881
:10948C00704700BFA8290020014B1868704700BF27
:10949C00A0290020014B1868704700BF9C290020B0
:1094AC00014B1868704700BF94290020014B1868C5
:1094BC00704700BFA4290020014B1868704700BFFB
:1094CC0088290020014B1868704700BF90290020A4
:1094DC00014B1868704700BF8C290020014B18689D
:1094EC00704700BF98290020014B1868704700BFD7
:1094FC00440A0020014B1860704700BFA8290020C7
:10950C00014B1860704700BFA0290020014B186068
:10951C00704700BF9C290020014B1860704700BFAA
:10952C0094290020014B1860704700BFA42900202B
:10953C00014B1860704700BF88290020014B186050
:10954C00704700BF90290020014B1860704700BF86
:10955C008C290020014B1860704700BF982900200F
:10956C00014B1860704700BF440A0020094B03F5FB
:10957C00FA5C00221A605A609A60DA601033634514
:10958C00F7D1054B59600121DA60187059721A72C3
:10959C00704700BF480A0020E0020020024B002266
:1095AC00DA605A721A727047E0020020014B187A86
:1095BC00704700BFE0020020014B587A704700BF93
:1095CC00E0020020014BD868704700BFE002002089
:1095DC0008B5064B0021DA6819610132B2F5FA7F41
:1095EC00DA6001D1FFF7DAFF08BD00BFE00200200E
:1095FC00F0B585B0EC468CE80F00114B11491A6997
:10960C000E680132B2421A6103990298019C009DC6
:10961C0013DB1A7A8AB1DB68B3F5FA7F0DDA0A4AE2
:10962C004FEA031C02EB03170CEB02064CF802503A
:10963C007C60B860F160FFF7CBFF05B0F0BD00BFF8
:10964C00E002002088010020480A00204FF4FA7044
:10965C00704700BF4FF4FA50704700BF04207047AA
:10966C00B0F5FA7F07DA032905D8044B01EB80002B
:10967C0053F8200000E00020704700BF480A00208B
:10968C00074B032809D8DFE800F008020406012282
:10969C0004E0022202E0032200E000225A6170473B
:1096AC00E0020020014B5869704700BFE002002027
:1096BC00014B1860704700BF88010020014B1868EF
:1096CC00704700BF8801002010B5154B93F800C0FF
:1096DC00BCF1060F1DD8DFE80CF00406090C0F12C4
:1096EC001600012214E05B689A420AE05B689A4219
:1096FC000BE05B68994204E05B68994205E05B68AB
:10970C00984206DA02E05B68984202DD044B0122C3
:10971C001A72034B1A7A012A01D1013A5A7210BDFE
:10972C00E0020020024B1A6840EA02021A607047FD
:10973C00F8020020024B1A6822EA00021A607047F5
:10974C00F8020020034B1B6818420CBF00200120BC
:10975C00704700BFF802002008B56D20FFF7EAFF44
:10976C0008BD00BF034B10B51C68FFF7F5FF204682
:10977C0010BD00BFF8020020034B10B51C68FFF7AA
:10978C00EBFF04F06F0010BDF802002062B67047CA
:10979C0072B6704708B5FDF7E5FF08BD08B5FDF7D3
:1097AC00D9FF08BD08B510B105F024FC01E005F0A7
:1097BC0029FC08BD07B5104B1B78E3B1FEF728F860
:1097CC00FDF7ECFFFEF70AF8002301E0019B0133E3
:1097DC000193019A094B9A42F8D9FDF7E5FFFDF781
:1097EC00F7FF002301E0019B01330193019A034B26
:1097FC009A42E3D8F7E70EBDB50300203F0D0300F6
:10980C0008B5FEF789F8014B187008BDB5030020A8
:10981C002DE9F341234B05461B788846012B164650
:10982C001DD1002418E001AF4FEA152C3946022255
:10983C00A6231D488DF804C08DF8055002F06CFB72
:10984C00A62339461848022202F0DCFB9DF80430AE
:10985C00013508F804300134B442E4D31FE0002091
:10986C000321024602F07AF90020C5F307210246D3
:10987C0002F074F90020E9B2024602F06FF90024FC
:10988C0008E0944214BF0022012202F067F908F8A4
:10989C00040001340020721EB4420146F1D3BDE82D
:1098AC00FC8100BF210200200058004073B5174B0B
:1098BC00050A1B780446012B13D101AE3146022256
:1098CC00A53313488DF804508DF8054002F024FBA5
:1098DC0031460F480222A62302F094FB9DF80400A7
:1098EC0013E000200321024602F038F90020E9B20F
:1098FC00024602F033F90020E1B2024602F02EF9E2
:10990C0000200146012202F029F97CBD2102002031
:10991C000058004037B52D4B0C461B78012B4CD012
:10992C000725454300200321024602F017F905F5EF
:10993C0000650020C5F30721024602F00FF9002054
:10994C00E9B2024602F00AF900200146024602F092
:10995C0005F98DF8000000200146024602F0FEF8E1
:10996C008DF8010000200146024602F0F7F88DF850
:10997C00020000200146024602F0F0F88DF80400C7
:10998C0000200146024602F0E9F88DF8050000209F
:10999C000146024602F0E2F88DF806000020012292
:1099AC00014602F0DBF82368009A23F07F4322F093
:1099BC007F429A428DF8070001D0002005E06368D1
:1099CC000198984214BF002001203EBD21020020C6
:1099DC0038B5234B1B78012B41D0224B1C683BE044
:1099EC0000200621012202F0B9F8002005210246D0
:1099FC0002F0B4F800200122014602F0AFF810F09A
:109A0C00020FF2D000200221024602F0A7F800203B
:109A1C00C4F30721024602F0A1F80020E1B202468D
:109A2C0002F09CF8002500203F2D14BF00220122DB
:109A3C000146013502F092F8402DF4D100200521A9
:109A4C00024602F08BF800200122014602F086F853
:109A5C0010F0010FF2D14034B4F5804FC0D338BDB3
:109A6C00210200201000002038B5224B0C461B7838
:109A7C00012B3DD00725454300200321024602F06F
:109A8C006DF805F500650020C5F30721024602F0CC
:109A9C0065F80020E9B2024602F060F800200146A9
:109AAC00024602F05BF8207000200146024602F0EC
:109ABC0055F8607000200146024602F04FF8A07085
:109ACC0000200146024602F049F8207100200146B0
:109ADC00024602F043F8607100200146024602F093
:109AEC003DF8A07100200146012202F037F8E07128
:109AFC0038BD00BF2102002010B500F09BFD0446CC
:109B0C0000F098FD001B0028B8BF40420628F7DD86
:109B1C0010BD00BF2DE9F3414D4B06461B780F4697
:109B2C00012B14461AD100250DE017F805E08DF82D
:109B3C0004C08DF806E08DF8056002F0EDF9FFF732
:109B4C00DBFF01360135A5424FEA162C01A94FF077
:109B5C0003024FF0A6033F48E7D376E0002006212E
:109B6C00012201F0FBFF00200521024601F0F6FF67
:109B7C0000200122014601F0F1FF10F0020FF2D09B
:109B8C0000200221024601F0E9FF0020C6F3072164
:109B9C00024601F0E3FF0020F1B2024601F0DEFFC5
:109BAC00002543E0013616F03F08795D01D1012212
:109BBC0004E0621E954214BF00220122002001F035
:109BCC00CDFFB8F1000F30D1631E9D422DD2002085
:109BDC000521024601F0C2FF00200122014601F0DE
:109BEC00BDFF10F00100F2D10621012201F0B6FFF9
:109BFC0000200521024601F0B1FF002001220146A0
:109C0C0001F0ACFF10F0020FF2D00020022102464E
:109C1C0001F0A4FF0020C6F30721024601F09EFFCD
:109C2C000020F1B2024601F099FF0135A542B9D3EB
:109C3C0000200521024601F091FF0020012201467F
:109C4C0001F08CFF10F0010FF2D1BDE8FC8100BFD8
:109C5C00210200200058004037B5264B04461B78E3
:109C6C000D46012B10D14FEA102C01A90322A5336C
:109C7C0021488DF804C08DF805408DF8065002F08F
:109C8C004BF9FFF739FF33E000200621012201F0E8
:109C9C0065FF00200521024601F060FF0020012233
:109CAC00014601F05BFF10F0020FF2D00020022100
:109CBC00024601F053FF0020C4F30721024601F0D5
:109CCC004DFF0020E1B2024601F048FF294600207A
:109CDC00012201F043FF00200521024601F03EFF66
:109CEC0000200122014601F039FF10F0010FF2D1E2
:109CFC003EBD00BF210200200058004038B5154B76
:109D0C000C461B78012B24D00725454305F500652F
:109D1C00284609780135FFF79FFF28466178013501
:109D2C00FFF79AFF2846A1780135FFF795FF2846E3
:109D3C0021790135FFF790FF284661790135FFF74E
:109D4C008BFF2846A179FFF787FF681CE179FFF7A5
:109D5C0083FF38BD21020020194B70B505461868E9
:109D6C000C46FFF7A3FD174B1B78834202D1164B11
:109D7C001B78BBB1124E00213068FFF76DFFFFF767
:109D8C0027FE124B294618682822FFF7C3FE104BFA
:109D9C00214618686822FFF7BDFE0A4B3068197817
:109DAC00FFF75AFF094B294618682822FFF730FDA8
:109DBC00074B214618686822FFF72AFD70BD00BFCB
:109DCC000C00002000000020B503002090010020B2
:109DDC0004000020084B9A7852B95B78142B05D8F4
:109DEC00064A1168064A42F8231004E0032200E0F8
:109DFC000422044B1A7070474C030020B00300205F
:109E0C005C030020A0040020054B01205A78054972
:109E1C008242087002D15A68034B1A60704700BF27
:109E2C004C0300208C0400204C040020014B022227
:109E3C001A7070478C040020074A00231360074AED
:109E4C001370074A1360074A1360074A1370074AD6
:109E5C001360074A13607047540300208C040020E1
:109E6C004C0400209404002048030020B003002080
:109E7C00D8040020014B00221A7070478C0400207B
:109E8C0030B5234B5B78032B3ED8DFE803F0080298
:109E9C002F39204B18681E4B5C68002322E01D4AAA
:109EAC001368092B07D81A491B484C68591C40F8F1
:109EBC00234011602BE0092227E052F82350591C53
:109ECC00A5420ED102EB810204E052F8041C0133CE
:109EDC0042F8081C411E04328B42F6D30D4B19601C
:109EEC0015E00B4683420C4AE7D310E0094A0023E5
:109EFC001360094A002199500433282BF9D106E04C
:109F0C00064B0A225A6002E00322044B1A7030BD41
:109F1C004C0300209004002050040020A0040020DA
:109F2C00264A274B5278092A3BD8DFE802F0050A6B
:109F3C000F141A22282E343720491A6849688A18B7
:109F4C002EE01E4A196852688A1A29E01B4A1968C1
:109F5C0052684A4324E0194A1968526891FBF2F29C
:109F6C001EE0164A1968526891FBF2F002FB1012BF
:109F7C0016E012491A68496801EA020210E00F491A
:109F8C001A68496841EA02020AE00C491A684968F1
:109F9C0081EA020204E01A68D24301E0074A5268DF
:109FAC001A60074A074B12681AB91A6842F008027D
:109FBC0002E01A6822F008021A6070474C03002075
:109FCC00B0030020540300202A4A2B4B52780A2A53
:109FDC0043D8DFE802F0060B11161C242A30363A5F
:109FEC003D0026491A6809688A1803E0234A196853
:109FFC0012688A1A1A6030E0204A196812684A43BB
:10A00C00F8E71E4A1968126891FBF2F2F2E71B4A54
:10A01C001968126891FBF2F002FB1012EAE717497B
:10A02C001A68096801EA0202E4E714491A68096827
:10A03C0041EA0202DEE711491A68096881EA020264
:10A04C00D8E70E4B1A68D243D4E71A680B4BD1E70A
:10A05C000A4A1868116810601960074A084B1268A0
:10A06C001AB91A6842F0080202E01A6822F00802D3
:10A07C001A6070474C030020B0030020D804002065
:10A08C0054030020134B5B78052B22D8DFE803F038
:10A09C0003080D12171C104B1A6802F00F0217E080
:10A0AC000D4B1A6822F0100212E00B4B1A6822F0CA
:10A0BC0020020DE0084B1A6822F0400208E0064B23
:10A0CC001A6822F0800203E0034B1A6822F48072B3
:10A0DC001A6070474C03002054030020124B1A687E
:10A0EC00124B5B689A4206DD114B196841F0040172
:10A0FC0021F003010CE00E4B05D1196821F006018B
:10A10C0041F0010104E0196821F0070141F002015E
:10A11C001960074B1AB91A6842F0080202E01A6873
:10A12C0022F008021A607047B00300204C03002094
:10A13C005403002010F0020F0CD111F0100F07D0B7
:10A14C00064B04215A68064B1970064B1A6004E042
:10A15C000A2200E00822044B1A7070474C030020BE
:10A16C008C04002044030020A0040020014B00229A
:10A17C001A7070478C0400200F4B5B78032B1AD895
:10A18C00DFE803F0020413150C4B00E00C4B1A68CB
:10A19C000C4B110A93F800C00B4B18780B4B1A712F
:10A1AC0083F807C09871597105E0094B00E0094B21
:10A1BC001A68064B5A6070474C0300204403002079
:10A1CC004C0400208C04002048030020A004002034
:10A1DC00B0030020D8040020014B02221A707047F3
:10A1EC00B4030020024B5A68024B1A60704700BF40
:10A1FC004C0300204C040020294B5B780C2B4ED8D0
:10A20C00DFE803F0070C11161C21262B30353A3FE2
:10A21C004400244B1B6813F0080F3BE0214B1B68D8
:10A22C0013F0080F08E01F4B1B6813F0010F31E00F
:10A23C001C4B1B6813F0010F31D12CE0194B1B6820
:10A24C0013F0040F26E0174B1B6813F0050F21E0E9
:10A25C00144B1B6813F0020F1CE0124B1B6813F01D
:10A26C00030F17E00F4B1B6813F0100F12E00D4B90
:10A27C001B6813F0200F0DE00A4B1B6813F0400F06
:10A28C0008E0084B1B6813F0800F03E0054B1B68BC
:10A29C0013F4807F03D0024B5A68034B1A6070474B
:10A2AC004C030020540300204C040020074970B5D7
:10A2BC000B68072B09D8064A064816684068064DF5
:10A2CC005C1C45F823600C60106070BD9404002089
:10A2DC004C0400204C0300202C040020054B1A6871
:10A2EC0032B10549013A51F822101A60034B19603A
:10A2FC00704700BF940400202C0400204C04002064
:10A30C00014B00221A7070478C040020084B9A787D
:10A31C004AB95A78142A04D85968064B43F82210C3
:10A32C0004E0032200E00422034B1A70704700BFC4
:10A33C004C0300205C030020A0040020114B9A78F1
:10A34C0052B95A78104B142A04D8104951F82220CB
:10A35C005A6004E0032201E00B4B04221A700C4BF0
:10A36C001B786BB1084B0B495A680B4B0A601AB936
:10A37C001A6842F0080202E01A6822F008021A6019
:10A38C00704700BF4C030020A00400205C03002099
:10A39C0084040020B00300205403002010B5094BA6
:10A3AC009A7852B95C78142C05D8FAF701F8064B58
:10A3BC0043F8240004E0032200E00422034B1A704B
:10A3CC0010BD00BF4C0300205C030020A004002043
:10A3DC0038B5284B1B788BB9274A284B5268B2F1F9
:10A3EC00FF3F04BF264A12680A214A431A6000F054
:10A3FC0021F9244B012218601E4B1A701E4B5C78FD
:10A40C0014B1012C35D10EE000F014F91D4B1A6873
:10A41C001A4B821A002A1B68B8BF52429A4224D99E
:10A42C00144B1C7025E0FFF79DF910F4804507D004
:10A43C00154B10491A68002022F01002087017E022
:10A44C000E4C23688BB100F0F5F80E4A23681268A5
:10A45C00821A002AB8BF52429A4206D90A4B0549C1
:10A46C001A680D7042F0100202E0084B1A68013AAB
:10A47C001A6038BD480300204C030020DC08002083
:10A48C00B003002078040020540300204C0400206A
:10A49C0070B5104D104E2868104C32787368B0F5BA
:10A4AC00006F627063600FD83146FFF727FC3146AE
:10A4BC002868FFF72FFA20B12B6801332B60652336
:10A4CC0000E00723237004E007232370044B0022D1
:10A4DC001A7070BD440300204C030020A00400201F
:10A4EC008C04002037B5124C657815B1012D1AD1AA
:10A4FC000FE0104B042201A91868FFF789F9616875
:10A50C00019A0D4B914202D101225A600EE05D601E
:10A51C000CE0A3782A2B06D1064B211D18680422C7
:10A52C00FFF7F8FA02E0044B03221A703EBD00BF9D
:10A53C004C03002008000020A00400202DE9F3416A
:10A54C001E4B1F4C5B681F4A0125B3F5006F15703D
:10A55C00207027DC11EA050624D118466946FFF75E
:10A56C0083FA9DF800809DF801709DF802C09DF85B
:10A57C0007009DF806109DF805209DF80430267202
:10A58C0084F80180A77084F803C020716171A271F6
:10A59C00E3710B4BE95C1A7A01358A18082D1A7293
:10A5AC00F7D108E00123064A002199540133082B06
:10A5BC00F9D113781372BDE8FC8100BF4C03002065
:10A5CC00B8030020B403002008B50A4B0A491A68E6
:10A5DC0002EA010169B95A6840F2D2439A4208D1A1
:10A5EC00064B1868FFF738FBFFF7F2F90120FFF76D
:10A5FC00D9F808BD4C03002000FFFF000C00002020
:10A60C0008B5034B1A68034B5A60FBF771F908BD88
:10A61C00B00300204C03002008B5044B05201A6839
:10A62C00034B5A60FBF7B4FA08BD00BFB00300201F
:10A63C004C030020014B1868704700BFFC0200203F
:10A64C0008B50C4B1B78012B01D1F9F7BDFD04208B
:10A65C0004F052F848F6A04004F05EF8012004F033
:10A66C0061F805480321002204F0F4FC012004F0F9
:10A67C006FF808BD200200209AC3020008B5174BE2
:10A68C001A79CAB11968164A01311960154B11684B
:10A69C001B780131012B116005D1134B1A6812B1D3
:10A6AC001A68013A1A60114B1B78012B01D1F9F78A
:10A6BC008DFD0022094B00E001221A71094B1A781A
:10A6CC00012A09D10A4B196831B11968013919608D
:10A6DC001B680BB9074B1A7008BD00BFFC020020A9
:10A6EC006C0900204200002080090020200200207C
:10A6FC007C0900207809002043F2B60102B24A43DB
:10A70C00494903144B434FF0020C991891FBFCF18F
:10A71C009A1A82B0002992FBFCF2019004DA002A0A
:10A72C002ADB002B6CDC04E0002A56DA002B47DC19
:10A73C0034E003F5E150801A4FF4802190FBF1F0E6
:10A74C0000F5617080B200EB6242A1F5003193FB21
:10A75C00F1F192B2511A89B2344BB3F820C02CF4F7
:10A76C00005C4FEA0C4C4FEA1C4CA3F820C09886B6
:10A77C001A87998702B0704701F5E150801A4FF49F
:10A78C00802390FBF3F000F56170A3F5003380B2E9
:10A79C0092FBF3F291FBF3F182182EE0C3F5E1503A
:10A7AC00401880144FF4003200F5617091FBF2F107
:10A7BC0080B2411A93FBF2F289B28A1892B2CBE7BB
:10A7CC0003F5E150801A801400F561704FF40031EC
:10A7DC0080B292FBF1F28218B9E701F5E150801AD0
:10A7EC004FF4802390FBF3F000F56170A3F5003378
:10A7FC0080B291FBF3F100EB6242411A92B2AAE7EC
:10A80C00C3F5E15040184FF4802290FBF2F000F5B4
:10A81C006170A2F5003291FBF2F180B2411A89B25B
:10A82C0001EB63439AB297E7E0E3FFFF002C014092
:10A83C00064B00F5617001F5617102F5617280B231
:10A84C0089B292B2988619879A877047002C01407A
:10A85C00014B1878704700BFAD290020014B1878C8
:10A86C00704700BFAC290020013808B5052874D802
:10A87C00DFE800F0034D0328284D00210A46374835
:10A88C0003F0C2FC00210A46344803F0CBFC3348E9
:10A89C000421002203F0B8FC30480421002203F00C
:10A8AC00C1FC2E480821402203F0CAFC2B48082189
:10A8BC00012203F0A9FC04222848082103F0B2FC71
:10A8CC00022248E000210A46244803F09DFC0021A6
:10A8DC000A46224803F0A6FC20480421402203F03B
:10A8EC00AFFC1E480421012203F08EFC04210A4611
:10A8FC001A4803F097FC19480821002203F084FC45
:10A90C0000221648082103F08DFC012223E0134895
:10A91C000021402203F094FC10480021012203F096
:10A92C0073FC0E480021042203F07CFC0B4804212C
:10A93C00002203F069FC09480421002203F072FC98
:10A94C0006480821002203F05FFC0022034808217E
:10A95C0003F068FC0022024B1A7008BD002C014069
:10A96C00AC290020013808B5052800F21481DFE875
:10A97C0010F03300E40006008D006000B7000021E9
:10A98C000A46854803F040FC00210A46824803F041
:10A99C0049FC81480421602203F052FC7E480421CA
:10A9AC00012203F031FC7C480421002203F03AFC24
:10A9BC0079480821402203F043FC77480821012202
:10A9CC0003F022FC04227448082103F02BFC734B87
:10A9DC0001221A709218DCE06F480021602203F00B
:10A9EC002FFC6D480021012203F00EFC00210A46C9
:10A9FC00694803F017FC68480421002203F004FCAA
:10AA0C0065480421002203F00DFC63480821402214
:10AA1C0003F016FC60480821012203F0F5FB042228
:10AA2C005D48082103F0FEFB5C4B00221A700232D9
:10AA3C00AFE059480021602203F002FC5648002187
:10AA4C00012203F0E1FB00210A46534803F0EAFB24
:10AA5C0051480421402203F0F3FB4F48042101220A
:10AA6C0003F0D2FB04210A464B4803F0DBFB4A48B7
:10AA7C000821002203F0C8FB00224748082103F0FC
:10AA8C00D1FB464B00221A70013282E000210A46AB
:10AA9C00414803F0B9FB00210A463F4803F0C2FBD2
:10AAAC003D480421402203F0CBFB3B48042101220A
:10AABC0003F0AAFB04210A46374803F0B3FB3648DF
:10AACC000821602203F0BCFB33480821012203F06B
:10AADC009BFB00223048082103F0A4FB022255E026
:10AAEC002D480021402203F0ABFB2B480021012212
:10AAFC0003F08AFB28480021042203F093FB26482C
:10AB0C000421002203F080FB23480421002203F0DF
:10AB1C0089FB21480821602203F092FB1E48082182
:10AB2C00012203F071FB00221B48082103F07AFB81
:10AB3C001A4B02221A7000222BE0174800214022E7
:10AB4C0003F07EFB14480021012203F05DFB124848
:10AB5C000021042203F066FB0F480421602203F05D
:10AB6C006FFB0D480421012203F04EFB0A4804211F
:10AB7C00002203F057FB08480821002203F044FB95
:10AB8C0000220548082103F04DFB0122034B1A70EB
:10AB9C00013A034B1A7008BD002C0140AD2900206E
:10ABAC00AC29002008B5034608460AB981F0070015
:10ABBC0013B9FFF759FE01E0FFF7D4FE08BD00BF43
:10ABCC0037B501AD1A23002428468DF804308DF8D2
:10ABDC00074004F071F9284619238DF804308DF8DC
:10ABEC00074004F069F9024803F024FD3EBD00BFA4
:10ABFC00002C0140F0B58F4B8FB01C780546012C12
:10AC0C0007D12146402004F089F821464FF400601A
:10AC1C0002E040F60C00012104F080F8864803F0B5
:10AC2C0009FD08A803F0FCF84FF00002ADF8202055
:10AC3C0045B940F60F63ADF82250ADF82430ADF8AD
:10AC4C0026500BE04FF06002ADF822204FF4E16388
:10AC5C004FF48072ADF82430ADF8262076480023EE
:10AC6C0008A98DF8283002F083FF684603F0E2F85B
:10AC7C0025B9ADF80050ADF8065007E04FF0700361
:10AC8C0040F20552ADF80030ADF806204FF001034C
:10AC9C00ADF80230694B4FF004021B78ADF804207C
:10ACAC00012B0CD125B9ADF80850ADF80A500EE0C7
:10ACBC004FF00203ADF808304FF0080205E04FF0FA
:10ACCC000003ADF808304FF00202ADF80A204FF443
:10ACDC0080734FF4007258486946ADF80C30ADF8EB
:10ACEC000E2002F067FF5448694602F0ABFF0DAC32
:10ACFC006946514802F0F6FF204604F0A5FC4D4B86
:10AD0C001978012916D14E4804F0E4FC18238DF86B
:10AD1C003730032321468DF836304A484FF47C53A4
:10AD2C00ADF8343004F046FC46484FF4285104F09A
:10AD3C00B3FC15E01823444821468DF837304FF406
:10AD4C00E06203238DF83630ADF8342004F032FC89
:10AD5C004EF2000321463D48ADF8343004F02AFC95
:10AD6C00354C0021204603F095F92046002103F0D4
:10AD7C009BF92046002103F0A1F9354B4FF40062FA
:10AD8C001B884FF00006ADF816304FF4806304A911
:10AD9C002046ADF81020ADF812304FF400524FF4AD
:10ADAC008043ADF81C30ADF81A20ADF81460ADF846
:10ADBC00186003F01DF82046012103F077FA0121F9
:10ADCC000A46204603F072F80121204603F054F99C
:10ADDC004FF4A06004F066F801271A230BA88DF835
:10ADEC002C308DF82D708DF82E608DF82F7004F0AE
:10ADFC0063F819230CA88DF830308DF832608DF87B
:10AE0C0033708DF8317004F057F81DB9A58625877D
:10AE1C00A58704E04FF46172A2862287A2870121E4
:10AE2C00054803F025F80448012103F02FF80FB072
:10AE3C00F0BD00BF18020020002C0140460000208D
:10AE4C00C00016000018014000080140000C014031
:10AE5C0048000020024B1A6801321A60704700BF8C
:10AE6C00B42900200028B8BF404240438B6DC9690B
:10AE7C004FF0140C48430CFB03FC154B70B51A68CF
:10AE8C0044F620655C6890FBF5F5BCFBF1F06421A1
:10AE9C000132B0FBF1F02D1982421A605D6016DBB5
:10AEAC009A680C4C501C90FBF1FC01FB1C01DE68F9
:10AEBC0054F822004FF47A7CB5FBFCF5361A76195F
:10AECC000020586044F82250DE609960186070BD14
:10AEDC0004030020B8290020014BD868704700BF3C
:10AEEC0004030020014B1868704700BFB4290020F0
:10AEFC00014B1860704700BFB429002008B5054B02
:10AF0C001B7C012B05D1044B044918680422FEF765
:10AF1C0001FE08BD04030020B0290020B429002044
:10AF2C0008B5054B042218600449FEF771FC044B6C
:10AF3C0001221A7408BD00BFB0290020B4290020DA
:10AF4C0004030020014B1868704700BF502B0020F1
:10AF5C00014B1860704700BF502B002008B5074B01
:10AF6C001B78012B09D1064B064918680422FEF701
:10AF7C00D1FDFFF75FFB044B186008BD18030020E0
:10AF8C004C2B0020502B0020482B002038B50F4BA9
:10AF9C001B78012B18D1FFF74DFB0D4C4EF65F22A1
:10AFAC002368C31A002BB8BF5B4293420CDD094BDC
:10AFBC00094A1D6810680135194604221D60FEF708
:10AFCC00A9FDFFF737FB206038BD00BF1803002038
:10AFDC00482B0020502B00204C2B002008B5074B91
:10AFEC00042218600649FEF713FCFFF723FB054B00
:10AFFC0001221860044B1A7008BD00BF4C2B0020B6
:10B00C00502B0020482B002018030020014BB3F9D3
:10B01C00000070471C030020884203D0164B4FF0F1
:10B02C0000021A800138052822D8DFE800F0071743
:10B03C00030F0B13012916D0022912E0052912D097
:10B04C0003290EE004290ED001290AE006290AD0B2
:10B05C00052906E0022906D0042902E0032902D0C2
:10B06C00062905D101E0012003E04FF6FF7000E056
:10B07C00002000B2704700BF1C030020014B586039
:10B08C00704700BF1C030020014B5868704700BF7D
:10B09C001C03002000F13B03762B10B50D4B0BD994
:10B0AC0051430D4AB3F800C0800392FBF1F190FBC1
:10B0BC00F1F06044188002E04FF000021A80054C59
:10B0CC000649B4F9000042F6AA2201F077F9208073
:10B0DC0010BD00BF1C030020206CFBFF56D5FFFFEA
:10B0EC00012008B5FCF702FC0138C0B2052801D9D3
:10B0FC00002002E0024B33F8100000B208BD00BF84
:10B10C001807010810B50B4C00222068022102F030
:10B11C00CDFE20684FF448730385002103F012F92B
:10B12C002068012102F0A4FE20680221012202F015
:10B13C00BDFE10BD340000200C4B07B51B78012B55
:10B14C0001D11B3304E00A4B1B78012B02D11D33B8
:10B15C008DF80430002301A88DF8073003F0ACFE05
:10B16C00044B186803F066FA0EBD00BF38000020CF
:10B17C001902002034000020F0B5694B89B01C780E
:10B18C000546012C16D12046214603F0D5FD21465B
:10B19C00042006AC03F0C2FD204604F055FA03234C
:10B1AC008DF81A3001338DF81B3021465D484FF075
:10B1BC00070335E05C4B1E78012E35D10420314657
:10B1CC0003F0BAFD594B06AC1F78012F1AD1394642
:10B1DC00202003F0A3FD204604F036FA03238DF85B
:10B1EC001A30013321468DF81B3051484FF4E0439F
:10B1FC00ADF8183004F0DEF939464FF4805004F005
:10B20C0069FA11E03146082003F088FD204604F06D
:10B21C001BFA482347488DF81B3021464FF4E07346
:10B22C00ADF8183004F0C6F9434C03AE206803F0B7
:10B23C0001FA304602F0F4FD4FF0FF33314620683E
:10B24C00ADF810304FF00003ADF8123002F090FC66
:10B25C00684602F0F9FD4FF00003ADF800304FF0F6
:10B26C000203ADF802304FF00B0369462068ADF8CD
:10B27C0008304FF00303ADF8043003F077F90122E6
:10B28C004FF44871206802F05FFE206802F02CFE3B
:10B29C000121206803F018F84021206802F062FEBA
:10B2AC000421206803F036F80121206802F0FEFF2B
:10B2BC00012D6E4628D11A4B1B78012B01D11B3363
:10B2CC0004E0194B1B78012B02D11D338DF81C3077
:10B2DC00194C01250023022607A88DF81E308DF885
:10B2EC001D608DF81F5003F0E7FD206841F65F618B
:10B2FC0003F092F8314620682A4602F0D7FD294621
:10B30C0020682A4602F0D2FD0B4C0021206803F085
:10B31C0019F82068012102F0ABFD09B0F0BD00BFA7
:10B32C0038000020000801401902002018020020FB
:10B33C0000140140000C014034000020014B188027
:10B34C00704700BF582B0020014B1860704700BF9E
:10B35C00542B002010B504460846FFF7EFFF20469B
:10B36C00FFF7F2FF10BD00BF014B1878704700BF0C
:10B37C0024030020014B00221A7070472403002084
:10B38C00014B1870704700BF8C010020014B1878DE
:10B39C00704700BF8C010020704700BF034B1B7827
:10B3AC001BB9034B80B21B689884704722020020A3
:10B3BC003C000020014B5860704700BF2403002064
:10B3CC00014B5868704700BF240300200549064B09
:10B3DC004A8909891B688A18B2FBF3F103FB112314
:10B3EC0098B2704724030020542B0020014B188185
:10B3FC00704700BF2403002008B50520002101225E
:10B40C0000F06CFB054B80111B7B1BB1044B1B68C4
:10B41C00013B181A014B588108BD00BF24030020C2
:10B42C00542B002008B5044B01461B781BB9034B69
:10B43C00186802F087FF08BD220200203C000020A3
:10B44C0008B5054B1B7823B9044B186802F0D6FFDE
:10B45C0001E0034B588908BD220200203C0000206B
:10B46C002403002008B50E4B1B7823B90D4B18682C
:10B47C0002F0C4FF09E00C4B5A8918890B4B801859
:10B48C001B68B0FBF3F203FB1200084BC0EB00404F
:10B49C001A68074BB0FBF2F01B88584380B208BD0A
:10B4AC00220200203C00002024030020542B00200A
:10B4BC00582B002007B5184B1B78012B2AD0174BA3
:10B4CC001B78012B04D107338DF80430143310E0B2
:10B4DC00134B1B78012B04D116338DF80430063333
:10B4EC0007E0104B1B78012B14D116338DF8043068
:10B4FC0007338DF8003001A800238DF803308DF848
:10B50C00073003F0D9FC684603F0D6FC064B1868EC
:10B51C0003F090F80EBD00BF220200201A0200209A
:10B52C00400000201B0200203C000020F0B58A4B9C
:10B53C008A4A1B788BB0012B0D461173074600F01D
:10B54C000881874B1C78012C18D12046214603F02A
:10B55C00F3FB2146042008AC03F0E0FB204604F08A
:10B56C0073F848238DF8233021464FF007037D48AC
:10B57C00ADF8203004F01EF81C233CE07A4B1C780C
:10B58C00012C1CD10220214603F0D6FB08AE21462B
:10B59C00102003F0C3FB304604F056F84823314624
:10B5AC0072488DF823304FF4E073ADF8203004F07E
:10B5BC0001F821466E4804F08DF81D231BE06D4BFD
:10B5CC001C78012C19D12146042003F0B5FB21462F
:10B5DC00082008AC03F0A2FB204604F035F8482301
:10B5EC008DF8233021464FF4E0736348ADF82030DA
:10B5FC0003F0E0FF1E238DF824300223002409A859
:10B60C008DF82530013B8DF827308DF8264003F05E
:10B61C0053FC5A4B013F186803F00CF803A802F0D6
:10B62C00FFFB012D18BFADF80E40ADF80C40ADF886
:10B63C001240524C08BF102303A9206808BFADF874
:10B64C000E30ADF8107002F093FA012D01D10022EA
:10B65C0000E0022203211346206802F097FC6846A2
:10B66C0002F0F2FB454B694618684FF00803ADF841
:10B67C00083002F07BFF3A4B1B78012B02D14FF0C4
:10B68C0004030CE0384B1B78012B02D14FF008035C
:10B69C0005E0384B1B78012B03D14FF00C03ADF8B0
:10B6AC000030364C6946206802F060FF01212068AA
:10B6BC0002F0B2FE01210A46206802F0F7FB206876
:10B6CC004FF000030121838402F0D2FB244B1B7842
:10B6DC00012B05D10020022104F02AF804230EE0EE
:10B6EC00214B1B78012B01D1022003E0214B187850
:10B6FC00012805D1082104F01BF84FF48073069340
:10B70C00002308248DF81C3006A801338DF81E3058
:10B71C008DF81D4004F0B4F8114B1B78012B02D1AD
:10B72C008DF824400AE0104B1B78012B03D0114BF1
:10B73C001B78012B02D116338DF824300023012203
:10B74C0009A88DF826308DF827208DF8253003F0C8
:10B75C00B3FB0BB0F0BD00BF22020020240300207D
:10B76C001A02002000080140400000200010014097
:10B77C00000C1A001B020020000C01403C000020B1
:10B78C00B0F90030B0F9022003FB03F102FB021107
:10B79C0010B50C4CA14214D94FEA116CACF13A0C17
:10B7AC0009495FFA8CFC31F81CC04FF4004102FBD4
:10B7BC000CF203FB0CF392FBF1F293FBF1F14280E0
:10B7CC00018010BD0044FA3A24070108124B37B52A
:10B7DC00B3F902C0B3F90010B0F90220B0F90000BF
:10B7EC0002FB0CF400FB01F500FB0CFC4A434FF48C
:10B7FC00004395FBF3F194FBF3F492FBF3F2641822
:10B80C009CFBF3F3D31A0020A2B262F30F009BB29D
:10B81C0063F31F403EBD00BF34030020A0F5004081
:10B82C00C0F3891000F44073B3F5807F82B037D039
:10B83C0001DC23B305E0B3F5007F05D0B3F5407F01
:10B84C000FD00023184639E0C0B21E4B420082F4E0
:10B85C00FF7203EB4000D218B0F88C00B2F88C30B9
:10B86C002CE0184AC0B202EB4003400080F4FF7099
:10B87C00B3F88C3082185B42B2F88C000EE0114B9E
:10B88C00C0B2420082F4FF7203EB4000D218B0F851
:10B89C008C00B2F88C3040425B4280B29BB20DE01F
:10B8AC00C0B2084B420082F4FF72D218B2F88C205E
:10B8BC0003EB40035242B3F88C3090B243EA0040A1
:10B8CC0002B070472407010830B5044685B008461D
:10B8DC00FFF7A4FFC0F30F43ADF80230ADF8000042
:10B8EC00134A00994FF400431160B4F90210B2F9F5
:10B8FC000200B4F900C0B2F9002001FB00F50CFB0A
:10B90C0002F40CFB00F04A4394FBF3F495FBF3F1C7
:10B91C0092FBF3F2641A90FBF3F3D3180020A2B25B
:10B92C0062F30F009BB263F31F4005B030BD00BF44
:10B93C0034030020032903D8DFE801F004081014B5
:10B94C00002018E00D4B03EB400004E040000B4BD3
:10B95C0080F4FF70C018B0F88C000CE0074B03EBC0
:10B96C00400004E04000054B80F4FF70C018B0F8B4
:10B97C008C00404280B200B2704700BF240701081F
:10B98C0083B244F6E61100140FFA83FC484301FB22
:10B99C000CF14FF4004291FBF2F190FBF2F290B2F9
:10B9AC004A42A2EB4002002063F30F0092B284B033
:10B9BC0062F31F4004B0704730B585B06B4683E826
:10B9CC000300BDF90410BDF9020040F2C46202FB91
:10B9DC0001F402FB00FCBDF900506FF0020290FB79
:10B9EC00F2F003236D0091FBF2F1091895FBF3F5CE
:10B9FC0040F6B8339CFBF3FC4A1994FBF3F3CCEB05
:10BA0C00030392B2002062F30F009BB263F31F405A
:10BA1C0005B030BD30B52E4B87B01B780546012BD9
:10BA2C0003D1012801D12B4C00E02B4C20460021E6
:10BA3C0002F0ECFE4FF00003ADF804304FF48273CB
:10BA4C00ADF806304FF00003ADF808304FF00203AC
:10BA5C00ADF80A304FF00103ADF80C304FF4007321
:10BA6C00ADF80E304FF00003ADF81230ADF81430D5
:10BA7C00052D1ED8DFE805F00306061D09104FF052
:10BA8C00100318E04FF0080315E04FF40063ADF815
:10BA9C0008304FF0100305E04FF40063ADF80830A8
:10BAAC004FF02803ADF810304FF00003ADF80A301A
:10BABC0003E04FF01803ADF8103001A9204602F056
:10BACC0069FE2046012102F0A1FE07B030BD00BF87
:10BADC001F0200200038004000300140F8B51D4D19
:10BAEC0004462B780E468342174602D0FFF792FF8E
:10BAFC002C70042C05D0052C06D04CBBFBF742FE59
:10BB0C0004E0FBF77DFE01E0FBF77EFE124802210C
:10BB1C0002F010FF0028F9D031460F4802F0AEFEBB
:10BB2C000D48012102F006FF0028F9D067B1042C62
:10BB3C0005D0052C06D05CB9FBF72AFE04E0FBF718
:10BB4C0061FE01E0FBF762FE034802F099FE00E0A3
:10BB5C000020F8BD3803002000300140F8B52D4D11
:10BB6C0004462B780E468342174602D0FFF752FF4D
:10BB7C002C70052C4CD8DFE804F00306090C0F12CE
:10BB8C00FBF700FE0DE0FBF72FFE0AE0FBF730FEA3
:10BB9C0007E0FBF731FE04E0FBF732FE01E0FBF7B8
:10BBAC0033FE1D4B1B78012B03D1012C01D11B4DF6
:10BBBC0000E01B4D2846022102F0BCFE0028F9D003
:10BBCC003146284602F05AFE2846012102F0B2FE08
:10BBDC000028F9D0BFB1052C1AD8DFE804F0030611
:10BBEC00090C0F12FBF7D4FD0DE0FBF7FFFD0AE08B
:10BBFC00FBF700FE07E0FBF701FE04E0FBF702FE9B
:10BC0C0001E0FBF703FE284602F03AFEC0B200E06A
:10BC1C000020F8BD380300201F020020003800402F
:10BC2C00003001402DE9F041012186B04FF48050E5
:10BC3C0003F074F80120014605AF03F06FF81824E7
:10BC4C0003264FF0A00348483946ADF814308DF860
:10BC5C0016608DF8174003F0ADFC4FF040034248DE
:10BC6C003946ADF814308DF816608DF8174003F096
:10BC7C00A1FC0120002103F02DFD4FF00003ADF8D5
:10BC8C0000304FF48273ADF802304FF00003ADF882
:10BC9C0004304FF00203ADF806304FF00103ADF85D
:10BCAC0008304FF4007331486946ADF80A304FF054
:10BCBC000003ADF80E30ADF81030ADF80C4002F0CA
:10BCCC0069FD0121294802F0A1FD294BE8461D78A8
:10BCDC00012D42D14FF48040294603F02DF84AF251
:10BCEC00000324483946ADF814308DF816608DF8F1
:10BCFC00174003F05FFC4FF4804339461D48ADF804
:10BD0C0014308DF816608DF8174003F053FC4FF08B
:10BD1C000003ADF800304FF48273ADF802304FF0F1
:10BD2C000003ADF804304FF00203ADF806304FF4C9
:10BD3C00007369461048ADF80A304FF00003ADF8B7
:10BD4C000C40ADF80850ADF80E30ADF8103002F0E4
:10BD5C0021FD2946084802F059FD084B4FF0FF32EF
:10BD6C001A7006B0BDE8F0810008014000300140B7
:10BD7C001F020020000C0140003800403803002056
:10BD8C0082B000211C4A0191938A9BB20193019BC2
:10BD9C0013F4806F06D0938A23F480631B041B0C6E
:10BDAC0093820191019B13F4007F08D0124A938A6D
:10BDBC0023F480631B041B0C938200230193019BCF
:10BDCC0013F4807F08D00C4A938A23F480731B04ED
:10BDDC001B0C938200230193019B13F4006F08D07A
:10BDEC00054A938A23F400631B041B0C93820023E3
:10BDFC00019302B0704700BF0054004082B0002194
:10BE0C001C4A0191938A9BB20193019B13F4806F9E
:10BE1C0006D0938A23F480631B041B0C938201913C
:10BE2C00019B13F4007F08D0124A938A23F4806399
:10BE3C001B041B0C938200230193019B13F4807F42
:10BE4C0008D00C4A938A23F480731B041B0C938236
:10BE5C0000230193019B13F4006F08D0054A938AC9
:10BE6C0023F400631B041B0C93820023019302B088
:10BE7C00704700BF0058004038B50D461F4C19469E
:10BE8C00E3B91033A3601E4B65609842E2600AD19F
:10BE9C0010331C48236003F0FFFD1A48214603F0C1
:10BEAC00CBFD184826E0184B1848236003F0F4FD2E
:10BEBC001648214603F0C0FD14481BE0104B00212E
:10BECC0098426560E260A1600AD11033104823608B
:10BEDC0003F0E2FD0E48214603F0AEFD0C4809E0EC
:10BEEC00094B0C48236003F0D7FD0A48214603F0A8
:10BEFC00A3FD0848012103F0CFFD38BD5C2B0020C9
:10BF0C00005400406C0002401058004044000240B5
:10BF1C00800002405800024073B50026019600963E
:10BF2C00B0F804C004461FFA8CFC4CF4807CA0F8DA
:10BF3C0004C01D4633464FF6FF760096FFF79CFF74
:10BF4C00A3889BB243F40063A38023889BB243F481
:10BF5C008073238004E0009B5A1E0092002B46D075
:10BF6C00A38A13F0010FF6D0224B05F0FE054FF615
:10BF7C00FF7200921D701B78238204E0009B5A1EF6
:10BF8C000092002B33D0A38A13F0020FF6D0238B30
:10BF9C009BB20193184B9C420CD14FF4001003F050
:10BFAC0093FD0028F9D01548002103F075FD4FF4DE
:10BFBC0000100BE04FF4005003F086FD0028F9D080
:10BFCC000F48002103F068FD4FF4005003F08CFD86
:10BFDC00A38A13F0040FFBD023889BB243F40073A5
:10BFEC002380238813F4007FFBD1012000E0002084
:10BFFC007CBD00BF882B0020005400406C00024028
:10C00C004400024037B5002401940094B0F804C0F9
:10C01C0004461FFA8CFC4CF4807C1D46A0F804C02E
:10C02C000123FFF729FFA3889BB243F48053A3801D
:10C03C00A3889BB243F40063A3804FF6FF73009375
:10C04C0023889BB243F48073238004E0009B5A1E28
:10C05C000092002B42D0A38A13F0010FF6D0204B94
:10C06C0045F001054FF6FF7200921D701B7823827C
:10C07C0004E0009B5A1E0092002B2FD0A38A13F0D1
:10C08C00020FF6D0238B9BB20193164B9C420CD122
:10C09C004FF0007003F018FD0028F9D01248002171
:10C0AC0003F0FAFC4FF000700BE04FF4003003F09B
:10C0BC000BFD0028F9D00D48002103F0EDFC4FF4E6
:10C0CC00003003F011FD23889BB243F400732380EE
:10C0DC00238813F4007FFBD1012000E000203EBD3B
:10C0EC00882B002000540040800002405800024081
:10C0FC0070B5012186B00646082002F00FFE012023
:10C10C00014602F0FDFD644B05AC9E4204AD28D106
:10C11C004FF40010012102F00FFE03238DF81630AE
:10C12C00193321465D488DF817304FF04003ADF8B8
:10C13C00143003F03FFA4FF0800321465748ADF816
:10C14C00143003F037FA4FF40010012102F010FE06
:10C15C004FF40010002102F00BFE28460123202290
:10C16C0027E04FF48000012102F0E6FD03238DF857
:10C17C0016301933494821468DF817304FF4806337
:10C18C00ADF8143003F016FA4FF40063214643481F
:10C19C00ADF8143003F00EFA4FF48000012102F0D8
:10C1AC00E7FD4FF48000002102F0E2FD2846012358
:10C1BC0022228DF8102006228DF813308DF81230C3
:10C1CC008DF8112002F078FE334B00259E4244F688
:10C1DC00206303934BF6FF73ADF802304FF480638A
:10C1EC00ADF806304FF48043ADF80050ADF8083090
:10C1FC0069462B4C25D14FF028033046ADF804305E
:10C20C0003F04CF9274803F0A7FB274B214623608A
:10C21C001023A3604FF6FF73E3608023636103F583
:10C22C003E5320486362A56265602561A561E561A6
:10C23C00256203F001FC1D4803F08EFB21461B48D0
:10C24C0025E04FF0300369461948ADF8043003F08F
:10C25C0025F9184803F080FB174B21462360102367
:10C26C00A3604FF6FF73E3608023636103F53E53D5
:10C27C0010486362A56265602561A561E561256270
:10C28C0003F0DAFB0D4803F067FB0C48214603F082
:10C29C00D3FB06B070BD00BF00540040000C014041
:10C2AC005C2B00206C0002401054004080000240C7
:10C2BC000058004044000240105800405800024012
:10C2CC0008B5FFF715FF08BD03464FF6FF70834214
:10C2DC0046DDB3F1807F23DBB3F1805F0FDBB3F17D
:10C2EC00804F07DB334A934263DC33491A168A5C6E
:10C2FC0012020FE030499A158A5CD2010AE0B3F1C0
:10C30C00806F2D4A03DB1915525C920102E09914DF
:10C31C00525C520193FBF2F101325218521019E0A7
:10C32C00B3F5801F0BDBB3F5800F234A03DB191425
:10C33C00525C12010EE09913525CD2000AE0B3F584
:10C34C00802F1D4A03DB1913525C920002E09912F4
:10C35C00525C520093FBF2F1501C401840101BE051
:10C36C00FF2B1FDDB3F5805F0ADBB3F5804F124A5C
:10C37C0002DB1912505C0EE09911505C40080AE087
:10C38C00B3F5806F0C4A03DB1911505C800802E096
:10C39C009910505CC008013000FB00F29A4208DD95
:10C3AC00013806E0002BA9BF034A4FF0FF30D05CE8
:10C3BC00000970470080FE7FB0090108904203DC41
:10C3CC008142ACBF0A4602461046704770B504461F
:10C3DC0010460E4603F0FEFE05462946204604F0A4
:10C3EC0009F940B9304603F0F5FE054629462046CA
:10C3FC0004F0E2F800B12C46204670BD70B514462E
:10C40C000E4603F0E7FE0546204603F0DFFE044629
:10C41C002146284603F0E6FF0146284603F024FE99
:10C42C000546304603F0D6FE214603F0DBFF0146FD
:10C43C00284603F01BFE04F0E7F870BD70B51BB185
:10C44C002D2301F8013B40424B1CB0FBF2F402FBE4
:10C45C00140C5D1EBCF1090F8CBF0CF1570C0CF1C8
:10C46C00300C03F801CC1E4620460133002CECD1D5
:10C47C0034702B780A7805F8012901F8013BA942A0
:10C48C00F7D3304670BD00BF0A2A08B58446134660
:10C49C008E4603D1002801DA012303E01A466046D8
:10C4AC0071460023FFF7CAFF08BD00BF642303FBDE
:10C4BC0000F292FBF1F29A420BDD47F6122359433C
:10C4CC006FF00303584391FBF0F000F574505C30AF
:10C4DC0019E012F1640F0BDA47F6122359436FF08F
:10C4EC000303584391FBF0F0A0F574505C380AE05C
:10C4FC001C224B43424393FBF0F092FBF1F1024BB5
:10C50C00401893FBF0F0704700410F00002908B56C
:10C51C0002DDFFF7CBFF14E006D1002811D0D4BF09
:10C52C00084843F65C500CE0002805DBFFF7BEFF23
:10C53C0000F5F440B83004E0FFF7B8FFA0F5F44084
:10C54C00B83808BDA4C2FFFF014B1860704700BF8C
:10C55C00405C0040014B186880B27047405C004062
:10C56C00014B1860704700BF445C0040014B1868D9
:10C57C0080B27047445C0040014B186880B2704731
:10C58C00485C0040014B1860704700BF4C5C004099
:10C59C00014B186880B270474C5C00404FF6F87342
:10C5AC00024A00EA03031360704700BF505C00406E
:10C5BC00014B186880B27047505C0040014B43F847
:10C5CC0020107047005C0040024B53F8200080B2F2
:10C5DC00704700BF005C0040054B10B553F820407D
:10C5EC0048F68F1204EA02020A4343F8202010BDD9
:10C5FC00005C0040024B53F8200000F4C060704710
:10C60C00005C00400A4B10B553F8202048F6BF746C
:10C61C0002EA040411F0100F18BF84F0100411F09A
:10C62C00200F18BF84F0200443F8204010BD00BF39
:10C63C00005C00400A4B10B553F820204BF68F7469
:10C64C0002EA040411F4805F18BF84F4805411F4DE
:10C65C00005F18BF84F4005443F8204010BD00BFA5
:10C66C00005C004038B50D460446FFF7ADFF012DC8
:10C67C0002D120F4805003E0022D04D120F01000F0
:10C68C00014B43F8240038BD005C0040024B53F8CA
:10C69C00200000F030007047005C0040024B53F863
:10C6AC00200000F440507047005C0040054B48F6F9
:10C6BC00BF7253F8201001EA020282F0300243F8F4
:10C6CC0020207047005C0040054B4BF68F7253F8EE
:10C6DC00201001EA020282F4405243F820207047F5
:10C6EC00005C0040054B48F68F6253F8201001EABD
:10C6FC00020242F4807243F820207047005C004034
:10C70C00044B48F68F6253F8201001EA020243F8FA
:10C71C0020207047005C0040044B48F68F6253F8B1
:10C72C00201001EA020243F820207047005C004010
:10C73C00054B48F68F6253F8201001EA020242F4CE
:10C74C00807243F820207047005C0040054B48F68F
:10C75C008F6253F8201001EA020242F4807243F80F
:10C76C0020207047005C0040044B48F68F6253F861
:10C77C00201001EA020243F820207047005C0040C0
:10C78C00044B53F8200000F03000102814BF002098
:10C79C0001207047005C0040054B53F8200000F46A
:10C7AC004050B0F5805F14BF00200120704700BFDF
:10C7BC00005C0040044B40F68F7253F8201001EAE5
:10C7CC00020243F820207047005C0040044B48F6FE
:10C7DC000F7253F8201001EA020243F82020704730
:10C7EC00005C0040054B48F68F7253F8201001EAAC
:10C7FC00020242F4804243F820207047005C004063
:10C80C00054B48F68F7253F8201001EA020242F0F1
:10C81C00400243F820207047005C0040084B53F85E
:10C82C00202012F4804F09D053F8201048F68F7254
:10C83C0001EA020242F4804243F82020704700BF14
:10C84C00005C0040084B53F8202012F0400F09D038
:10C85C0053F8201048F68F7201EA020242F04002AF
:10C86C0043F82020704700BF005C0040054B10B51A
:10C87C0053F8204048F68F7204EA02020A4343F848
:10C88C00202010BD005C0040024B53F8200000F04B
:10C89C000F007047005C0040064B49081B684900BC
:10C8AC009BB203EBC00303F1005303F540535B0051
:10C8BC0019607047505C0040054A064B12684908E5
:10C8CC0092B202EBC002D3185B00490019607047AA
:10C8DC00505C004004300020054B1B689BB203EBFE
:10C8EC00C00303F1005303F540535B0018887047F5
:10C8FC00505C0040044A054B126892B202EBC00235
:10C90C00D3185B0018887047505C0040043000203E
:10C91C00044A054B126892B202EBC002D3185B00BA
:10C92C0019607047505C0040023000203E2909D944
:10C93C004B0911F01F0F01D1013B9BB29B0243F439
:10C94C00004305E04B0811F0010F18BF01339B02A7
:10C95C00036070470D4A0E4B126892B2D31803EB6A
:10C96C00C0035B003E2909D94A0911F01F0F01D100
:10C97C00013A92B2920242F4004205E04A0811F0E8
:10C98C00010F18BF013292021A607047505C0040D0
:10C99C0006300020054A064B126892B202EBC00228
:10C9AC00D3185B0018688005800D7047505C004000
:10C9BC0002300020054A064B126892B202EBC0020C
:10C9CC00D3185B0018688005800D7047505C0040E0
:10C9DC00063000200C4B30B51D681C68C0001FFAD7
:10C9EC0085FC8444A4B2094B00190CF1005CC318FB
:10C9FC000CF5405C490852084FEA4C0049005B00BA
:10CA0C00520001601A6030BD505C004004300020C0
:10CA1C00064B49081B6849009BB203EBC00303F1AA
:10CA2C00005303F540535B0019607047505C0040A5
:10CA3C00054A064B1268490892B202EBC002D318A1
:10CA4C005B00490019607047505C004004300020C6
:10CA5C00054B1B689BB203EBC00303F1005303F5BA
:10CA6C0040535B0018887047505C0040044A054BEB
:10CA7C00126892B202EBC002D3185B0018887047A0
:10CA8C00505C004004300020012910B524D1254B06
:10CA9C0025491B68C0009BB2591809184B003E2A47
:10CAAC0009D9510912F01F0F01D1013989B289023C
:10CABC0041F4004105E0510812F0010F18BF01319B
:10CACC00890219601749194B096889B2CB181818D3
:10CADC0040003E2A1ED913E0022922D1114BC0007E
:10CAEC001C681B68A4B21FFA83FC0F490F4B8444CB
:10CAFC0000194118634449005B000A601A6010E099
:10CB0C00530912F01F0F01D1013B9BB29B0243F45E
:10CB1C00004305E0530812F0010F18BF01339B02CC
:10CB2C00036010BD505C0040023000200630002035
:10CB3C0001291BD11349144B096889B2CB1803EB9B
:10CB4C00C00040003E2A09D9530912F01F0F01D131
:10CB5C00013B9BB29B0243F4004305E0530812F0E7
:10CB6C00010F18BF01339B0203600AE0022908D1B0
:10CB7C000449054B096889B201EBC000C3185B007E
:10CB8C001A607047505C00400230002001291BD114
:10CB9C001349144B096889B2CB1803EBC000400051
:10CBAC003E2A09D9530912F01F0F01D1013B9BB248
:10CBBC009B0243F4004305E0530812F0010F18BF29
:10CBCC0001339B0203600AE0022908D10449054B9A
:10CBDC00096889B201EBC000C3185B001A6070478A
:10CBEC00505C004006300020054A064B126892B299
:10CBFC0002EBC002D3185B0018688005800D7047EB
:10CC0C00505C004002300020054A064B126892B27C
:10CC1C0002EBC002D3185B0018688005800D7047CA
:10CC2C00505C0040063000200D4BC00019680D4AC6
:10CC3C0089B241188A185200128812F47C4F01D024
:10CC4C0001200CE01A68084B92B28018C3185B00E4
:10CC5C0018888005800D002814BF02200020704722
:10CC6C00505C00400630002002300020012909D120
:10CC7C000B4A48F68F7352F8201001EA030343F075
:10CC8C0040030AE002290AD1054A48F68F7352F88C
:10CC9C00201001EA030343F4804342F8203070472C
:10CCAC00005C004041EA0020704700BF030AC0B29C
:10CCBC0043EA0020704700BF01F10051013201F539
:10CCCC00405110B549005208002308E010F803C089
:10CCDC006478013A4CEA042C21F813C00233C418CE
:10CCEC00002AF3D110BD00BF01F10051013201F552
:10CCFC00405110B549005208002304E031F81340AC
:10CD0C00013AC4520233002AF8D110BD08B529E00B
:10CD1C0047F6FF700860198801F00F018B0003F1D2
:10CD2C008043117003F5B843196889B211F4004FB0
:10CD3C0009D0186840F68F7100EA01011960127869
:10CD4C000E4B013A0BE011F0800F0BD0186848F62F
:10CD5C000F7100EA010119601278094B013A53F87E
:10CD6C00223098470749084B0868084A80B2188057
:10CD7C00188800B20028CBDB08BD00BF40010020A2
:10CD8C0024010020445C0040860900208E0900200C
:10CD9C00F8B59AE047F6FF761E601688564F06F0F7
:10CDAC000F06B30003F1804303F5B8433E70002E29
:10CDBC0064D127682668236807F4405C03EA000006
:10CDCC0080F400502060236806F0300003EA010173
:10CDDC0081F0200121601388484A13F0100F108055
:10CDEC00A5F800C004D023689BB213F0800F08D0C4
:10CDFC00226848F60F7302EA0303236000F0CEFAB0
:10CE0C0016E013F4006F08D0226840F68F7302EA24
:10CE1C000303236000F062FB0AE013F4004F54D0CC
:10CE2C00226840F68F7302EA0303236000F0F8F9DE
:10CE3C0021682A884BF68F7301EA030312F4805F92
:10CE4C0018BF83F4805312F4005F2D4A18BF83F48B
:10CE5C0000531360294B11681A8848F6BF7301EA16
:10CE6C00030312F0100F18BF83F0100312F0200F01
:10CE7C00234A18BF83F0200313603BE01C68A4B264
:10CE8C0014F4004F0BD0196840F68F7201EA0202BD
:10CE9C001A603A781B4B013A53F82230984714F039
:10CEAC00800F12D0144948F60F720B789B0003F1D7
:10CEBC00804303F5B843186800EA02021A600A7846
:10CECC00114B013A53F822309847104B104A1D6809
:10CEDC000B4C1FFA85FCA2F800C0B2F800C04BF650
:10CEEC008F700FFA8CFCBCF1000F48F6BF71094D26
:10CEFC00FFF650AFF8BD00BF8E0900208C2B002030
:10CF0C00005C00404001002024010020445C0040F3
:10CF1C00860900208A2B0020074A022108B5074801
:10CF2C0011720749074B086007490A60074A1360EA
:10CF3C001B68984708BD00BF9409002060010020C1
:10CF4C00B009002090000020F4090020880900207E
:10CF5C0010B5074C20B922684FF00103138205E08D
:10CF6C00044B1B681B68984720680A3010BD00BF33
:10CF7C00F4090020B009002010B50A4B0A4A1B68BE
:10CF8C005178DA7891420AD3997841B99C8834B9AE
:10CF9C009A72064B1B685B689847204600E002209B
:10CFAC0010BD00BFF40900205C010020B009002076
:10CFBC0010B5074C20B922684FF00103138205E02D
:10CFCC00044B1B689B68984720680C3010BD00BF51
:10CFDC00F4090020B009002038B50E4C0E4B226825
:10CFEC001B68D1789B695079984723689A7A7AB1F3
:10CFFC0070B91A7962B99D7855B9084B1B68DB6812
:10D00C009847236828465979DA78D9721A7300E060
:10D01C00022038BDF409002088090020B009002046
:10D02C0008B50246244B20B91B684FF00201198247
:10D03C0040E0224A4FF000011B681180197811F072
:10D04C007F0113D15B7A13F0200F03D0117841F0DC
:10D05C000201117013F0400F184B15BF1A781A7893
:10D06C0022F0010242F001021A701EE0012921D0C7
:10D07C00022901D000221DE0597911F0800F01F036
:10D08C000F0306D00E4951F8233003F03003102B58
:10D09C0006E00B4951F8233003F44053B3F5805F9D
:10D0AC0003D1137843F001031370064B1B681B6903
:10D0BC009847024A104608BDF4090020902B002026
:10D0CC00005C0040B009002010B51E4B19684A796D
:10D0DC0012F0800F22F0800305D01B4850F823007B
:10D0EC0000F0300004E0184850F8230000F44050E1
:10D0FC00164C94F800C0634522D24C8804BBF8B19E
:10D10C00897AE9B112F0800F09D00F4948F6BF7245
:10D11C0051F8230000EA020282F0100208E00A49EA
:10D12C004BF68F7251F8230000EA020282F480520F
:10D13C0041F82320064B1B689B699847002000E0B0
:10D14C00022010BDF4090020005C00405C010020AE
:10D15C00B009002008B5064B1B685A7A42F0200231
:10D16C005A72044B1B68DB699847002008BD00BF4E
:10D17C00F4090020B0090020054B1A68538A18B92D
:10D18C008988CB1A138201E008681818704700BF11
:10D19C00F409002030B50E4B1C78002310E05FFA28
:10D1AC0083FC4FEA8C0202F1804202F5B84215680A
:10D1BC0048F68F7105EA010141EA0C011160013357
:10D1CC00A342ECD3034B40F08000186030BD00BF8D
:10D1DC005C0100204C5C0040704700BF08B50C4B54
:10D1EC00002093F82C10FFF7B5FB0A4B1B68187A3C
:10D1FC00082807D1084B4FF480521A80074B4FF088
:10D20C0010021A80092814BF0020012008BD00BF9D
:10D21C0090000020F40900208A2B00208C2B002089
:10D22C0070B52D4B1C68237A032B01D0052B46D1EE
:10D23C00A369228AABB1A2B1A58A954228BF154633
:10D24C0028469847228A638A521BEB18064622828C
:10D25C0063820020FFF74EFB2A4601463046FFF75B
:10D26C0043FD238A5BB11D4B4FF4405200201A80C2
:10D27C000146FFF74DFB1A4B4FF030021A80A28A81
:10D28C00238A9A4203D8144B03221B6803E0124AE8
:10D29C001BB1136805221A720DE012680621117277
:10D2AC00104A1168104A89B28A18520013600C4B4C
:10D2BC004FF030021A80084B1B681B7A06E0072BD4
:10D2CC0003D10A4B1B68DB6898470823024A126893
:10D2DC001372FFF783FF70BDF40900208A2B002026
:10D2EC008C2B0020505C004002300020880900206C
:10D2FC00F8B5244B1C68238A267ABBB9042E15D1A9
:10D30C00214822490278012A0BD1214C214A246858
:10D31C000370A0B28218520013604FF030020A80E2
:10D32C002BE04FF010030B80072626E0A68AA2699B
:10D33C009E4234BF35461D462846B34294BF042650
:10D34C000226904707460020FFF7C6FA2A460146F8
:10D35C003846FFF7B1FC29460020FFF7D9FA638A5B
:10D36C00228AEB186382094B551B4FF03002258241
:10D37C001A80094B4FF440521A80024B1B681E72E4
:10D38C00F8BD00BFF4090020390300208C2B0020CD
:10D39C00505C0040023000208A2B002008B5144B52
:10D3AC001B681A7A022A01D0042A05D1FFF7A0FFC4
:10D3BC000F4B1B681B7A14E0062A11D15A78052AE8
:10D3CC000AD11A7812F07F0F06D1D878FFF7E2FE57
:10D3DC00084B1B681B6A9847074B1B689B68984750
:10D3EC000823034A12681372FFF7F8FE08BD00BF4A
:10D3FC00F4090020B00900208809002038B5324B10
:10D40C001B68187810F07F0004D15A7A22F02002A1
:10D41C005A7258E0022855D15A88002A52D11A79EA
:10D42C00002A4FD15A7912F0800F22F0800405D0D7
:10D43C00264951F8241001F0300104E0234951F839
:10D44C00241001F440512248007884423AD2002939
:10D45C0038D09B7A002B35D012F0800F0FD01B4B9D
:10D46C0053F8243003F03003102B25D1E4B22046BE
:10D47C00FFF7E8F920463021FFF7C4F81CE0134D04
:10D48C0055F8243003F44053B3F5805F14D134B90C
:10D49C00104B204693F82C10FFF75CFA02E0204664
:10D4AC00FFF7BCF955F824204BF68F7302EA0303FF
:10D4BC0083F4405345F82430074B1B685B6998474D
:10D4CC00002000E0022038BDF4090020005C004080
:10D4DC005C01002090000020B0090020F7B58D4BB6
:10D4EC008D4E1A6835688D4B92B2D3182A7A5B0030
:10D4FC00092A1B681BD09BB203F1005303F5405360
:10D50C005B001C4614F8012B03F10A072A705B78A8
:10D51C006B70B4F80300FFF7C9FB6880B4F8070020
:10D52C003468FFF7C3FBA08033687F88DF807A4CB8
:10D53C0001212368DA8819725D78002A62D11A7881
:10D54C0012F07F022ED1092D02D1FFF715FD3BE021
:10D55C00052D0DD193F90320002A4EDB9A78002A71
:10D56C004BD19A88002A48D19B7A002B37D044E0C3
:10D57C00032D0BD1DA78012A27D19A882ABB5B7A42
:10D58C0013F0200F21D0FFF7E5FD1DE0012D1CD17C
:10D59C00DA78012A19D19A88BAB95B7A13F0200F7C
:10D5AC0013D00AE0012A04D10B2D0ED1FFF714FD84
:10D5BC000AE0022A09D1012D02D1FFF71FFF03E077
:10D5CC00032D02D1FFF780FD48B1554B28461B684F
:10D5DC005B699847032801D109230FE068B94D4ACC
:10D5EC00504B12684FF0300192B2D3185B000022FE
:10D5FC001A604D4B1980062300E00823464A126836
:10D60C001372E3E0062D18D11A7812F07F0F40F058
:10D61C0097809B78012B03D1414B1B68DB696EE033
:10D62C00022B03D13E4B1B681B6A68E0032B40F0B6
:10D63C0087803B4B1B685B6A61E0002D3CD15988AD
:10D64C0000297DD15A6822F47F42B2F5003F77D190
:10D65C001A7812F07F0203D19B88002B70D129E03D
:10D66C00012A0BD158792E4B1B689B6998470028CF
:10D67C0066D123689B7A002B62D01BE0022A5FD113
:10D68C005B7913F0800F03F00F0205D0274951F896
:10D69C00221001F0300104E0244951F8221001F469
:10D6AC0040512348007882424AD213F0700F47D180
:10D6BC00002945D01F4B23E0082D05D11B7813F012
:10D6CC007F0F3DD11C4B1BE00A2D39D11A7802F08B
:10D6DC007F02012A34D19A7A002A31D05988002944
:10D6EC002ED15A6822F47F42B2F5803F28D1587966
:10D6FC000B4B1B689B69984710BB104B00E0FBB1B0
:10D70C00054A4FF00001126800209361518298473E
:10D71C00002020E0505C0040F40900200430002080
:10D72C0088090020023000208C2B0020005C004077
:10D73C005C0100202DD000085DCF0008BDCF000893
:10D74C00244C254B22681B6850781B69984703288A
:10D75C0001D1236806E01F4B4FF6FF711B681A8A34
:10D76C008A4201D1092203E0022800D012B9082212
:10D77C001A722BE093F90010002921DAD988019153
:10D78C000198824202D9019A1A8211E08A420FD280
:10D79C001149096891F82C108A4201D2002105E048
:10D7AC0092FBF1F001FB102212B901210B4A11700E
:10D7BC00094A126892F82C209A82FFF799FD05E02D
:10D7CC0003221A72064B4FF440521A80FFF706FDE3
:10D7DC00FEBD00BFF4090020880900203903002099
:10D7EC008A2B0020002383814FF416528380C38040
:10D7FC0003814FF00C030260438170470A8810B517
:10D80C004C88B1F804C0038AC98844EA020242EA8F
:10D81C000C0223F470630A431B041B0C92B242EA01
:10D82C000303038210BD00BF0023C3800380438029
:10D83C008380704721B183899BB243F4005304E089
:10D84C00838923F400531B041B0C8381704700BF96
:10D85C0001F01F034FF0010CC1F3421161450CFAAA
:10D86C0003F301D10C3004E0022901D1103000E0A7
:10D87C0014301AB1026842EA030302E0026822EA99
:10D88C0003030360704700BF1AB1838A9BB219432C
:10D89C0003E0838A9BB223EA01018182704700BFB7
:10D8AC00038A23F00F031B041B0C0382038A9BB215
:10D8BC0041EA030303827047838923F400631B044A
:10D8CC001B0C838183899BB241EA030383817047DC
:10D8DC0021B183899BB243F0020304E0838923F0D6
:10D8EC0002031B041B0C8381704700BF038A23F0C7
:10D8FC0020031B041B0C0382038A9BB241EA030323
:10D90C000382704721B1038A9BB243F4804304E045
:10D91C00038A23F480431B041B0C0382704700BF53
:10D92C00C905C90D818070478088C005C00D70473E
:10D93C0083899BB243F0010383817047038BDBB275
:10D94C000383038B9BB243EA01230383704700BF1D
:10D95C00038B03F47F430383038B9BB241EA0303E2
:10D96C000383704721B1838A9BB243F0200304E008
:10D97C00838A23F020031B041B0C8382704700BF97
:10D98C0021B1838A9BB243F0100304E0838A23F015
:10D99C0010031B041B0C8382704700BF21B1838AC8
:10D9AC009BB243F0080304E0838A23F008031B04B2
:10D9BC001B0C8382704700BF838A23F004031B0473
:10D9CC001B0C8382838A9BB241EA030383827047D8
:10D9DC0021B1838A9BB243F0020304E0838A23F0D3
:10D9EC0002031B041B0C8382704700BF038819427F
:10D9FC000CBF002001207047C94389B201807047D9
:10DA0C004FF0010CC1F3421201F01F0362450CFAF6
:10DA1C0003F301D1828903E0022A0CBF028A828AB5
:10DA2C0092B21340028892B20BB9184607E0090A69
:10DA3C00012313FA01F111420CBF002001207047A1
:10DA4C00090A01238B40DB439BB20380704700BF64
:10DA5C00038ACA8823F440531B041B0C1343038210
:10DA6C0083898A8830B5044608890D4623F4B0535F
:10DA7C00498940EA020223F00C030A431B041B0CE5
:10DA8C0092B242EA0303A381A38AAA8923F44073C6
:10DA9C001B041B0C134387B0A38201A801F0E8F808
:10DAAC000E4B2A689C420CBF049B039B19215943C3
:10DABC0092006423B1FBF2F1B1FBF3F212011009F5
:10DACC0003FB101109013231B1FBF3F303F00F0327
:10DADC0043EA020292B2228107B030BD0038014005
:10DAEC0008B5214B98422BD008D8A3F50063984277
:10DAFC0016D003F58063984234D119E01B4B984241
:10DB0C0026D003F5684398422CD101214FF4804074
:10DB1C0001F020F94FF48040002101F01BF921E0C5
:10DB2C004FF40030012101F023F94FF4003016E0DE
:10DB3C004FF48020012101F01BF94FF480200EE0FE
:10DB4C004FF40020012101F013F94FF4002006E0FE
:10DB5C004FF48010012101F00BF94FF480100021DB
:10DB6C0001F006F908BD00BF004C00400050004019
:10DB7C00038803F08F0303800388B1F806C04A883A
:10DB8C009BB243EA0C0313439BB203808B888385BF
:10DB9C000B880385064B984203D003F5006398422B
:10DBAC0001D10B7A03864FF001038382704700BFCB
:10DBBC00002C0140038C2DE9F04123F001031B04E0
:10DBCC001B0C0384038C0A894C8823F002031C4E23
:10DBDC0014431B048288B1F806C0058B1B0CA4B23D
:10DBEC00B04244EA030392B20C88ADB2A0F834C040
:10DBFC0003D006F50066B04218D18E894F89B1F872
:10DC0C000E804FF6F77C03EA0C0C4CEA070748EA47
:10DC1C0006064FF6FB73898847F6FF4C02EA0C0C9C
:10DC2C0007EA0303B2B20B4342EA0C024FF68F71C0
:10DC3C0005EA01012143828001830384BDE8F08160
:10DC4C00002C0140038C2DE9F04123F010031B0440
:10DC5C001B0C0384028CB1F808C022F020021204C1
:10DC6C008488120C4B8842EA0C1242EA0313A2B2CB
:10DC7C001B4C068BB1F806C0A0420D88B6B29BB205
:10DC8C00A0F838C003D004F50064A0421BD1B1F851
:10DC9C000A804FF67F748F8903EA040447F2FF3C35
:10DCAC0002EA0C0C44EA0814CA894FF6BF7389883F
:10DCBC0004EA03034CEA870C43EA01134CEA8202A0
:10DCCC003C469BB292B248F6FF7106EA010141EA6A
:10DCDC00052189B2828001830384BDE8F08100BFF5
:10DCEC00002C0140038C2DE9F04123F480731B04BC
:10DCFC001B0C0384028CB1F808C022F400721204CD
:10DD0C008488120C4B8842EA0C2242EA0323A2B20A
:10DD1C001A4C868BB1F806C0A0420D88B6B29BB2E5
:10DD2C00A0F83CC003D004F50064A0421BD1B1F8AC
:10DD3C000A804FF2FF748F8903EA040444F6FF7CD7
:10DD4C0002EA0C0C44EA0824CA894FF6FF3389888E
:10DD5C0004EA03034CEA071C43EA01234CEA0212CF
:10DD6C003C469BB292B24FF68F7106EA01012943F1
:10DD7C00828081830384BDE8F08100BF002C0140C8
:10DD8C00038CF0B523F480531B041B0C0384B1F8F3
:10DD9C0006C0078C0C8882880D89868B4B88A0F86E
:10DDAC0040C0DFF848C0BFB2604592B2B6B203D0F3
:10DDBC000CF5006C604505D192048989920C42EAFD
:10DDCC00811292B24DF6FF7C07EA0C0C48F6FF71FB
:10DDDC0006EA01014CEA053C41EA04214CEA033312
:10DDEC0089B29BB2828081830384F0BD002C0140F8
:10DDFC00B1F802C00B888A884CEA0303B1F806C05C
:10DE0C0013430A8943EA0C03B1F80AC013438A8905
:10DE1C0043EA0C0313439BB2A0F84430704700BF95
:10DE2C0000234FF0FF320372438082800380C38053
:10DE3C00704700BF0023C381038043808380C3806D
:10DE4C00038143818381704700234FF001020381DA
:10DE5C00038043808280C380704700BF002383818E
:10DE6C00038043808380C38003814381704700BF5C
:10DE7C0021B103889BB243F0010304E0038823F033
:10DE8C0001039B059B0D0380704700BF39B1B0F8AF
:10DE9C0044306FEA43436FEA53439BB203E0B0F85C
:10DEAC0044305B045B0CA0F8443070471AB1838992
:10DEBC009BB2194303E083899BB223EA0101818160
:10DECC00704700BF818270470A43A0F84820704712
:10DEDC001AB183899BB2194303E083899BB223EA6D
:10DEEC0001018181704700BF038923F007031B04E4
:10DEFC001B0C0381704700BFB0F808C05FFA8CFCA4
:10DF0C0041EA0C0C42EA0C0C4CEA032C1FFA8CFC78
:10DF1C00A0F808C0704700BF10B50446FFF7ECFF2F
:10DF2C0023899BB243F48043238110BD10B5044672
:10DF3C00FFF7E2FF238923F077031B041B0C43F04C
:10DF4C007703238110BD00BF01858282704700BF1B
:10DF5C00038823F070039B059B0D41EA03030380A8
:10DF6C00704700BF038923F070031B041B0C41EAAC
:10DF7C0003030381704700BF10B50446FFF7F2FF9F
:10DF8C0023899BB243F00703238110BD30B504896C
:10DF9C00B0F818C0058C2CF4407CADB22CF0030CFE
:10DFAC0024F007044FEA0C4C25F0220542EA050543
:10DFBC0024044FEA1C4C45EA0315240C4CF4807CD9
:10DFCC0021434CF0010CADB20181A0F818C00584BE
:10DFDC0030BD00BF038B23F070031B041B0C41EA04
:10DFEC0003030383704700BF038B23F4E0431B043C
:10DFFC001B0C43EA01239BB203837047838B23F0F2
:10E00C0070031B041B0C41EA03038383704700BF9E
:10E01C00838B23F4E0431B041B0C43EA01239BB2C8
:10E02C008383704721B103889BB243F0800304E0E3
:10E03C00038823F080039B059B0D0380704700BF72
:10E04C0021B183889BB243F0040304E0838823F05E
:10E05C0004031B041B0C8380704700BF21B1838811
:10E06C009BB243F0080304E0838823F008031B04ED
:10E07C001B0C8380704700BF21B183889BB243F097
:10E08C00010304E0838823F001031B041B0C838031
:10E09C00704700BF038B23F008031B041B0C41EAE1
:10E0AC0003030383704700BF038B23F400631B043B
:10E0BC001B0C43EA01239BB203837047838B23F031
:10E0CC0008031B041B0C41EA03038383704700BF46
:10E0DC00838B23F400631B041B0C43EA01239BB2C8
:10E0EC0083837047038B23F004031B041B0C41EA4E
:10E0FC0003030383704700BF038B23F480631B046B
:10E10C001B0C43EA01239BB203837047838B23F0E0
:10E11C0004031B041B0C41EA03038383704700BFF9
:10E12C00838B23F480631B041B0C43EA01239BB2F7
:10E13C0083837047038B23F080031B041B0C41EA81
:10E14C0003030383704700BF038B5B045B0C43EA40
:10E15C0001239BB203837047838B23F080031B0442
:10E16C001B0C41EA03038383704700BF838B5B0462
:10E17C005B0C43EA01239BB283837047038C23F02F
:10E18C0002031B041B0C41EA03030384704700BF0A
:10E19C00038C23F008031B041B0C41EA03030384C8
:10E1AC00704700BF038C23F020031B041B0C43EAB5
:10E1BC0001139BB203847047038C23F080031B0470
:10E1CC001B0C43EA01139BB203847047038C23F4AA
:10E1DC0000731B041B0C43EA01239BB2038470479E
:10E1EC00038C23F400631B041B0C43EA01239BB236
:10E1FC0003847047038C23F400531B041B0C43EA69
:10E20C0001339BB20384704701238B408A40018CFD
:10E21C0089B221EA03030384018C0A4392B202847B
:10E22C00704700BF04238B408A40018C89B221EADD
:10E23C0003030384018C0A4392B20284704700BF2B
:10E24C0001238B40B0F820C010B51FFA8CFC2CEACF
:10E25C000303038409B1082909D11830490844582B
:10E26C004FF68F7304EA0303435043580CE0043910
:10E27C001830C1F34E01445848F6FF7304EA030307
:10E28C0043501202435892B243EA0202425010BD6C
:10E29C0021B103889BB243F0020304E0038823F00E
:10E2AC0002039B059B0D0380704700BF21B10388BF
:10E2BC009BB243F0040304E0038823F004039B05A2
:10E2CC009B0D0380704700BF21B183889BB243F044
:10E2DC00800304E0838823F080031B041B0C8380E1
:10E2EC00704700BF038823F008039B059B0D038038
:10E2FC0003889BB241EA030303807047838823F0B1
:10E30C0070031B041B0C838083889BB241EA0303BC
:10E31C0083807047038923F007031B041B0C0381C4
:10E32C0003899BB241EA030303817047038923F0FD
:10E33C0080031B041B0C038103899BB241EA03037A
:10E34C00038170478184704781857047818670474F
:10E35C000187704781877047A0F84010704700BF55
:10E36C00038B23F00C031B041B0C0383038B9BB24A
:10E37C0041EA030303837047038B23F440631B04BC
:10E38C001B0C0383038B9BB243EA01239BB20383D5
:10E39C00704700BF838B23F00C031B041B0C83837F
:10E3AC00838B9BB241EA030383837047838B23F4F3
:10E3BC0040631B041B0C8383838B9BB243EA0123B6
:10E3CC009BB28383704700BF0388DBB20380038852
:10E3DC009BB241EA03030380704700BF808E80B27A
:10E3EC00704700BF008F80B2704700BF808F80B233
:10E3FC00704700BFB0F8400080B27047808C80B28C
:10E40C00704700BF008D80B2704700BF038A19426D
:10E41C000CBF002001207047C94389B201827047AC
:10E42C00038A828911EA030092B203D011420CBF15
:10E43C0000200120704700BFC94389B20182704798
:10E44C00B0F820C010B52CF0010C4FEA0C4C4FEA80
:10E45C001C4CA0F820C0048BB0F820C0A4B21FFA4A
:10E46C008CFC24F0F30442EA04042CF0020C44EA81
:10E47C0003144CF0010C4CEA010CA4B20483A0F878
:10E48C0020C010BDB0F820C010B52CF0100C4FEA15
:10E49C000C4C4FEA1C4CA0F820C0B0F818C0048CEF
:10E4AC002CF4407CA4B24FEA0C5C4FEA1C5C24F0C8
:10E4BC0020044CEA022C44F010044CEA033C44EADD
:10E4CC0001141FFA8CFCA4B2A0F818C0048410BD6F
:10E4DC0038B50D46602D1146044603D10122FFF7D5
:10E4EC00D1FF02E00122FFF7ABFF29462046FFF7E0
:10E4FC0039FD23899BB243F00703238138BD00BF4C
:10E50C00F8B50C46A2884988B4F800C00546002925
:10E51C000CBF02270027012A0CBF022601262389E3
:10E52C00BCF1000F10D1FFF78BFF2846E188FFF7F5
:10E53C0017FF2846394632462389FFF7A3FF2846A2
:10E54C00E188FFF719FF0FE0FFF79CFF2846E188F1
:10E55C00FFF712FF2846394632462389FFF770FF32
:10E56C002846E188FFF7FCFEF8BD00BF38B50B88E4
:10E57C000C4605464BB94988A2882389FFF760FFF2
:10E58C002846E188FFF7ECFE53E0042B09D14988BB
:10E59C00A2882389FFF776FF2846E188FFF7ECFE77
:10E5AC0047E0082BB1F802C0B1F804E0098920D18A
:10E5BC00028C22F480721204120C0284838B028C63
:10E5CC009BB292B223F0F30322F4007243EA0111DE
:10E5DC0042EA0C2C89B21FFA8CFC41EA0E0E4CF468
:10E5EC00807CA0F81CE0A0F820C0E188FFF7D2FEE8
:10E5FC001FE0028C22F480521204120C0284838BD2
:10E60C00028C23F4407392B21B051B0D22F40052B2
:10E61C0043EA0E2342EA0C3C43EA01331FFA8CFC1A
:10E62C009BB24CF4805C8383A0F820C0E188FFF798
:10E63C00BDFE38BD08B52D4B984237D00BD8A3F58D
:10E64C000063984226D003F58063984228D0B0F13D
:10E65C00804F4AD118E0264B984233D004D8A3F50A
:10E66C008063984241D127E0224B984204D003F5B5
:10E67C000063984239D12EE04FF40060012100F084
:10E68C0069FB4FF400602DE00120014600F070FBA7
:10E69C0001201CE00220012100F06AFB022016E0A0
:10E6AC000420012100F064FB042010E0082001216B
:10E6BC0000F05EFB08200AE01020012100F058FB5E
:10E6CC00102004E02020012100F052FB202000212A
:10E6DC0000F04EFB09E04FF40050012100F03AFB32
:10E6EC004FF40050002100F035FB08BD000C004039
:10E6FC0000140040002C0140042804D1054B1A687A
:10E70C0042F0040203E0034B1A6822F004021A6080
:10E71C00704700BF10E000E0014B5860704700BF2D
:10E72C0010E000E0012804D1084B1A6842F0010205
:10E73C0006E010F1020F05D1044B1A6822F0010219
:10E74C001A6002E0014B00229A60704710E000E072
:10E75C0020B1054B1A6842F0020203E0024B1A6822
:10E76C0022F002021A60704710E000E0014B98683A
:10E77C00704700BF10E000E0C308022B0BBF044B36
:10E78C00034B1B68DB6833FA00F000F001007047A4
:10E79C0010E000E00B884A88B1F804C01A43CB881B
:10E7AC0042EA0C02B1F808C01A434B8930B542EA70
:10E7BC000C028D89B0F800C0CC891A432A4322433D
:10E7CC000CF4415313439BB20380838B23F40063FB
:10E7DC001B041B0C83830B8A038230BD00234FF078
:10E7EC000702C3810282038043808380C38003813C
:10E7FC0043818381704700BF0023438103804380A2
:10E80C008380C3804FF002030381704721B10388DA
:10E81C009BB243F0400304E0038823F040031B0445
:10E82C001B0C0380704700BF21B1838B9BB243F458
:10E83C00806304E0838B23F480631B041B0C8383B1
:10E84C00704700BF0909012313FA01F189B21AB10B
:10E85C0083889BB2194303E083889BB223EA0101AE
:10E86C00818070471AB183889BB2194303E0838877
:10E87C009BB223EA01018180704700BF8181704700
:10E88C00808980B2704700BF4FF6FF63994205D074
:10E89C0003889BB243F48073038002E00388194021
:10E8AC000180704721B183889BB243F0040304E0DC
:10E8BC00838823F004031B041B0C8380704700BF68
:10E8CC00038823F400631B041B0C038003889BB296
:10E8DC0041EA03030380704703889BB243F48053DF
:10E8EC000380704721B103889BB243F4005304E0CA
:10E8FC00038823F400531B041B0C0380704700BFD8
:10E90C00012914BF008B808A80B27047008A80B2C4
:10E91C00704700BFB1F5804F04D103889BB243F41C
:10E92C00804304E0038823F480431B041B0C038006
:10E93C00704700BF038919420CBF002001207047AB
:10E94C00202906D1038903889BB243F0400303803E
:10E95C0008E0402901D0082901D1038902E0C9430C
:10E96C0089B20181704700BF012301F00F0213FA35
:10E97C0002F2B0F804C000891FFA8CFC80B210407F
:10E98C0006D009098B401CEA030F0CBF00200120A4
:10E99C00704700BF552906D1038903889BB243F009
:10E9AC00400303800DE0562901D0532901D103897E
:10E9BC0007E001F00F01012313FA01F1C94389B2F9
:10E9CC0001817047838BF0B523F47A6323F01F0326
:10E9DC001B041B0C83834FF0020303840B89868B6F
:10E9EC00022B87B004460D46B6B201D1002225E0B9
:10E9FC0001A88F8800F03CF9EB88002F0CBF012791
:10EA0C000227B3F5007F2989019A06D1A3F5FB7380
:10EA1C0053430902B3FBF1F305E00A2349015A43BE
:10EA2C004F43B2FBF7F305330A229BB2B3FBF2F36D
:10EA3C0003F001021202C3F34F0392B2991E89B282
:10EA4C00FE2928BF002228BF0223E98842EA0303DB
:10EA5C000B439BB223842B886A8846EA0303A9885C
:10EA6C0043F4006313436A890B4313439BB2A383A0
:10EA7C0007B0F0BD08B5154B98421BD003F5744395
:10EA8C00984204D0A3F5784398421DD10AE00121A5
:10EA9C004FF4805000F05EF94FF48050002100F0EC
:10EAAC0059F911E04FF48040012100F061F94FF465
:10EABC00804006E04FF40040012100F059F94FF47A
:10EACC000040002100F054F908BD00BF003C00409C
:10EADC000D4B0E4A196841F001011960596801EAA1
:10EAEC0002025A601A6822F0847222F480321A6090
:10EAFC001A6822F480221A605A6822F4FE025A60C4
:10EB0C0000229A60704700BF001002400000FFF81E
:10EB1C000C4BB0F5803F1A6822F480321A601A68E8
:10EB2C0022F480221A6003D0B0F5802F08D103E0C4
:10EB3C001A6842F4803202E01A6842F4A0221A6089
:10EB4C00704700BF00100240034B1A6822F0F80215
:10EB5C0042EAC0021A60704700100240014B186074
:10EB6C00704700BF00004242044B5A6822F47C12EA
:10EB7C0040EA02020A435A60704700BF001002408C
:10EB8C00014B1860704700BF60004242034B5A684B
:10EB9C0022F0030240EA02025A6070470010024061
:10EBAC00024B586800F00C00704700BF0010024088
:10EBBC00034B5A6822F0F00240EA02025A60704796
:10EBCC0000100240034B5A6822F4E06240EA020251
:10EBDC005A60704700100240034B5A6822F460528E
:10EBEC0042EAC0025A6070470010024019B1054B4E
:10EBFC001A78104303E0034B1A7822EA00001870CD
:10EC0C00704700BF09100240014B1860704700BFED
:10EC1C00D8004242034B5A6822F4404240EA0202B6
:10EC2C005A60704700100240064B002201281A70EF
:10EC3C001A7002D0042804D101E0187001E00522FA
:10EC4C001A70704720100240014B1860704700BFCB
:10EC5C0080044242024B1A6A40EA02021A6270476E
:10EC6C0000100240014B1860704700BF3C04424248
:10EC7C001F4B10B55A6802F00C02042A13D0082A54
:10EC8C0011D15A685968C2F38342023211F4803FA1
:10EC9C0003D05B6813F4003F01D0164B00E0164B19
:10ECAC005A43026001E0144B0360114A134B516844
:10ECBC000468C1F30311595C34FA01F141605468E2
:10ECCC00C4F3022C13F80C4031FA04F48460546839
:10ECDC00C4F3C22C13F80CC021FA0CF1C1605268B9
:10ECEC00C2F381329B181B7CB1FBF3F1016110BDA7
:10ECFC000010024000093D0000127A00B00A010821
:10ED0C0019B1054B5A69104303E0034B5A6922EAC7
:10ED1C0000005861704700BF0010024019B1054B4C
:10ED2C009A69104303E0034B9A6922EA0000986148
:10ED3C00704700BF0010024019B1054BDA6910434F
:10ED4C0003E0034BDA6922EA0000D861704700BF88
:10ED5C000010024019B1054BDA68104303E0034B75
:10ED6C00DA6822EA0000D860704700BF0010024049
:10ED7C0019B1054B1A69104303E0034B1A6922EAD7
:10ED8C0000001861704700BF00100240014B186072
:10ED9C00704700BF40044242014B1860704700BFEF
:10EDAC004C004242014B1870704700BF07100240E4
:10EDBC004309012B02D1084B1B6805E0022B0BBF4A
:10EDCC00054B054B1B6A5B6A00F01F0033FA00F021
:10EDDC0000F00100704700BF0010024008B5312060
:10EDEC00FFF7E6FF094B18705A6801325A601A781F
:10EDFC0022B95A6840F2FF139A42F0D13120FFF742
:10EE0C00D7FF003818BF012008BD00BF3C0300200D
:10EE1C00024B5A6A42F080725A62704700100240EC
:10EE2C00034B9B6818420CBF00200120704700BFA9
:10EE3C0000100240014B1870704700BF0A100240CE
:10EE4C000B4B4FF0FF316FF07042C3F88010C3F8DA
:10EE5C008420C3F88011C3F88421002303F1C0017E
:10EE6C00034A013300200F2B42F82100F6D17047E2
:10EE7C0000E100E0094B4FF0206058600848002288
:10EE8C004FF0FF319A60D8601A615A619A61DA6169
:10EE9C001A625A629962D9621963704700ED00E0F8
:10EEAC000000FA0540F0BE60024B40F42020D86010
:10EEBC00704700BF00ED00E030B5C27803787AB33C
:10EECC001C4A4178D2684FF00F0CD243C2F3022295
:10EEDC002CFA02FCC2F104029140807803F0030288
:10EEEC000CEA000C4CEA010CD2004FEA0C1CFF207F
:10EEFC0090400CFA02FC012403F01F029440990884
:10EF0C000D4AC03152F821500CEA000C25EA0000E1
:10EF1C004CEA00005B0942F8210042F8234008E06B
:10EF2C0003F01F02012191405B09034A203342F890
:10EF3C00231030BD00ED00E000E100E00023C370C1
:10EF4C000370437083707047024B5868C0F30930EC
:10EF5C00704700BF00ED00E0012200F01F0312FA21
:10EF6C0003F34009044A403052F8200018409842FC
:10EF7C0014BF00200120704700E100E0014B186035
:10EF8C00704700BF00EF00E000F01F0301229A4021
:10EF9C004009024B603043F82020704700E100E04C
:10EFAC00024B58688005800D704700BF00ED00E0F3
:10EFBC00012200F01F0312FA03F34009044A8030C7
:10EFCC0052F820001840984214BF002001207047CE
:10EFDC0000E100E0014B1868704700BF00ED00E055
:10EFEC0021F0604121F07F01014B01439960704792
:10EFFC0000ED00E0014A024BDA6070470400FA05AC
:10F00C0000ED00E0014A024BDA6070470100FA059E
:10F01C0000ED00E019B1054B1A69104303E0034BF6
:10F02C001A6922EA00001861704700BF00ED00E089
:10F03C0000F01F00012313FA00F019B1044B5A6AB7
:10F04C00104303E0024B5A6A22EA000058627047F0
:10F05C0000ED00E0144B70B5DC684FF0FF0CE4439E
:10F06C00C4F302242CFA04F5C4F1040411FA04F4D8
:10F07C00C0F30126F6000CFA06FC02EA050545EA87
:10F08C000404240114FA06F6C0F38110063053F878
:10F09C00202022EA0C0243F8202053F820201643AB
:10F0AC0043F8206070BD00BF00ED00E0C0F383208A
:10F0BC0001238340044A506A03EA0000984214BFBB
:10F0CC0000200120704700BF00ED00E000F01F00A1
:10F0DC0001228240024B59680A435A60704700BFB4
:10F0EC0000ED00E000F01F020123013A13FA02F2D6
:10F0FC00024B59680A435A60704700BF00ED00E0AC
:10F10C00C0F3833001238340044A506A03EA0000B1
:10F11C00984214BF00200120704700BF00ED00E0B2
:10F12C00C0F3814313B90A4BD86A10E0012B0CD100
:10F13C00074AC0F30153906ADA00D040022B14BF87
:10F14C0000F00F0000F0FF0001E0014B186B70475E
:10F15C0000ED00E010F4800F0BBF024B014B586B1D
:10F16C00986B704700ED00E008B5F4F7F9FF08BDA7
:10F17C0008B50001F4F7F1FF08BD00BF08B5F4F7BE
:10F18C00EAFF08BD08B5F4F7E4FF08BD08B5F4F7CD
:10F19C00DEFF08BD08B5F4F7D8FF08BD002341F227
:10F1AC008832C260C38003804BF6FF7283804FF4B9
:10F1BC00804342800381704721B103889BB243F0A6
:10F1CC00010304E0038823F001031B041B0C0380E0
:10F1DC00704700BF21B183889BB243F4006304E005
:10F1EC00838823F400631B041B0C8380704700BFCF
:10F1FC0021B183889BB243F4805304E0838823F4C9
:10F20C0080531B041B0C8380704700BF21B1038803
:10F21C009BB243F4807304E0038823F480731B04D3
:10F22C001B0C0380704700BF21B103889BB243F4D1
:10F23C00007304E0038823F400731B041B0C03808D
:10F24C00704700BF21B103889BB243F4806304E094
:10F25C00038823F480631B041B0C0380704700BFDE
:10F26C00838901F0FE019BB223F0FE0341EA030304
:10F27C008381704721B183899BB243F0010304E081
:10F28C00838923F001031B041B0C8381704700BF8F
:10F29C0021B103889BB243F0400304E0038823F0C0
:10F2AC0040031B041B0C0380704700BF1AB18388FA
:10F2BC009BB2194303E083889BB223EA010181804E
:10F2CC00704700BF01827047008AC0B2704700BF10
:10F2DC0012B141F0010101E001F0FE010182704721
:10F2EC0082B0019B0190CB5A98B202B0704700BF1C
:10F2FC0031B103886FEA43436FEA53439BB202E098
:10F30C0003885B045B0C0380704700BFB1F5005FA2
:10F31C0004D103889BB243F4005304E0038823F424
:10F32C0000531B041B0C0380704700BF21B10388E2
:10F33C009BB243F4805304E0038823F480531B04F2
:10F34C001B0C0380704700BFB1F5006F04D103881C
:10F35C009BB243F4006304E0038823F400631B04B2
:10F36C001B0C0380704700BF21B103889BB243F094
:10F37C00200304E0038823F020031B041B0C0380F0
:10F38C00704700BF008BC0F30720704721B1038882
:10F39C009BB243F0100304E0038823F010031B041A
:10F3AC001B0C0380704700BF21B903889BB243F04C
:10F3BC00800304E0038823F080031B041B0C0380F0
:10F3CC00704700BFB1F5804F05D0838B23F4804389
:10F3DC001B041B0C03E0838B9BB243F4804383839D
:10F3EC00704700BF828A038B90B240EA034020F042
:10F3FC007F407047828A038B90B240EA034020F032
:10F40C007F40884214BF002001207047838A028B02
:10F41C009BB243EA02430B4023F07F40003818BFF5
:10F42C00012070470B0F012B03D1C94389B2818294
:10F43C000EE0022B01D1838A0AE0062B06D1838AC7
:10F44C0003889BB243F00103038001E0838A038BA2
:10F45C00704700BF838A028B9BB243EA02430B4086
:10F46C0023F07F40003818BF012070470B0F012B91
:10F47C0003D1C94389B281820EE0022B01D1838A68
:10F48C000AE0062B06D1838A03889BB243F0010362
:10F49C00038001E0838A038B704700BF70B586B090
:10F4AC000446868801A80D46FFF7E2FB0399304815
:10F4BC0026F03F063604B1FBF0F0360C80B240EA81
:10F4CC000606A6802288EB6822F001021204120CB8
:10F4DC002280284A93420AD85B00B1FBF3F3013037
:10F4EC009BB280B22084032B98BF042323E0B5F891
:10F4FC0002C04BF6FF72944505D103225343B1FB76
:10F50C00F3F39BB206E019225343B1FBF3F39BB226
:10F51C0043F480431A05120D0AB943F001034FF46A
:10F52C009672504302F52F7290FBF2F0013080B2CC
:10F53C00208443F40043A38323889BB243F001034C
:10F54C0023802388E98823F480632A8823F00A0324
:10F55C001B0441EA02021B0C13439BB223802B8930
:10F56C00AA8842EA03039BB2238106B070BD00BF98
:10F57C0040420F00A086010008B50D4B984204D004
:10F58C0003F58063984212D107E04FF4001001217B
:10F59C00FFF7EEFB4FF4001006E04FF48000012162
:10F5AC00FFF7E6FB4FF480000021FFF7E1FB08BDFD
:10F5BC0000540040CB78F0B513F0100F18BF8A78C8
:10F5CC00098803F00F0C18BF4CEA020C11F0FF0F66
:10F5DC001AD0046800220126964006EA0105B542BD
:10F5EC000ED196000F27B7400CFA06F624EA070452
:10F5FC003443282B01D1456102E0482B08BF05613B
:10F60C000132082AE7D10460FF291CD94468002282
:10F61C0002F108050126AE4006EA0105B5420ED1FD
:10F62C0096000F27B7400CFA06F624EA0704344379
:10F63C00282B01D1456102E0482B08BF056101323E
:10F64C00082AE5D14460F0BD0423C3700223837003
:10F65C004FF0FF3303807047836819420CBF0020C2
:10F66C0001207047806880B2704700BFC3681942A0
:10F67C000CBF002001207047C06880B2704700BFEB
:10F68C0001617047416170470AB1016100E041615D
:10F69C00704700BFC160704741F480338361816162
:10F6AC008361836983697047064A10B514684FF605
:10F6BC00807341EA001104EA030341EA0303136077
:10F6CC0010BD00BF00000140014B1860704700BF27
:10F6DC001C0020420304154A00F4401C1B0CBCF512
:10F6EC00401F30B5546806D1556824F0706425F07D
:10F6FC007065556011E010F4801F06D0C0F3034212
:10F70C004FF0030C0CFA02F203E0420D120113FA53
:10F71C0002F224EA020444F0706419B1400D0001B5
:10F72C0083401C43014B5C6030BD00BF00000140B6
:10F73C0001F003039B000F229A4010FA03F310B55B
:10F74C008908074C023154F8210020EA020244F8DF
:10F75C00212054F82120134344F8213010BD00BF60
:10F76C00000001400120014608B5FFF7F3FA012023
:10F77C000021FFF7EFFA08BD08B5264B98422BD0B5
:10F78C000CD8A3F5006398421AD003F58063984215
:10F79C001CD0A3F5006398423AD10BE01E4B984263
:10F7AC0026D003F58063984228D0A3F500639842D5
:10F7BC002ED117E004200121FFF7CCFA042024E01D
:10F7CC0008200121FFF7C6FA08201EE010200121B5
:10F7DC00FFF7C0FA102018E020200121FFF7BAFA39
:10F7EC00202012E040200121FFF7B4FA40200CE069
:10F7FC0080200121FFF7AEFA802006E04FF48070E4
:10F80C000121FFF7A7FA4FF480700021FFF7A2FA4D
:10F81C0008BD00BF00140140001C0140044B1A68D5
:10F82C0002F038021A601A6840EA02021A60704745
:10F83C0000200240044B1A6822F008021A601A6871
:10F84C0040EA02021A60704700200240044B1A681A
:10F85C0022F010021A601A6840EA02021A6070471D
:10F86C0000200240044B00221A605A609A60DA6051
:10F87C00024A5A61704700BF00040140FFFF0700B5
:10F88C00837930B5016802794BB3184BCC431D68B2
:10F89C0090F805C004EA05051D605D682C405C60AD
:10F8AC00D45844EA0101D15002689868D14301EA66
:10F8BC0000009860D8680140BCF1100FD96007D1E6
:10F8CC00996811439960D96841EA0202DA600BE049
:10F8DC005CF8031041EA02024CF8032004E0034BED
:10F8EC00D05820EA0101D15030BD00BF00040140C6
:10F8FC0000230C228371427103600371704700BFB7
:10F90C00024B1A6940EA02021A6170470004014076
:10F91C00034B5B6918420CBF00200120704700BFED
:10F92C0000040140014B5861704700BF00040140C6
:10F93C00054B1A685B69034001D1184603E010427D
:10F94C000CBF00200120704700040140014B58619E
:10F95C00704700BF000401400268002322F001023E
:10F96C000260036043608360C3602D4B984233D0C8
:10F97C0011D83C3B984229D006D8283B984221D03C
:10F98C00143398424BD11FE0264B984220D01433AD
:10F99C00984244D11EE0244B98422CD008D8A3F5B1
:10F9AC00677398421DD003F56273984237D11DE0FE
:10F9BC001E4B984229D0143398422BD0283B9842A6
:10F9CC002DD11DE01A4B12E0194B15E0184B18E025
:10F9DC00174B1BE0164B1EE0154B5A6842F4700295
:10F9EC001CE0134B5A6842F0706217E0114B5A68D6
:10F9FC0042F00F0212E00F4B5A6842F0F0020DE099
:10FA0C000C4B5A6842F4706208E00A4B5A6842F494
:10FA1C00704203E0074B5A6842F470225A607047F8
:10FA2C006C000240440002401C04024044040240AA
:10FA3C0000000240000402408A6870B50C6A0B6931
:10FA4C0044EA02024C691A438B692243CC6905686B
:10FA5C004E6A42EA030323438C6A334325F4FE4C7B
:10FA6C0023432CF0F00C43EA0C030360CB68436097
:10FA7C000B6883604B68C36070BD00BF002383625A
:10FA8C00036043608360C360036143618361C3614E
:10FA9C0003624362704700BF19B1036843F001036E
:10FAAC0002E0036823F001030360704712B103689E
:10FABC00194302E0036823EA01010160704700BFAB
:10FACC00406880B2704700BF10F0805F14BF044BD9
:10FADC00044B1B6803420CBF00200120704700BF81
:10FAEC00000402400000024010F0805F14BF024B83
:10FAFC00024B5860704700BF0004024000000240F7
:10FB0C0010F0805F14BF044B044B1B6803420CBF06
:10FB1C0000200120704700BF00040240000002409A
:10FB2C0010F0805F14BF024B024B5860704700BF4F
:10FB3C000004024000000240436830B523F47023F7
:10FB4C000C680A7923F48073234343EA022343604D
:10FB5C0082688D68CC680A4B45EA040C02EA030300
:10FB6C004A794CEA030343EA420383600B7CC26A82
:10FB7C00013B22F47002DBB242EA0353C36230BD94
:10FB8C00FDF7F1FF002301220274C36003600371CF
:10FB9C0043718360704700BF19B1836843F0010360
:10FBAC0002E0836823F001038360704719B1836816
:10FBBC0043F4807302E0836823F48073836070479E
:10FBCC00C9B212B14368194302E0436823EA010148
:10FBDC0041607047836843F008038360704700BF3F
:10FBEC008068C0F3C0007047836843F004038360EF
:10FBFC00704700BF8068C0F38000704719B18368FC
:10FC0C0043F4A00302E0836823F4A00383607047ED
:10FC1C008068C0F3805070474368013923F4604317
:10FC2C0043EA41334360704719B1436843F40063BE
:10FC3C0002E0436823F4006343607047092930B540
:10FC4C0011D94FF0030C0CFB01FC0725ACF11E0C79
:10FC5C0005FA0CF503FA0CFCC46824EA050343EA24
:10FC6C000C03C3600EE04FF0030C0CFB01FC0725EA
:10FC7C0005FA0CF503FA0CFC046924EA050343EAC3
:10FC8C000C030361062A0DD80523013A5A434FF0A1
:10FC9C001F0C0CFA02FC9140436B23EA0C020A4342
:10FCAC0042631CE00C2A0DD805235A434FF01F0C5D
:10FCBC00233A0CFA02FC9140036B23EA0C020A4330
:10FCCC0002630CE005235A434FF01F0C413A0CFA27
:10FCDC0002FC9140C36A23EA0C020A43C26230BDA3
:10FCEC0019B1836843F4801302E0836823F4801312
:10FCFC0083607047C06C80B2704700BF014B1868BE
:10FD0C00704700BF4C24014019B1436843F4806331
:10FD1C0002E0436823F480634360704719B1436881
:10FD2C0043F4805302E0436823F4805343607047EC
:10FD3C00836823F4E04341EA03038360704700BF08
:10FD4C0019B1836843F4004302E0836823F4004351
:10FD5C008360704719B1836843F4021302E083682F
:10FD6C0023F40213836070478068C0F340507047DF
:10FD7C00092930B511D94FF0030C0CFB01FC0725F8
:10FD8C00ACF11E0C05FA0CF503FA0CFCC46824EA61
:10FD9C00050343EA0C03C3600EE04FF0030C0CFBAD
:10FDAC0001FC072505FA0CF503FA0CFC046924EA9E
:10FDBC00050343EA0C030361836BC3F3015CCCEBD7
:10FDCC00020202324FF0050CD2B20CFB02F20CF123
:10FDDC001A0C0CFA02FC914023EA0C030B438363CC
:10FDEC0030BD00BF836B013923F4401343EA015348
:10FDFC00836370470A5070472830405880B2704770
:10FE0C00436823F4400323F4007341EA0303436083
:10FE1C00704700BF41628262704700BF436823F0A5
:10FE2C001F0341EA03034360704700BF20B1054B39
:10FE3C009A6842F4000203E0024B9A6822F4000232
:10FE4C009A60704700240140036819420CBF0020DF
:10FE5C0001207047C9430160704700BF43680068C8
:10FE6C0010EA112004D0C9B219420CBF00200120A5
:10FE7C00704700BF6FEA11210160704708B5134B42
:10FE8C0098420FD003F5A053984213D0A3F5C0535A
:10FE9C00984219D14FF400700121FEF75BFF4FF42B
:10FEAC0000700EE04FF480600121FEF753FF4FF419
:10FEBC00806006E04FF400400121FEF74BFF4FF449
:10FECC0000400021FEF746FF08BD00BF002801409E
:10FEDC00032A2DE9F0070BD83AB1002311F803C01F
:10FEEC0000F803C001339342F8D1BDE8F007704726
:10FEFC0082180C46034603E014F8011C03F8011C9D
:10FF0C0003F003061946A44601330134002EF3D145
:10FF1C001CF00304634608BFC1EB020C68D06542B9
:10FF2C00C4F1040A0CEB050733464FEACA0A5CF825
:10FF3C0005604FEAC408551A08E057F8044F2646E6
:10FF4C0004FA0AF449EA0404CC5004335C18032D77
:10FF5C0026FA08F9A5F104050CEB0306EDDC0023E9
:10FF6C0002E0F15CE154013319199142F9D3BCE779
:10FF7C0053F8404C41F8404C53F83C4C41F83C4C45
:10FF8C0053F8384C41F8384C53F8344C41F8344C55
:10FF9C0053F8304C41F8304C53F82C4C41F82C4C65
:10FFAC0053F8284C41F8284C53F8244C41F8244C75
:10FFBC0053F8204C41F8204C53F81C4C41F81C4C85
:10FFCC0053F8184C41F8184C53F8144C41F8144C95
:10FFDC0053F8104C41F8104C53F80C4C41F80C4CA5
:10FFEC0053F8084C41F8084C53F8044C41F8044CB5
:04FFFC001C460D464C
:020000040801F1
:1000000040334031BCF13F0FACF1400CB6DC21462F
:100010002B46541B0FE051F8105C43F8105C51F86C
:100020000C5C43F80C5C51F8085C43F8085C51F830
:10003000045C43F8045C0F2C0D469C4601F1100152
:1000400003F11003A4F11004E5DCCCEB0201002362
:1000500003E0EC584CF8034004335E19032903EB2A
:100060000C04A1F10401F4DC7FE700BF80F0004044
:1000700002E000BF81F0004142001FBF5FEA410380
:1000800092EA030F7FEA226C7FEA236C6AD04FEA80
:100090001262D2EB1363C1BFD218414048404140C5
:1000A000B8BF5B42192B88BF704710F0004F40F477
:1000B000000020F07F4018BF404211F0004F41F493
:1000C000000121F07F4118BF494292EA030F3FD05F
:1000D000A2F1010241FA03FC10EB0C00C3F1200372
:1000E00001FA03F100F0004302D5494260EB400001
:1000F000B0F5000F13D3B0F1807F06D340084FEA6C
:10010000310102F10102FE2A51D2B1F1004F40EB60
:10011000C25008BF20F0010040EA030070474900C8
:1001200040EB000010F4000FA2F10102EDD1B0FA93
:1001300080FCACF1080CB2EB0C0200FA0CF0AABF88
:1001400000EBC25052421843BCBFD0401843704726
:1001500092F0000F81F4000106BF80F4000001322C
:10016000013BB5E74FEA41037FEA226C18BF7FEA03
:10017000236C21D092EA030F04D092F0000F08BF45
:100180000846704790EA010F1CBF0020704712F02C
:100190007F4F04D1400028BF40F00040704712F16B
:1001A00000723CBF00F50000704700F0004343F0D0
:1001B000FE4040F4000070477FEA226216BF084606
:1001C0007FEA23630146420206BF5FEA412390EAC9
:1001D000010F40F4800070474FF0000304E000BFBF
:1001E00010F0004348BF40425FEA000C08BF704770
:1001F00043F0964301464FF000001CE050EA010234
:1002000008BF70474FF000030AE000BF50EA010248
:1002100008BF704711F0004302D5404261EB410135
:100220005FEA010C02BF84460146002043F0B6435A
:1002300008BFA3F18053A3F50003BCFA8CF2083A7F
:10024000A3EBC25310DB01FA02FC634400FA02FC88
:10025000C2F12002BCF1004F20FA02F243EB02008F
:1002600008BF20F00100704702F1200201FA02FCF1
:10027000C2F1200250EA4C0021FA02F243EB0200E4
:1002800008BF20EADC7070474FF0FF0C1CEAD05228
:100290001EBF1CEAD15392EA0C0F93EA0C0F6FD0E9
:1002A0001A4480EA010C400218BF5FEA41211ED0C7
:1002B0004FF0006343EA501043EA5111A0FB0131B3
:1002C0000CF00040B1F5000F3EBF490041EAD37188
:1002D0005B0040EA010062F17F02FD2A1DD8B3F104
:1002E000004F40EBC25008BF20F00100704790F073
:1002F000000F0CF0004C08BF49024CEA502040EAC5
:1003000051207F3AC2BFD2F1FF0340EAC25070478A
:1003100040F400004FF00003013A5DDC12F1190FC8
:10032000DCBF00F000407047C2F10002410021FA3A
:1003300002F1C2F1200200FA02FC5FEA310040F152
:10034000000053EA4C0308BF20EADC70704792F0CB
:10035000000F00F0004C02BF400010F4000F013A03
:10036000F9D040EA0C0093F0000F01F0004C02BFFE
:10037000490011F4000F013BF9D041EA0C018FE76D
:100380000CEAD15392EA0C0F18BF93EA0C0F0AD073
:1003900030F0004C18BF31F0004CD8D180EA010099
:1003A00000F00040704790F0000F17BF90F0004F32
:1003B000084691F0000F91F0004F14D092EA0C0F14
:1003C00001D142020FD193EA0C0F03D14B0218BFA7
:1003D000084608D180EA010000F0004040F0FE40ED
:1003E00040F40000704740F0FE4040F44000704789
:1003F0004FF0FF0C1CEAD0521EBF1CEAD15392EA08
:100400000C0F93EA0C0F69D0A2EB030280EA010CF7
:1004100049024FEA402037D04FF0805343EA111190
:1004200043EA10130CF000408B4238BF5B0042F1EE
:100430007D024FF4000C8B4224BF5B1A40EA0C0093
:10044000B3EB510F24BFA3EB510340EA5C00B3EBC5
:10045000910F24BFA3EB910340EA9C00B3EBD10FB3
:1004600024BFA3EBD10340EADC001B0118BF5FEA05
:100470001C1CE0D1FD2A3FF650AF8B4240EBC2502E
:1004800008BF20F0010070470CF0004C4CEA5020EF
:100490007F32C2BFD2F1FF0340EAC250704740F43E
:1004A00000004FF00003013A37E792F0000F00F030
:1004B000004C02BF400010F4000F013AF9D040EAAE
:1004C0000C0093F0000F01F0004C02BF490011F442
:1004D000000F013BF9D041EA0C0195E70CEAD1533A
:1004E00092EA0C0F08D142027FF47DAF93EA0C0F21
:1004F0007FF470AF084676E793EA0C0F04D14B0205
:100500003FF44CAF08466EE730F0004C18BF31F0B6
:10051000004CCAD130F000427FF45CAF31F00043B0
:100520007FF43CAF5FE700BF4FF0FF3C06E000BF49
:100530004FF0010C02E000BF4FF0010C4DF804CD6C
:100540004FEA40024FEA41037FEA226C18BF7FEA7C
:10055000236C11D001B052EA530C18BF90EA010F7E
:1005600058BFB2EB030088BFC81738BF6FEAE1700D
:1005700018BF40F0010070477FEA226C02D15FEAA9
:10058000402C05D17FEA236CE4D15FEA412CE1D015
:100590005DF8040B704700BF844608466146FFE7DC
:1005A0000FB5FFF7C9FF002848BF10F1000F0FBDBE
:1005B0004DF808EDFFF7F4FF0CBF012000205DF8B7
:1005C00008FB00BF4DF808EDFFF7EAFF34BF01203C
:1005D00000205DF808FB00BF4DF808EDFFF7E0FFD5
:1005E00094BF012000205DF808FB00BF4DF808ED26
:1005F000FFF7D2FF94BF012000205DF808FB00BF89
:100600004DF808EDFFF7C8FF34BF012000205DF86A
:1006100008FB00BF4FEA4002B2F1FE4F0FD34FF08C
:100620009E03B3EB12620DD94FEA002343F000435F
:1006300010F0004F23FA02F018BF404270474FF00D
:100640000000704712F1610F01D1420205D110F094
:10065000004008BF6FF0004070474FF00000704747
:100660005400520049004E0041004D004900430033
:1006700020004D006F00740069006F006E002000C4
:1006800043006F006E00740072006F006C002E005B
:1006900054004D004300200043004400430020006C
:1006A0004400450056002E0009024300020100C02C
:1006B00032090400000102020100052400100105B6
:1006C000240100010424020205240600010705821A
:1006D000030800FF09040100020A000000070503E7
:1006E00002400000070581024000000004030904E5
:1006F00026035400720069006E0061006D006900FD
:1007000063004D006F00740069006F006E002000F0
:10071000430074006C0000005515AC6A004001C035
:10072000ABEA57956B7FD87EB87DA07C8F7B857AAE
:10073000827985780878147726763D7559747B73AD
:10074000A172367264719670CC6F076F456EE66D5C
:100750002A6D726CBE6B0D6B5F6AB5696169BB68AF
:1007600019687967DC664266AB656065CC643B649A
:10077000AD63206396620F62CB614761C4604460E1
:10078000C65F495FCE5E925E1A5EA45D2F5DBD5C62
:100790004B5CDC5BA55B385BCC5A625AF9599259C9
:1007A0002C59F95895583358D15771571257B45698
:1007B0000000C90092015B022403ED03B6047F052B
:1007C00048061107D907A2086A09330AFB0AC40BB5
:1007D0008C0C540D1C0EE30EAB0F72103A1101126B
:1007E000C8128F1355141C15E215A8166E1733186E
:1007F000F918BE19821A471B0B1CCF1C931D571EDC
:100800001A1FDD1F9F2061212322E522A6236724D2
:100810002825E825A82667272628E528A329612A70
:100820001F2BDC2B992C552D112ECC2E872F4130D0
:10083000FB30B5316E322633DF3396344D35043616
:10084000BA366F372438D9388C39403AF23AA53B5A
:10085000563C073DB83D683E173FC53F73402141B8
:10086000CE417A422543D0437A442445CD4575464E
:100870001C47C34769480F49B449584AFB4A9D4B36
:100880003F4CE04C814D204EBF4E5D4FFB4F97508B
:100890003351CE51685202539B533254C954605560
:1008A000F5558A561D57B0574258D3586459F359D5
:1008B000825A0F5B9C5B285CB35C3E5DC75D4F5EFC
:1008C000D75E5D5FE35F6860EB606E61F0617162EF
:1008D000F1627063EE636C64E8646365DD655666BF
:1008E000CF664667BC673268A66819698B69FD697F
:1008F0006D6ADC6A4A6BB76B236C8E6CF86C616D49
:10090000C96D306E966EFB6E5E6FC16F2270837024
:10091000E27040719D71F9715472AE7207735E732B
:10092000B5730A745F74B27404755575A575F37563
:1009300041768D76D87622776B77B377FA773F78E2
:100940008478C77809794A798979C879057A417AAA
:100950007C7AB67AEE7A267B5C7B917BC57BF87BD2
:10096000297C597C887CB67CE37C0E7D397D627D58
:10097000897DB07DD57DFA7D1D7E3E7E5F7E7E7E4B
:100980009C7EB97ED57EEF7E097F217F377F4D7FAC
:10099000617F747F867F977FA67FB47FC17FCD7F85
:1009A000D87FE17FE97FF07FF57FF97FFD7FFE7FD4
:1009B0000010161B2023272A2D30323537393B3DB6
:1009C0004041434547494B4C4E505153545657595B
:1009D0005A5B5D5E60616263656667686A6B6C6DD9
:1009E0006E707172737475767778797A7B7C7D7EA0
:1009F00080808182838485868788898A8B8C8D8E8E
:100A00008F9090919293949596969798999A9B9B94
:100A10009C9D9E9FA0A0A1A2A3A3A4A5A6A7A7A8B2
:100A2000A9AAAAABACADADAEAFB0B0B1B2B2B3B4DF
:100A3000B5B5B6B7B7B8B9B9BABBBBBCBDBDBEBF1B
:100A4000C0C0C1C1C2C3C3C4C5C5C6C7C7C8C9C960
:100A5000CACBCBCCCCCDCECECFD0D0D1D1D2D3D3AC
:100A6000D4D4D5D6D6D7D7D8D9D9DADADBDBDCDD02
:100A7000DDDEDEDFE0E0E1E1E2E2E3E3E4E5E5E65E
:100A8000E6E7E7E8E8E9EAEAEBEBECECEDEDEEEEC1
:100A9000EFF0F0F1F1F2F2F3F3F4F4F5F5F6F6F726
:100AA000F7F8F8F9F9FAFAFBFBFCFCFDFDFEFEFF96
:100AB0000000000001020304010203040607080904
:100AC0000204060836303356322E3039000000005A
:100AD000D100000040000000FB070000FF070000FD
:100AE00000080000010000000200000005000000F6
:100AF0000300000004000000C40A01080B0C0D0AEA
:100B00000E0F09000000004001000000000400403A
:100B1000010101010101010001000000A00000002D
:100B200000127A000048004000C2010000000800E6
:100B3000EC06010804000000F00601082600000091
:100B4000D400002032000000080100201A0000003C
:100B5000A806010843000000C000002012000000A9
:100B6000AD930008B1910008FD8F000811900008B6
:100B7000159000087590000899900008A191000850
:100B8000919100086D9100080000000040000000F5
:100B900012011001020000403C2A0000020801027C
:100BA00003010000320354004D0043004D002D00AE
:100BB000300030003000300020002800760069004E
:100BC00072007400750061006C00200043004F004B
:100BD0004D002900200000001A0354004D0043007E
:100BE0004D003000300030003000000000000000F8
:100BF00000000000FD8E0008E5D10008E5D10008E6
:100C0000E5D10008E5D10008E5D10008E5D10008EC
:100C1000E5D10008E5D1000801930008E5D10008FE
:100C2000E5D10008E5D10008E5D100080401000085
:100C3000E5D10008D98F0008E5D10008E5D100080A
:100C4000E5D10008E5D10008E5D10008E5D10008AC
:100C5000F18F000801000000010000000100000009
:040000050800410CA2
:00000001FF
